:08000000E827040002000000E3
:04000C00D24C0000D2
:10001000624C00002A4C00009A4C0000D24C0000B8
:10002000D24C0000D24C0000D24C0000D24C000058
:10003000D24C0000D24C0000D24C0000D24C000048
:10004000D24C0000D24C0000A44E0000D24C000064
:10005000D24C0000064D0000D24C0000D24C0000F3
:10006000D24C0000D24C0000D24C0000D24C000018
:10007000D24C0000D24C0000D24C0000D24C000008
:10008000D24C0000D24C0000D24C0000D24C0000F8
:10009000D24C0000D24C0000D24C0000D24C0000E8
:1000A000384E0000D24C0000D24C0000D24C000070
:1000B000D24C0000D24C0000D24C0000D24C0000C8
:1000C000D24C0000D24C0000D24C0000D24C0000B8
:1000D000D24C0000D24C0000D24C0000D24C0000A8
:1000E000D24C0000D24C0000D24C0000D24C000098
:1000F000D24C00008A5A0000D24C0000D24C0000C2
:10010000D24C0000D24C0000D24C0000D24C000077
:10011000D24C0000D24C0000D24C0000D24C000067
:10012000D24C0000D24C0000D24C0000BA4B000070
:10013000F24B0000D24C0000D24C0000D24C000028
:10014000D24C0000D24C0000D24C0000D24C000037
:10015000D24C0000D24C0000D24C0000D24C000027
:10016000D24C0000D24C0000D24C0000D24C000017
:10017000D24C0000D24C0000D24C0000D24C000007
:10018000D24C0000D24C0000D24C0000D24C0000F7
:10019000D24C0000D24C0000D24C0000D24C0000E7
:1001A000D24C0000D24C0000D24C0000D24C0000D7
:1001B000D24C0000D24C0000D24C0000D24C0000C7
:1001C000D24C0000D24C0000D24C0000D24C0000B7
:1001D000D24C0000D24C0000D24C0000D24C0000A7
:1001E000D24C0000D24C0000D24C0000D24C000097
:1001F000D24C0000D24C0000D24C0000D24C000087
:100400003220EF00C3202000008041001040BA00DD
:100410000160EF00000006000A0D000052650000B8
:1004200061640000436F00006E66000069670000B1
:1004300045450000507200006F6D0000204500002F
:10044000727200006F72000028730000293A0000E9
:100450000A0D0000000000003220EF00832320007E
:10046000008041001040BA000160EF00000006006B
:10047000254C0000583A000020250000327800008A
:10048000202100003D20000025320000780A0000F5
:100490000D0000003220EF006325200000804100A5
:1004A0001040BA000160EF00000006004368000041
:1004B000656300006B730000756D00002052000042
:1004C000656100006420000025320000782C0000E7
:1004D00020430000616C0000637500006C61000047
:1004E000746500006420000025320000780A0000D6
:1004F0000D0000003220EF00632820000080410042
:100500001040BA000160EF0000000600202000004B
:10051000204300006F6E0000666900006720000045
:100520005361000076650000642000002020000078
:10053000000000003220EF00632A2000008041000C
:100540001040BA000160EF0000000600436F000099
:100550006E660000696700002053000061760000AD
:10056000656400000A0D0000000000003220EF006A
:10057000232C2000008041001040BA000160EF00F1
:1005800000000600537400006F7200006520000038
:1005900046610000637400006F7200007920000063
:1005A000446500006661000075740000732000005F
:1005B00046610000696C0000656400000A0D0000DF
:1005C000000000003220EF00E32E200000804100F8
:1005D0001040BA000160EF00000006005265000004
:1005E000616400002045000045500000726F00006B
:1005F0006D20000046610000696C00006564000029
:100600000A0D0000000000003220EF00033120003E
:10061000008041001040BA000160EF0000000600B9
:10062000537400006F7200006520000044650000F4
:1006300066610000757400007320000046610000D0
:10064000696C0000656400000A0D000000000000F5
:100650003220EF00430320008301500005003100E9
:1006600043342000008041001040BA000160EF00D8
:100670000000060040342000838141008081410059
:100680001380BA00000006000A0D2500446F4C00DC
:100690004C6F5800616420005072250065734C0057
:1006A00065745800202020002532250078204C0059
:1006B0002532580078202000253263007820680019
:1006C000254C650058206300254C6B0058207300B2
:1006D000254C750058206D00254C3D005820250004
:1006E000254C320058205800254C000058200000AE
:1006F0003220EF0023032000830150000500310069
:1007000043392000008041001040BA000160EF0032
:1007100000000600403920008381410080814100B3
:100720001380BA0000000600446F25004C6F3200B1
:1007300061647800507220006573210065743D008B
:100740003A20200043204100256463002C207400DF
:1007500050206900256476002C2865006B3D200040
:10076000254C43005829610020426D00616420003F
:10077000202D2500205032007265640073650A0048
:1007800074200D00436100006D2000003220EF0056
:10079000230220008301500005003100233E200089
:1007A000008041001040BA000160EF000000060028
:1007B000203E200083814100808141001380BA00E7
:1007C00000000600446F6F004C6F20006164500011
:1007D0005072720065736500657473003A2065009D
:1007E00043207400256420002C20660050206F00F8
:1007F000256475002C286E006B3D6400254C0A00B2
:1008000058290D00204E00003220EF002303200065
:1008100083015000050031000342200000804100A8
:100820001040BA000160EF00000006000042200006
:1008300083814100808141001380BA0000000600DE
:10084000446F6B004C6F73006164750050726D00F3
:1008500065732000657425003A203200432058005B
:10086000256420002C20210050203D00256420001C
:100870002C2843006B3D6100254C6C005829630017
:100880002042200061642500202D320020505800B5
:1008900072650A0073650D00742000006368000033
:1008A000656300003220EF00230320008301500025
:1008B00005003100E3462000008041001040BA00EE
:1008C0000160EF0000000600E04620008381410047
:1008D000808141001380BA0000000600446F2500AB
:1008E0005265320061647800507220006573210007
:1008F00065743D003A2020004320410025646300D8
:100900002C20740050206900256476002C28650096
:100910006B3D2000254C43005829610020426D00AA
:1009200061642000202D2500205032007265640093
:1009300073650A0074200D00436100006D20000003
:100940003220EF0023022000830150000500310017
:10095000C34B2000008041001040BA000160EF004E
:1009600000000600C04B20008381410080814100CF
:100970001380BA0000000600446F6F00526520002B
:100980006164500050727200657365006574730095
:100990003A20650043207400256420002C20660066
:1009A00050206F00256475002C286E006B3D64009C
:1009B000254C0A0058290D00204E00003220EF007F
:1009C000230320008301500005003100A34F2000C5
:1009D000008041001040BA000160EF0000000600F6
:1009E000A04F200083814100808141001380BA0024
:1009F00000000600446F6B0052657300616475006F
:100A000050726D0065732000657425003A20320035
:100A100043205800256420002C20210050203D0058
:100A2000256420002C2843006B3D6100254C6C00A0
:100A3000582963002042200061642500202D3200E7
:100A40002050580072650A0073650D007420000084
:100A500063680000656300003220EF00030220009D
:100A600083015000050031008354200000804100C4
:100A70001040BA000160EF00000006008054200022
:100A800083814100808141001380BA00000006008C
:100A90004C6F650063206E0025327400782C2000B6
:100AA000205043006F72610074206D002564650062
:100AB0002C5072007265610073652500742032004D
:100AC000256464002C200A0043750D00727200003A
:100AD0003220EF00C30220008301500005003100E6
:100AE00043582000008041001040BA000160EF0030
:100AF00000000600405820008381410080814100B1
:100B00001380BA00000006005361200076652500BE
:100B100020254C00327858002025200032786300D0
:100B2000202568004C586500202563004C586B0058
:100B3000202573004C58750020256D004C583D0051
:100B4000202525004C583200202558004C580A001A
:100B500020250D004C580000202500004C580000B6
:100B60003220EF00C35B2000008041001040BA003B
:100B70000160EF0000000600536F00006E79000076
:100B800020450000564900002D440000333000008D
:100B90002020000020200000202000002000000075
:100BA0003220EF00C35D2000008041001040BA00F9
:100BB0000160EF0000000600536F00006E79000036
:100BC00020450000564900002D440000333000004D
:100BD0002F440000333100002020000020000000DE
:100BE0003220EF00C35F2000008041001040BA00B7
:100BF0000160EF0000000600566100006464000020
:100C0000696F000020410000646400002D61000055
:100C10002D430000616D0000202000002000000036
:100C20003220EF00C3612000008041001040BA0074
:100C30000160EF0000000600536F00006E790000B5
:100C400020450000564900002D44000031300000CE
:100C500030200000202000002020000020000000A4
:100C60003220EF00C3632000008041001040BA0032
:100C70000160EF00000006005641000044440000FF
:100C8000494F000020480000442D0000313800008A
:100C90002020000020200000202000002000000074
:100CA0003220EF00C3652000008041001040BA00F0
:100CB0000160EF0000000600536F00006E79000035
:100CC00020450000564900002D4400003730000048
:100CD0002020000020200000202000002000000034
:100CE0003220EF00C3672000008041001040BA00AE
:100CF0000160EF0000000600536F00006E790000F5
:100D000020420000524300002D330000303000002C
:100D100020200000202000002020000020000000F3
:100D20003220EF00C3692000008041001040BA006B
:100D30000160EF0000000600536F00006E790000B4
:100D400020420000524300002D48000037300000D0
:100D500030200000202000002020000020000000A3
:100D60003220EF00C36B2000008041001040BA0029
:100D70000160EF0000000600536F00006E79000074
:100D800020420000524300002D5A0000373000007E
:100D90003020000020200000202000002000000063
:100DA0003220EF00C36D2000008041001040BA00E7
:100DB0000160EF0000000600536F00006E79000034
:100DC00020420000524300002D5A0000333300003F
:100DD0003020000020200000202000002000000023
:100DE0003220EF00C36F2000008041001040BA00A5
:100DF0000160EF0000000600536F00006E790000F4
:100E000020450000564900002D48000044310000F4
:100E100020200000202000002020000020000000F2
:100E20003220EF00C3712000008041001040BA0062
:100E30000160EF0000000600506100006E610000DC
:100E4000736F00006E6900006320000041570000CE
:100E50002D48000045310000303000002000000027
:100E60003220EF00C3732000008041001040BA0020
:100E70000160EF000000060043650000696C00009F
:100E8000696E0000675600004945000057200000C9
:100E90002020000020200000202000002000000072
:100EA0003220EF00C3752000008041001040BA00DE
:100EB0000160EF0000000600436100006E6F00005B
:100EC0006E200000564300002D4300003530000026
:100ED000692F000072200000202000002000000088
:100EE0003220EF00C3772000008041001040BA009C
:100EF0000160EF0000000600436100006E6F00001B
:100F00006E200000425500002D34000035480000DE
:100F100020200000202000002020000020000000F1
:100F20003220EF00C3792000008041001040BA0059
:100F30000160EF0000000600436100006E6F0000DA
:100F40006E200000425500002D35000030480000A2
:100F500020200000202000002020000020000000B1
:100F60003220EF00C37B2000008041001040BA0017
:100F70000160EF0000000600556E00006B6E00007F
:100F80006F7700006E200000436100006D65000077
:100F900072610000202000002020000020000000DE
:100FA0003220EF00C37D2000008041001040BA00D5
:100FB0000160EF000000060045560000492D0000CA
:100FC00044330000302000002020000020200000DA
:100FD000000000003220EF00637F2000008041000D
:100FE0001040BA000160EF00000006004556000006
:100FF000492D000044330000302F0000443300002E
:1010000031200000000000003220EF0003812000AA
:10101000008041001040BA000160EF0000000600AF
:1010200041640000642D0000612D00004361000058
:101030006D20000020200000000000003220EF00A2
:10104000A3822000008041001040BA000160EF0040
:101050000000060045560000492D00004431000004
:1010600030300000202000002020000000000000A0
:101070003220EF0043842000008041001040BA007D
:101080000160EF0000000600484400002D31000020
:101090003820000020200000202000002020000038
:1010A000000000003220EF00E385200000804100B6
:1010B0001040BA000160EF00000006004556000035
:1010C000492D00004437000030200000202000009F
:1010D00020200000000000003220EF008387200065
:1010E000008041001040BA000160EF0000000600DF
:1010F00042520000432D0000333000003020000039
:101100002020000020200000000000003220EF001E
:1011100023892000008041001040BA000160EF00E8
:101120000000060042520000432D00004837000036
:1011300030300000202000002020000000000000CF
:101140003220EF00C38A2000008041001040BA0026
:101150000160EF000000060042520000432D000035
:101160005A3700003030000020200000202000000E
:10117000000000003220EF00638C2000008041005E
:101180001040BA000160EF0000000600425200006B
:10119000432D00005A3300003330000020200000AF
:1011A00020200000000000003220EF00038E20000D
:1011B000008041001040BA000160EF00000006000E
:1011C00045560000492D0000484400003120000031
:1011D0002020000020200000000000003220EF004E
:1011E000A38F2000008041001040BA000160EF0092
:1011F00000000600415700002D4800004531000066
:1012000030300000202000002020000000000000FE
:101210003220EF0043912000008041001040BA00CE
:101220000160EF000000060043650000696C0000EB
:10123000696E000067560000494500005720000015
:10124000000000003220EF00E39220000080410007
:101250001040BA000160EF00000006005643000095
:101260002D43000035300000692F0000722000007F
:1012700020200000000000003220EF0083942000B6
:10128000008041001040BA000160EF00000006003D
:10129000425500002D340000354800002020000099
:1012A0002020000020200000000000003220EF007D
:1012B00023962000008041001040BA000160EF003A
:1012C00000000600425500002D35000030480000A7
:1012D000202000002020000020200000000000004E
:1012E0003220EF00C3972000008041001040BA0078
:1012F0000160EF0000000600556E00006B6E0000FC
:101300006F7700006E2000002020000020200000E9
:10131000000000003220EF006399200000804100AF
:101320001040BA000160EF0000000600000000005D
:101330003220EF00439A2000008041001040BA00A4
:101340000160EF0000000600537900007374000094
:10135000656D000020430000616D00002049000021
:101360006E690000742000003A20000055730000F0
:101370006520000050720000657300006574000075
:1013800031340000000000003220EF00039D2000F7
:10139000008041001040BA000160EF00000006002C
:1013A0005379000073740000656D00002043000055
:1013B000616D0000204900006E690000742000008B
:1013C0003A200000486F00006D65000020430000D7
:1013D000616D0000657200006120000000000000E7
:1013E0003220EF00C39F2000008041001040BA006F
:1013F0000160EF00000006005072000065730000FD
:1014000065740000204C00006F63000061740000F0
:10141000696F00006E3A0000203100002D36000098
:10142000204900006E430000616D00002C37000071
:101430002D310000342000004C6F0000636100007B
:101440006C0000003220EF00E3A220000080410089
:101450001040BA000160EF0000000600507200006A
:101460006573000065740000204C00006F6300008D
:1014700061740000696F00006E3A000020310000C6
:101480002D310000342000004C6F0000636100002B
:101490006C0000003220EF0063A5200000804100B6
:1014A0001040BA000160EF0000000600486F000025
:1014B0007374000020530000657200006961000031
:1014C0006C200000496E000070750000743A000046
:1014D000204500006E610000626C00006564000041
:1014E000000000003220EF00E3A720000080410050
:1014F0001040BA000160EF0000000600486F0000D5
:1015000073740000205300006572000069610000E0
:101510006C200000496E000070750000743A0000F5
:101520002044000069730000616200006C650000E7
:10153000640000003220EF0063AA20000080410018
:101540001040BA000160EF00000006005365000083
:1015500072690000616C00002045000063680000B3
:101560006F3A0000204500006E610000626C0000D0
:1015700065640000000000003220EF0083AC200012
:10158000008041001040BA000160EF00000006003A
:101590005365000072690000616C00002045000086
:1015A000636800006F3A0000204400006973000087
:1015B000616200006C650000640000003220EF00F2
:1015C000A3AE2000008041001040BA000160EF008F
:1015D000000006005365000072690000616C0000A5
:1015E000204900006E6600006F3A0000204F0000A6
:1015F0006E0000003220EF0063B020000080410048
:101600001040BA000160EF000000060053650000C2
:1016100072690000616C0000204900006E660000E5
:101620006F3A0000204F00006666000000000000D6
:101630003220EF0043B22000008041001040BA0089
:101640000160EF0000000600546100006C6C0000B7
:10165000792000004C650000766500006C3A0000BF
:1016600020410000637400006976000065200000DE
:101670004869000067680000000000003220EF00A9
:10168000A3B42000008041001040BA000160EF00C8
:1016900000000600546100006C6C0000792000001E
:1016A0004C650000766500006C3A000020410000A7
:1016B0006374000069760000652000004C6F000034
:1016C000770000003220EF00E3B6200000804100E8
:1016D0001040BA000160EF0000000600486F0000F3
:1016E0006D6500002042000075740000746F0000FA
:1016F0006E3A00002044000069730000616200003F
:101700006C650000640000003220EF0003B9200087
:10171000008041001040BA000160EF0000000600A8
:10172000486F00006D6500002042000075740000E5
:10173000746F00006E3A0000204500006E610000EA
:10174000626C000065640000000000003220EF00C1
:1017500023BB2000008041001040BA000160EF0070
:101760000000060044690000616700006E6F000021
:101770007374000069630000204D00006F64000076
:10178000653A0000204F00006E0000003220EF009C
:1017900023BD2000008041001040BA000160EF002E
:1017A0000000060044690000616700006E6F0000E1
:1017B0007374000069630000204D00006F64000036
:1017C000653A0000204F000066660000000000003F
:1017D0003220EF0043BF2000008041001040BA00DB
:1017E0000160EF0000000600536500007269000010
:1017F000616C000020440000696100006720000067
:101800004D6F0000646500003A2000004F6E00003C
:10181000000000003220EF0063C120000080410082
:101820001040BA000160EF000000060053650000A0
:1018300072690000616C00002044000069610000D2
:10184000672000004D6F0000646500003A20000032
:101850004F660000660000003220EF0083C32000C6
:10186000008041001040BA000160EF000000060057
:10187000436100006D6500007261000020530000AC
:10188000656C000065630000742000006F6E00004E
:10189000203A0000204300006F6E000074720000C8
:1018A0006F6C000020410000000000003220EF00BB
:1018B00023C62000008041001040BA000160EF0004
:1018C00000000600436100006D65000072610000C9
:1018D00020530000656C0000656300007420000068
:1018E0006F6E0000203A0000204300006F6E000081
:1018F000747200006F6C00002042000000000000C5
:101900003220EF00C3C82000008041001040BA0020
:101910000160EF0000000600436100006D650000FB
:101920007261000020530000656C000065630000D8
:10193000742000006F6E00003A200000446900002F
:1019400073610000626C000065640000000000002C
:101950003220EF0043CB2000008041001040BA004D
:101960000160EF0000000600526500006D6F00008E
:1019700074650000204C0000696E00006B200000C0
:101980004D6F0000646500003A20000044750000BF
:10199000616C0000204D0000617300007465000060
:1019A000720000003220EF00E3CD200000804100F3
:1019B0001040BA000160EF00000006005265000010
:1019C0006D6F000074650000204C0000696E00001F
:1019D0006B2000004D6F0000646500003A2000009D
:1019E0004D6100007374000065720000203C00002F
:1019F0002D3E0000205300006C6100007665000061
:101A0000000000003220EF00E3D020000080410001
:101A10001040BA000160EF000000060044610000C1
:101A200074610000205300007769000074630000B7
:101A3000682000004D6F0000646500003A2000003F
:101A400045640000697200006F6C00000000000037
:101A50003220EF0043D32000008041001040BA0044
:101A60000160EF00000006004461000074610000A6
:101A700020530000776900007463000068200000B4
:101A80004D6F0000646500003A20000049530000DB
:101A900049530000000000003220EF0083D52000F1
:101AA000008041001040BA000160EF000000060015
:101AB0004461000074610000205300007769000059
:101AC00074630000682000004D6F00006465000032
:101AD0003A200000416E0000616C00006F6700005A
:101AE00057610000790000003220EF0003D8200089
:101AF000008041001040BA000160EF0000000600C5
:101B00004461000074610000205300007769000008
:101B100074630000682000004D6F000064650000E1
:101B20003A20000045780000747200006F6E0000DB
:101B3000000000003220EF0063DA20000080410046
:101B40001040BA000160EF00000006004461000090
:101B50007461000020530000776900007463000086
:101B6000682000004D6F0000646500003A2000000E
:101B70005573000065720000204400006566000097
:101B8000696E000065640000000000003220EF0074
:101B900023DD2000008041001040BA000160EF000A
:101BA0000000060044610000746100002053000042
:101BB0007769000074630000682000004D6F00002A
:101BC000646500003A200000446900007361000071
:101BD000626C000065640000000000003220EF002D
:101BE000A3DF2000008041001040BA000160EF0038
:101BF000000006005061000073730000204F0000D9
:101C00006E200000537400006174000075730000C2
:101C10003A2000004163000074690000766500000E
:101C2000000000003220EF00E3E1200000804100CE
:101C30001040BA000160EF00000006005061000093
:101C400073730000204F00006E20000053740000EA
:101C500061740000757300003A200000496E0000B6
:101C600061630000746900007665000000000000F8
:101C70003220EF0043E42000008041001040BA0011
:101C80000160EF0000000600506100007373000067
:101C90002052000065730000706F00006E7300003A
:101CA000652000005374000061740000757300002B
:101CB0003A200000506500006E640000696E00006C
:101CC000670000003220EF00E3E6200000804100C2
:101CD0001040BA000160EF000000060050610000F3
:101CE000737300002052000065730000706F0000E5
:101CF0006E730000652000005374000061740000E2
:101D0000757300003A200000496400006C65000013
:101D1000000000003220EF0063E920000080410055
:101D20001040BA000160EF000000060050610000A2
:101D300073730000204D00006F64000065200000F8
:101D400053740000617200007465000064000000BC
:101D50003220EF0043EB2000008041001040BA0029
:101D60000160EF0000000600506100007373000086
:101D7000204D00006F640000652000006E6F0000C1
:101D8000742000005374000061720000746500004C
:101D9000640000003220EF0063ED2000008041006D
:101DA0001040BA000160EF00000006005061000022
:101DB0006E2F0000546900006C7400002053000076
:101DC0007461000074750000733A00002041000047
:101DD0006374000069760000650000003220EF00A7
:101DE000A3EF2000008041001040BA000160EF0026
:101DF00000000600506100006E2F000054690000D2
:101E00006C740000205300007461000074750000C1
:101E1000733A000020490000646C00006500000077
:101E20003220EF00C3F12000008041001040BA00D2
:101E30000160EF00000006005A6F00006F6D0000A7
:101E4000205300007461000074750000733A0000B4
:101E50002041000063740000697600006500000006
:101E60003220EF00C3F32000008041001040BA0090
:101E70000160EF00000006005A6F00006F6D000067
:101E8000205300007461000074750000733A000074
:101E900020490000646C0000650000003220EF0063
:101EA000A3F52000008041001040BA000160EF005F
:101EB000000006004C6F0000636100006C20000011
:101EC000636100006D650000726100007320000016
:101ED000666F0000756E0000643A0000204E00003E
:101EE0006F0000003220EF00E3F720000080410087
:101EF0001040BA000160EF00000006004C6F0000C7
:101F0000636100006C200000636100006D650000EB
:101F10007261000073200000666F0000756E0000A3
:101F2000643A0000205900006573000000000000C2
:101F30003220EF0043FA2000008041001040BA0038
:101F40000160EF0000000600436100006D650000C5
:101F500072610000204300006F6E00007472000088
:101F60006F6C00003A2000004C6F000063610000BD
:101F70006C0000003220EF0063FC20000080410074
:101F80001040BA000160EF0000000600436100004D
:101F90006D65000072610000204300006F6E00005C
:101FA000747200006F6C00003A200000526500005F
:101FB0006D6F000074650000000000003220EF002B
:101FC000A3FE2000008041001040BA000160EF0035
:101FD00000000600526500006D6F0000746500008F
:101FE000284D000061730000746500007229000034
:101FF000204C0000696E00006B200000416300006F
:102000007469000076650000000000003220EF00D7
:1020100023012100008041001040BA000160EF0060
:1020200000000600526500006D6F0000746500003E
:10203000284D0000617300007465000072290000E3
:10204000204C0000696E00006B2000006E6F0000E5
:102050007420000041630000746900007665000090
:10206000000000003220EF00E30321000080410067
:102070001040BA000160EF00000006005265000049
:102080006D6F000074650000285300006C61000053
:1020900076650000292000004C6900006E6B00008E
:1020A00020410000637400006976000065000000B4
:1020B0003220EF0043062100008041001040BA00AA
:1020C0000160EF0000000600526500006D6F000027
:1020D00074650000285300006C6100007665000004
:1020E000292000004C6900006E6B0000206E00008B
:1020F0006F740000204100006374000069760000E6
:10210000650000003220EF00E3082100008041005C
:102110001040BA000160EF0000000600436F0000AD
:102120006E740000726F00006C6C0000657200003D
:10213000205300007461000074750000733A0000C1
:1021400020520000656D00006F7400006500000003
:102150003220EF00430B2100008041001040BA0004
:102160000160EF0000000600436F00006E74000085
:10217000726F00006C6C000065720000205300005C
:102180007461000074750000733A0000204C000078
:102190006F630000616C0000000000003220EF005F
:1021A000A30D2100008041001040BA000160EF0043
:1021B00000000600507200006F67000072610000AE
:1021C0006D2000004D6F0000646500003A200000A3
:1021D00041630000746900007665000000000000A3
:1021E0003220EF00C30F2100008041001040BA00F0
:1021F0000160EF0000000600507200006F670000F1
:10220000726100006D2000004D6F000064650000E9
:102210003A200000496400006C65000000000000E6
:102220003220EF00C3112100008041001040BA00AD
:102230000160EF000000060052580000205300002B
:1022400074610000746500003A200000584F0000DF
:1022500046460000000000003220EF0083132100FA
:10226000008041001040BA000160EF00000006004D
:102270005258000020530000746100007465000093
:102280003A200000584F00004E0000003220EF00BE
:1022900023152100008041001040BA000160EF00CA
:1022A0000000060054580000205300007461000034
:1022B000746500003A200000584F000046460000B8
:1022C000000000003220EF00E316210000804100F2
:1022D0001040BA000160EF000000060054580000F2
:1022E0002053000074610000746500003A20000073
:1022F000584F00004E0000003220EF0083182100EC
:10230000008041001040BA000160EF0000000600AC
:10231000505400005A200000536500006E64000015
:102320002053000074610000746500003A20000032
:10233000506500006E640000696E000067000000D8
:102340003220EF00C31A2100008041001040BA0083
:102350000160EF0000000600505400005A20000009
:10236000536500006E64000020530000746100009B
:10237000746500003A200000496400006C650000AC
:10238000000000003220EF00E31C2100008041002B
:102390001040BA000160EF0000000600446F00002A
:1023A000466900006E64000041630000746900002B
:1023B00076650000507200006573000065740000CF
:1023C00073200000506F0000727400002025000090
:1023D0006420000062610000640A00000D0000003B
:1023E0003220EF000302200083015000050031007D
:1023F000C3202100008041001040BA000160EF00BE
:1024000000000600C020210083814100808141003E
:102410001380BA00000006000A0D7200446F6500C8
:10242000466973006E64650041637400746920003E
:1024300076653100507220006573250065744C008C
:102440007320580043613A006D202000256420006D
:102450003A2020002D5000003220EF00832321007D
:10246000008041001040BA000160EF00000006004B
:102470000A0D0000553400005F490000535200006F
:1024800020250000325800002025000032580000AE
:10249000202500003258000020250000325800009E
:1024A0002025000032580000000000003220EF001C
:1024B00023262100008041001040BA000160EF0097
:1024C000000006002043000043550000204D00009E
:1024D0006F64000065200000416300007469000023
:1024E00076650000200000003220EF000328210064
:1024F000008041001040BA000160EF0000000600BB
:10250000553400005F4200003020000049530000B5
:10251000522D00004572000072200000253200009C
:10252000582000002532000058200000253200000D
:102530005820000025320000582000005B250000D4
:10254000325800005D0A00000D0000003220EF004C
:10255000232B2100008041001040BA000160EF00F1
:1025600000000600553400005F42000031200000EA
:1025700049530000522D00004572000072200000F7
:1025800025320000582000002532000058200000AD
:1025900025320000582000005B2500003258000062
:1025A0005D20000025320000580A00000D000000E8
:1025B0003220EF00432E2100008041001040BA007D
:1025C0000160EF0000000600553800005F42000087
:1025D0003220000049530000522D000045720000D7
:1025E0007220000025320000582000002532000033
:1025F000582000005B250000325800005D200000DC
:10260000253200005820000025320000580A000042
:102610000D0000003220EF006331210000804100F6
:102620001040BA000160EF0000000600524D0000AB
:1026300054200000506700006D2000004D6F000026
:102640006465000020250000750A00000D000000F0
:102650003220EF0043332100008041001040BA00D7
:102660000160EF0000000600205200004D54000001
:1026700020500000726F000067720000616D000062
:10268000204D00006F640000652000000000000085
:102690003220EF0043352100008041001040BA0095
:1026A0000160EF0000000600553400005F420000AA
:1026B0003320000049530000522D000045720000F5
:1026C0007220000025320000582000005B25000029
:1026D000325800005D200000253200005820000024
:1026E000253200005820000025320000582000004C
:1026F0000A0D0000000000003220EF0083382100A6
:10270000008041001040BA000160EF0000000600A8
:10271000553400005F42000034200000495300009F
:10272000522D000045720000722000005B25000061
:10273000325800005D2000002532000058200000C3
:1027400025320000582000002532000058200000EB
:1027500025320000582000000A0D00000000000093
:102760003220EF00C33B2100008041001040BA003E
:102770000160EF00000006000A0D00004E6F00002F
:102780004C6900006E6B0000000000003220EF007A
:10279000233D2100008041001040BA000160EF009D
:1027A000000006004E6F000020430000616D000035
:1027B0006572000061200000536500006C65000038
:1027C0006374000065640000000000003220EF0028
:1027D000233F2100008041001040BA000160EF005B
:1027E000000006000A0D0000576900006E6400003A
:1027F0006F770000205300006875000074640000CB
:102800006F7700006E2C0000204D00006178000002
:102810002825000075290000204300007572000083
:10282000726500006E740000282500007529000004
:10283000000000003220EF006342210000804100D0
:102840001040BA000160EF00000006000A0D000011
:102850002825000075290000536500006E64000003
:10286000204C0000696E00006B20000044610000F5
:10287000746100002025000032780000202500004F
:10288000327800002025000032780000202500006A
:1028900032780000000000003220EF000302200028
:1028A0008301500005003100834621000080410073
:1028B0001040BA000160EF000000060080462100D1
:1028C00083814100808141001380BA00000006002E
:1028D0000A0D78004F752000745125002046320003
:1028E000756C78006C2C2000206D2500657332001B
:1028F000736178006765200020642500726F3200E4
:1029000070707800656429002028000025320000DE
:102910003220EF0023032000830150000500310026
:10292000434A2100008041001040BA000160EF00DE
:1029300000000600404A210083814100808141005F
:102940001380BA00000006000A0D2500283132006D
:10295000294E78006F202000436125006D6532000C
:102960007261780020532900656C20006563530074
:1029700074657400642C6100206D740065737500CB
:10298000736173006765460020646C00726F6100BC
:10299000707067006564200020282500253234000F
:1029A00078204C0025327800782000003220EF009B
:1029B000230320008301500005003100234F210034
:1029C000008041001040BA000160EF0000000600E6
:1029D000204F210083814100808141001380BA0093
:1029E000000006000A0D250028323200294E78002A
:1029F0006F202000436125006D6532007261780010
:102A000020532900656C20006563530074657400D1
:102A1000642C6100206D7400657375007361730030
:102A20006765460020646C00726F6100707067001B
:102A300065642000202825002532340078204C00D1
:102A400025327800782000003220EF004303200078
:102A50008301500005003100035421000080410033
:102A60001040BA000160EF00000006000054210091
:102A700083814100808141001380BA00000006007C
:102A80000A0D250044514C00204D75006573290046
:102A90007361200067654800204469006174670025
:102AA00061206800282528003278250020254C0068
:102AB0003278750020252900327820002025570023
:102AC0003278690029206E00496E640064656F00E9
:102AD000782877002575280029202500436F750088
:102AE000756E2900742800003220EF000358210081
:102AF000008041001040BA000160EF0000000600B5
:102B00000A0D0000507200006F6300006573000042
:102B1000735200006D740000427400006E280000C3
:102B200029200000636D00006420000025320000B1
:102B300078200000253200007820000025320000B7
:102B40007820000025320000780000003220EF00DD
:102B5000235B2100008041001040BA000160EF00BB
:102B60000000060020200000204D0000616E0000E3
:102B7000756100006C200000466F00006375000066
:102B80007320000020200000000000003220EF0031
:102B9000235D2100008041001040BA000160EF0079
:102BA00000000600202000002020000041750000E9
:102BB000746F0000204600006F6300007573000012
:102BC0002020000020200000000000003220EF0044
:102BD000235F2100008041001040BA000160EF0037
:102BE00000000600204E00006F74000020730000FB
:102BF00075700000706F0000727400006564000062
:102C00002020000020200000000000003220EF0003
:102C100023612100008041001040BA000160EF00F4
:102C20000000060020200000202000004661000077
:102C300073740000204600006F630000757300008D
:102C40002020000020200000000000003220EF00C3
:102C500023632100008041001040BA000160EF00B2
:102C60000000060020200000466F00006375000091
:102C700073200000506F000073200000256C0000DE
:102C8000750000003220EF00E36421000080410065
:102C90001040BA000160EF0000000600204600006E
:102CA0006173000074200000466F0000637500002F
:102CB00073200000457800006974000020200000A7
:102CC000000000003220EF00E36621000080410098
:102CD0001040BA000160EF00000006002043000031
:102CE00043550000204D00006F6400006520000087
:102CF0004163000074690000766500002020000038
:102D0000000000003220EF00E36821000080410055
:102D10001040BA000160EF0000000600204D0000E6
:102D2000616E0000756100006C20000057680000B3
:102D30006974000065200000426100006C20000002
:102D4000000000003220EF00E36A21000080410013
:102D50001040BA000160EF0000000600417500005D
:102D6000746F00002057000068690000746500005F
:102D700020420000616C0000616E0000636500008D
:102D8000000000003220EF00E36C210000804100D1
:102D90001040BA000160EF0000000600204F000064
:102DA0006E65000020500000757300006820000070
:102DB00057420000202000002020000020200000BA
:102DC000000000003220EF00E36E2100008041008F
:102DD0001040BA000160EF000000060042610000F0
:102DE000636B00006C6900006768000074200000DD
:102DF000436F00006D700000206E00002F61000026
:102E0000000000003220EF00E3702100008041004C
:102E10001040BA000160EF00000006002020000012
:102E2000204D0000616E0000756100006C20000004
:102E3000497200006973000020200000202000007B
:102E4000000000003220EF00E3722100008041000A
:102E50001040BA000160EF000000060020200000D2
:102E600020410000757400006F20000049720000CE
:102E700069730000202000002020000020200000B6
:102E8000000000003220EF00E374210000804100C8
:102E90001040BA000160EF0000000600426100002F
:102EA000636B00006C69000067680000742000001C
:102EB000436F00006D700000204F00006666000048
:102EC000000000003220EF00E37621000080410086
:102ED0001040BA000160EF000000060042610000EF
:102EE000636B00006C6900006768000074200000DC
:102EF000436F00006D700000204F00006E20000046
:102F0000000000003220EF00E37821000080410043
:102F10001040BA000160EF00000006002020000011
:102F2000204800006F6D0000652000004361000034
:102F30006D6500007261000020200000202000006C
:102F4000000000003220EF00E37A21000080410001
:102F50001040BA000160EF000000060020200000D1
:102F600020200000436100006D65000072610000D8
:102F70002025000064200000202000002020000008
:102F8000200000003220EF00E37C2100008041009F
:102F90001040BA000160EF00000006004E6F000014
:102FA00020430000616D0000657200006120000098
:102FB000466F0000756E00006420000020200000B5
:102FC000000000003220EF00E37E2100008041007D
:102FD0001040BA000160EF000000060042740000DB
:102FE0006E20000025640000206E00006F74000059
:102FF0002064000065660000696E000065640000E2
:10300000200000003220EF00E3802100008041001A
:103010001040BA000160EF0000000600496E000099
:10302000436100006D6500007261000020500000E7
:1030300072650000736500007420000025320000F6
:10304000640000003220EF00E38221000080410094
:103050001040BA000160EF000000060020200000D0
:1030600050720000657300006574000020250000A8
:1030700032640000000000003220EF008384210051
:10308000008041001040BA000160EF00000006001F
:103090002020000042610000642000005072000007
:1030A0006573000065740000202500003264000094
:1030B00020200000000000003220EF008386210065
:1030C000008041001040BA000160EF0000000600DF
:1030D000202000004E6F00002050000072650000AC
:1030E0007365000074200000253200006420000099
:1030F000200000003220EF006388210000804100A2
:103100001040BA000160EF0000000600202000001F
:103110004E6F0000742000006F6E00002050000011
:10312000726500007365000074200000202000001C
:10313000000000003220EF00638A2100008041007F
:103140001040BA000160EF000000060020200000DF
:103150002049000072690000733A00002025000039
:10316000730000003220EF00E38B2100008041005B
:103170001040BA000160EF000000060020200000AF
:1031800020490000726900007320000025730000D0
:10319000000000003220EF00638D2100008041001C
:1031A0001040BA000160EF0000000600202000007F
:1031B000204900007269000073200000256C0000A7
:1031C000750000003220EF00E38E210000804100F6
:1031D0001040BA000160EF0000000600202000004F
:1031E0004D610000782000005A6F00006F6D0000F4
:1031F00020250000750000003220EF0083902100A0
:10320000008041001040BA000160EF00000006009D
:10321000202000004D610000782000005061000077
:103220006E20000025750000000000003220EF0035
:1032300023922100008041001040BA000160EF009D
:1032400000000600202000004D61000078200000F2
:10325000546900006C740000202500007500000017
:103260003220EF00C3932100008041001040BA00DB
:103270000160EF0000000600202000002052000046
:103280006564000020470000616900006E200000B6
:103290004E2F000041200000202000000000000010
:1032A0003220EF00C3952100008041001040BA0099
:1032B0000160EF00000006002020000052650000C1
:1032C0006420000047610000696E00003E2000009D
:1032D00025640000000000003220EF0083972100E9
:1032E000008041001040BA000160EF0000000600BD
:1032F00020200000526500006420000047610000AB
:10330000696E00003E200000254C000064000000B3
:103310003220EF0043992100008041001040BA00A4
:103320000160EF00000006002020000020420000A5
:103330006C7500006520000047610000696E0000A8
:10334000204E00002F41000020200000000000005F
:103350003220EF00439B2100008041001040BA0062
:103360000160EF000000060020200000426C000019
:103370007565000020470000616900006E3E000096
:1033800020250000640000003220EF00039D210092
:10339000008041001040BA000160EF00000006000C
:1033A00020200000426C00007565000020470000EE
:1033B000616900006E3E0000202500004C640000A2
:1033C000000000003220EF00E39E21000080410059
:1033D0001040BA000160EF0000000600202000004D
:1033E0002044000065740000616900006C2000004A
:1033F0004E2F00004120000020200000202000006F
:10340000000000003220EF00E3A021000080410016
:103410001040BA000160EF0000000600202000000C
:103420004465000074610000696C00003E200000EB
:1034300025640000000000003220EF0083A221007C
:10344000008041001040BA000160EF00000006005B
:1034500020200000506500006465000073740000C7
:10346000616C00003E2000002564000000000000A8
:103470003220EF0043A42100008041001040BA0038
:103480000160EF0000000600202000002020000066
:1034900047610000696E0000204E00002F410000CF
:1034A000202000002020000020200000000000005C
:1034B0003220EF0043A62100008041001040BA00F6
:1034C0000160EF0000000600204700006169000075
:1034D0006E3E000025730000000000003220EF0067
:1034E000A3A72100008041001040BA000160EF0056
:1034F00000000600204900007269000073200000EF
:1035000047610000696E00003E2500007564000000
:10351000420000003220EF0063A92100008041003A
:103520001040BA000160EF000000060020470000D4
:10353000616900006E3E000020250000750000005B
:103540003220EF00C3AA2100008041001040BA00E1
:103550000160EF000000060020410000574200001B
:10356000204D00006F6400006520000041630000F2
:103570007469000076650000202000000000000053
:103580003220EF00C3AC2100008041001040BA009F
:103590000160EF0000000600202000002020000055
:1035A0004972000069730000204E00002F410000A6
:1035B000202000002020000020200000000000004B
:1035C0003220EF00C3AE2100008041001040BA005D
:1035D0000160EF000000060020200000466F0000A0
:1035E0006375000073200000506F0000732000001E
:1035F0004E2F0000412000002020000000000000AD
:103600003220EF00C3B02100008041001040BA001A
:103610000160EF000000060020200000466F00005F
:1036200063750000732000004E65000061720000A9
:1036300020200000202000002020000000000000CA
:103640003220EF00C3B22100008041001040BA00D8
:103650000160EF000000060020200000466F00001F
:1036600063750000732000004661000072200000B6
:10367000202000002020000020200000000000008A
:103680003220EF00C3B42100008041001040BA0096
:103690000160EF000000060020410000757400008A
:1036A0006F20000049720000697300002041000093
:1036B00063740000697600006520000000000000CF
:1036C0003220EF00C3B62100008041001040BA0054
:1036D0000160EF0000000600205700006970000044
:1036E00065720000204100006374000069760000EC
:1036F00061740000656400002020000000000000EC
:103700003220EF00C3B82100008041001040BA0011
:103710000160EF000000060020200000486F00005C
:103720006D650000204400006973000061620000C4
:103730006C650000642000002020000000000000F4
:103740003220EF00C3BA2100008041001040BA00CF
:103750000160EF000000060020430000616E0000E1
:103760006F6E0000204900006D6700005374000078
:1037700061620000204F00004E20000000000000A9
:103780003220EF00C3BC2100008041001040BA008D
:103790000160EF000000060020430000616E0000A1
:1037A0006F6E0000204900006D6700005374000038
:1037B00061620000204F000046460000000000004B
:1037C0003220EF00C3BE2100008041001040BA004B
:1037D0000160EF00000006002020000020490000EA
:1037E0006E760000616C00006964000020430000F8
:1037F0006F64000065200000202000000000000031
:103800003220EF00C3C02100008041001040BA0008
:103810000160EF0000000600427400006E28000006
:1038200025320000782F000025750000292D0000AA
:103830004772000070310000200A00000D000000F7
:103840003220EF00C3C22100008041001040BA00C6
:103850000160EF000000060020200000504700003B
:103860004D2000004D6F0000646500002041000005
:1038700063740000697600006520000020000000ED
:103880003220EF00C3C42100008041001040BA0084
:103890000160EF0000000600506F00007765000037
:1038A000722000004F660000660A00000D00000054
:1038B0003220EF0043C62100008041001040BA00D2
:1038C0000160EF0000000600506F00007765000007
:1038D000722000004F6E00000A0D00000000000082
:1038E0003220EF00C3C72100008041001040BA0021
:1038F0000160EF0000000600466F000063750000E5
:10390000734D0000616E0000756100006C0A0000DC
:103910000D0000003220EF0063C92100008041004B
:103920001040BA000160EF0000000600466F000082
:103930006375000073410000757400006F0A000099
:103940000D0000003220EF00E3CA2100008041009A
:103950001040BA000160EF0000000600204E000099
:103960006F7400002073000075700000706F00001D
:103970007274000065640000202000002000000038
:103980003220EF00C3CC2100008041001040BA007B
:103990000160EF0000000600466100007374000043
:1039A000466F000063750000732000004F6E00003A
:1039B0000A0D0000000000003220EF0083CE21003D
:1039C000008041001040BA000160EF0000000600D6
:1039D0004661000073740000466F000063750000CC
:1039E000732000004F460000460A00000D00000052
:1039F0003220EF0043D02100008041001040BA0087
:103A00000160EF0000000600574200004D61000019
:103A10006E750000616C00000A0D000000000000DF
:103A20003220EF00C3D12100008041001040BA00D5
:103A30000160EF00000006005742000041750000E1
:103A4000746F00000A0D0000000000003220EF003B
:103A500023D32100008041001040BA000160EF0034
:103A600000000600204F00006E650000205000009E
:103A700075730000682000005742000020200000FD
:103A800020200000000000003220EF0003D52100BC
:103A9000008041001040BA000160EF000000060005
:103AA0004F6E000065200000507500007368000034
:103AB00020570000420A00000D0000003220EF00F5
:103AC000A3D62100008041001040BA000160EF0041
:103AD000000006002041000057420000204D000079
:103AE0006F640000652000004163000074690000FD
:103AF00076650000200000003220EF0083D821000E
:103B0000008041001040BA000160EF000000060094
:103B100049720000697300004D6100006E0A0000E8
:103B20000D0000003220EF00E3D9210000804100A9
:103B30001040BA000160EF0000000600497200006A
:103B40006973000041750000746F00000A0D0000E9
:103B5000000000003220EF0063DB21000080410004
:103B60001040BA000160EF0000000600424C000067
:103B7000432000004F660000660A00000D000000B0
:103B80003220EF00C3DC2100008041001040BA0069
:103B90000160EF0000000600424C000043200000DE
:103BA0004F6E00000A0D0000000000003220EF0000
:103BB00023DE2100008041001040BA000160EF00C8
:103BC0000000060020200000204800006F6D00006B
:103BD00065200000436100006D6500007261000017
:103BE00020200000200000003220EF0003E0210030
:103BF000008041001040BA000160EF0000000600A4
:103C0000486F00006D650000436100006D0A000010
:103C10000D0000003220EF0063E121000080410030
:103C20001040BA000160EF000000060020200000F4
:103C3000486F00006D6500002044000069730000BB
:103C4000616200006C65000064200000200000003C
:103C50003220EF0043E32100008041001040BA0011
:103C60000160EF00000006000A0D00004274000031
:103C70006E28000025320000782F00002575000016
:103C8000292D000047720000703300000000000082
:103C90003220EF0043E52100008041001040BA00CF
:103CA0000160EF000000060025630000494E00009F
:103CB000503A0000256400003B25000063540000DA
:103CC000414B00003A250000642E000025640000EE
:103CD0003B0000003220EF0063E72100008041003C
:103CE0001040BA000160EF000000060025630000EC
:103CF000494E0000503A0000256400003B000000DF
:103D00003220EF00C3E82100008041001040BA00DB
:103D10000160EF00000006000A0D00004361000092
:103D20006D65000072610000202500006420000025
:103D3000536500006C65000063740000656400005A
:103D4000000000003220EF00E3EA21000080410083
:103D50001040BA000160EF00000006004E6F000046
:103D600020500000726F000067720000616D00005B
:103D70002073000075700000706F00007274000006
:103D8000000000003220EF00E3EC21000080410041
:103D90001040BA000160EF0000000600506700000C
:103DA0006D2000004D6F00006465000020250000BC
:103DB000750A00000D0000003220EF0083EE2100A4
:103DC000008041001040BA000160EF0000000600D2
:103DD00020500000726F000067720000616D0000EB
:103DE000204D00006F6400006520000020200000CE
:103DF00020200000000000003220EF0083F02100AE
:103E0000008041001040BA000160EF000000060091
:103E1000436100006D650000726100002025000014
:103E2000640A00000D0000003220EF0003F22100C0
:103E3000008041001040BA000160EF000000060061
:103E4000496E000043740000726C000041200000C5
:103E5000256400000A0D0000000000003220EF0081
:103E6000A3F32100008041001040BA000160EF0080
:103E700000000600496E000043740000726C0000F0
:103E800042200000256400000A0D00000000000030
:103E90003220EF0043F52100008041001040BA00BD
:103EA0000160EF0000000600427400006E28000070
:103EB00025320000782F000025750000292D000014
:103EC0004772000070340000200A00000D0000005E
:103ED0003220EF0043F72100008041001040BA007B
:103EE0000160EF0000000600496E00002043000062
:103EF000616D0000657200006120000053740000D5
:103F00006F720000652000002564000000000000C2
:103F10003220EF0043F92100008041001040BA0038
:103F20000160EF0000000600496E00002043000021
:103F3000616D000065720000612000005374000094
:103F40006F72000065200000256400000A0D00006B
:103F5000000000003220EF0063FB210000804100E0
:103F60001040BA000160EF000000060020200000B1
:103F70005265000061640000696E00006720000067
:103F8000436100006D6500007261000020200000A8
:103F9000000000003220EF0063FD2100008041009E
:103FA0001040BA000160EF00000006002020000071
:103FB000537400006F720000696E000067200000FB
:103FC000507200006573000065740000202000003E
:103FD000200000003220EF0063FF2100008041003C
:103FE0001040BA000160EF000000060020530000FE
:103FF000746F0000726500002050000072650000C0
:104000007365000074200000253200006420000069
:10401000200000003220EF006301220000804100F8
:104020001040BA000160EF00000006005374000069
:104030006F72000065200000256400000A0D00007A
:10404000000000003220EF00E30222000080410067
:104050001040BA000160EF0000000600452D00008E
:10406000537400006F7200006520000025320000CC
:104070006420000046610000696C00006564000077
:10408000000000003220EF00E30422000080410025
:104090001040BA000160EF0000000600205300004D
:1040A000746F00007265000020250000326400007B
:1040B00020460000616900006C650000640000009B
:1040C0003220EF00C3062200008041001040BA00F9
:1040D0000160EF0000000600496E0000436100002F
:1040E0006D650000726100002050000072650000E4
:1040F0007365000074200000256400000A0D0000B4
:10410000000000003220EF00E308220000804100A0
:104110001040BA000160EF0000000600507200007D
:10412000657300006574000020250000640A00002B
:104130000D0000003220EF00630A220000804100E1
:104140001040BA000160EF00000006000A0D0000F8
:10415000507200006563000069730000696F000021
:104160006E430000616D0000436F00006E7400003C
:10417000726F00006C6C0000657200002573000017
:104180000A0D0000000000003220EF00030D2200A5
:10419000008041001040BA000160EF0000000600FE
:1041A0002020000020200000436F00006D70000000
:1041B000696C0000656400003A200000257300006F
:1041C0002061000074200000257300000A0D00002B
:1041D000000000003220EF00630F22000080410049
:1041E0001040BA000160EF00000006003235000008
:1041F0002D4D0000617900002D31000030000000DD
:104200003220EF00C3102200008041001040BA00AD
:104210000160EF0000000600313300003A31000079
:10422000303A000033370000000000003220EF0079
:1042300023122200008041001040BA000160EF000C
:1042400000000600202000002053000061760000DE
:10425000696E000067200000436F00006E6600007A
:104260006967000020200000000000003220EF00FD
:1042700023142200008041001040BA000160EF00CA
:104280000000060020460000696E0000646900001E
:104290006E67000020430000616D00006572000041
:1042A00061730000000000003220EF0003162200BE
:1042B000008041001040BA000160EF0000000600DD
:1042C000204300006C65000061720000696E000010
:1042D00067200000507200006573000065740000E4
:1042E000730000003220EF00E3172200008041003D
:1042F0001040BA000160EF000000060020430000FB
:104300006C65000061720000696E000067200000AB
:10431000416C00006C200000202000000000000024
:104320003220EF00C3192200008041001040BA0083
:104330000160EF00000006002052000065730000DD
:104340007461000072740000205300007973000053
:10435000746500006D200000000000003220EF00B6
:10436000A31B2200008041001040BA000160EF0052
:1043700000000600202000004E6F000074200000A6
:104380006F6E000020500000726500007365000031
:1043900074200000000000003220EF00831D220086
:1043A000008041001040BA000160EF0000000600EC
:1043B000456E0000616200006C650000204800004E
:1043C0006F730000742000005365000072690000E4
:1043D000616C0000000000003220EF00831F22000B
:1043E000008041001040BA000160EF0000000600AC
:1043F0004469000073610000626C000065200000E9
:104400005365000072690000616C0000202000000C
:1044100020200000000000003220EF008321220055
:10442000008041001040BA000160EF00000006006B
:104430000A0D0000436F00006D6D0000616E00000A
:1044400064200000436F00006D7000006C65000088
:10445000746500000A0D00003E0000003220EF00ED
:10446000A3232200008041001040BA000160EF0049
:104470000000060020200000536800007574000052
:10448000646F0000776E000020410000637400003C
:104490006976000065200000000000003220EF0077
:1044A000A3252200008041001040BA000160EF0007
:1044B0000000060020430000616D000065720000EE
:1044C00061200000506F00007765000072640000FA
:1044D0006F7700006E200000000000003220EF0027
:1044E000A3272200008041001040BA000160EF00C5
:1044F00000000600506F00007274000020250000CC
:10450000643A00000A0D0000000000003220EF00B5
:10451000430220008301500005003100232A2200BD
:10452000008041001040BA000160EF00000006006A
:10453000202A220083814100808141001380BA003B
:10454000000006000A0D670053632000686525001F
:10455000647534006C654C004275780074742000FA
:104560006F6E430028296F00202570003278790093
:104570002F25200032782500205331007461780007
:1045800074750000734600006C6100003220EF007B
:10459000232D2200008041001040BA000160EF008E
:1045A00000000600536500006172000063680000AF
:1045B000696E000067200000666F00007220000036
:1045C00041740000746100006368000065640000CD
:1045D00020430000616D00006572000061730000FF
:1045E0000D0A0000000000003220EF00033022001E
:1045F000008041001040BA000160EF00000006009A
:10460000436100006D6500007261000073200000CE
:10461000466F0000756E00006420000025640000F5
:104620000A0D0000000000003220EF0003322200DB
:10463000008041001040BA000160EF000000060059
:10464000506F00007274000020250000643A0000E2
:1046500020430000616D00006572000061200000D1
:10466000256400000A0D0000000000003220EF0069
:1046700023342200008041001040BA000160EF00A6
:1046800000000600436100006D65000072610000DB
:104690002053000065610000726300006820000084
:1046A000436F00006D7000006C65000074650000D1
:1046B0000A0D00000A0000003220EF0083362200BD
:1046C000008041001040BA000160EF0000000600C9
:1046D000204E00006F200000436100006D200000AC
:1046E00020200000205000006F72000074200000A5
:1046F00030200000200000003220EF00833822002C
:10470000008041001040BA000160EF000000060088
:10471000204300004355000020520000652D00009A
:10472000496E0000697400002057000061690000B4
:1047300074200000000000003220EF00833A2200C5
:10474000008041001040BA000160EF000000060048
:104750000D0A0000506100006E610000736F0000E0
:104760006E69000063200000415700002D480000E2
:1047700045310000303000000D0A0000000000004C
:104780003220EF00C33C2200008041001040BA00FC
:104790000160EF000000060020410000572D0000DE
:1047A000484500003130000030200000205000005B
:1047B0006F72000074200000302000002000000014
:1047C0003220EF00C33E2200008041001040BA00BA
:1047D0000160EF0000000600204700006574000043
:1047E00038200000000000003220EF0003402200CB
:1047F000008041001040BA000160EF000000060098
:1048000020200000202D00002D2000002532000077
:10481000582000002D2D00000A0D000000000000AF
:104820003220EF00C3412200008041001040BA0056
:104830000160EF00000006000A0D000020200000CB
:104840002067000065740000313600002000000081
:104850003220EF0043432200008041001040BA00A4
:104860000160EF000000060020200000202D000065
:104870002D200000254C0000582000002D2D0000A8
:10488000200A00000D0000003220EF000345220046
:10489000008041001040BA000160EF0000000600F7
:1048A0000A0D000020200000206700006574000051
:1048B00033320000200000003220EF008346220047
:1048C000008041001040BA000160EF0000000600C7
:1048D00020200000202D00002D200000254C00008D
:1048E000582000002D2D00000A0D000000000000DF
:1048F0003220EF0043482200008041001040BA00FF
:104900000160EF00000006000A0D000020430000D7
:10491000616D000065720000615400007970000054
:10492000652000002D200000000000003220EF0074
:10493000234A2200008041001040BA000160EF00CD
:1049400000000600536F00006E7900002045000053
:10495000564900002D44000033300000287200004A
:10496000290D00000A0000003220EF00034C220055
:10497000008041001040BA000160EF000000060016
:1049800020450000564900002D440000333000004F
:1049900028720000295000006F720000742000008F
:1049A00030200000200000003220EF00034E2200E3
:1049B000008041001040BA000160EF0000000600D6
:1049C000496E0000766100006C6900006420000000
:1049D000436100006D650000726100000D0A000077
:1049E000000000003220EF00E34F22000080410071
:1049F0001040BA000160EF000000060020490000EE
:104A00006E760000616C00006964000020430000C5
:104A1000616D000065720000610000003220EF004F
:104A2000A3512200008041001040BA000160EF0055
:104A3000000006000D0A0000536F00006E790000B0
:104A400020450000564900002D440000333000008E
:104A50002F330000312000000D0A0000000000008C
:104A60003220EF00C3532200008041001040BA0002
:104A70000160EF00000006002045000056490000DC
:104A80002D440000333000002F330000315000006F
:104A90006F72000074200000302000002000000031
:104AA0003220EF00C3552200008041001040BA00C0
:104AB0000160EF00000006000D0A0000536F0000C7
:104AC0006E79000020450000564900002D4400008A
:104AD000333000000D0A0000000000003220EF001B
:104AE000A3572200008041001040BA000160EF008F
:104AF0000000060020450000564900002D4400003B
:104B00003330000020200000205000006F720000B1
:104B10007420000030200000200000003220EF0050
:104B2000A3592200008041001040BA000160EF004C
:104B3000000006000D0A00005661000064640000D9
:104B4000696F000020410000646400002D410000F6
:104B50002D430000616D00000D0A00000000000000
:104B60003220EF00C35B2200008041001040BA00F9
:104B70000160EF00000006002041000064640000B6
:104B80002D4100002D430000616D00002050000009
:104B90006F72000074200000302000002000000030
:104BA0003220EF00C35D2200008041001040BA00B7
:104BB0000160EF00000006000D0A0000536F0000C6
:104BC0006E79000020450000564900002D44000089
:104BD00031300000300D00000A0000003220EF00EC
:104BE000A35F2200008041001040BA000160EF0086
:104BF0000000060020450000564900002D4400003A
:104C00003130000030200000205000006F720000A2
:104C10007420000030200000200000003220EF004F
:104C2000A3612200008041001040BA000160EF0043
:104C3000000006000D0A0000536F00006E790000AE
:104C400020450000564900002D4400003730000088
:104C50000D0A0000000000003220EF0083632200F4
:104C6000008041001040BA000160EF000000060023
:104C700020450000564900002D4400003730000058
:104C800020200000205000006F72000074200000FF
:104C900030200000200000003220EF008365220059
:104CA000008041001040BA000160EF0000000600E3
:104CB0000D0A0000536F00006E79000020420000D2
:104CC00052430000482D000037300000300D000036
:104CD0000A0000003220EF006367220000804100DC
:104CE0001040BA000160EF00000006002042000002
:104CF00052430000482D00003730000030200000F3
:104D0000205000006F72000074200000302000006E
:104D1000200000003220EF00636922000080410083
:104D20001040BA000160EF00000006000D0A00000C
:104D3000456C00006D6F000020430000616D0000B5
:104D400065720000610D00000A0000003220EF00D3
:104D5000236B2200008041001040BA000160EF0088
:104D600000000600204500006C6D00006F20000070
:104D70002020000020200000205000006F72000062
:104D80007420000030200000200000003220EF00DE
:104D9000236D2200008041001040BA000160EF0046
:104DA000000006000D0A0000536F00006E7900003D
:104DB00020420000524300002D330000303000003C
:104DC0000D0A0000000000003220EF00036F2200F7
:104DD000008041001040BA000160EF0000000600B2
:104DE00020420000524300002D330000303000000C
:104DF00020200000205000006F720000742000008E
:104E000030200000200000003220EF00037122005B
:104E1000008041001040BA000160EF000000060071
:104E20000D0A0000536F00006E7900002042000060
:104E3000524300002D5A000037300000300D0000B2
:104E40000A0000003220EF00E372220000804100DF
:104E50001040BA000160EF00000006002042000090
:104E6000524300002D5A000037300000302000006F
:104E7000205000006F7200007420000030200000FD
:104E8000200000003220EF00E37422000080410087
:104E90001040BA000160EF00000006000D0A00009B
:104EA000536F00006E790000204200005243000062
:104EB0002D5A000033330000300D00000A000000BE
:104EC0003220EF00C3762200008041001040BA007B
:104ED0000160EF0000000600204200005243000085
:104EE0002D5A000033330000302000002050000015
:104EF0006F720000742000003020000020000000CD
:104F00003220EF00C3782200008041001040BA0038
:104F10000160EF00000006000D0A0000564100008D
:104F200044440000494F000020480000442D000088
:104F3000313800000D0A0000000000003220EF00B0
:104F4000A37A2200008041001040BA000160EF0007
:104F5000000006005641000044440000494F000094
:104F6000204800004431000038200000506F00004D
:104F70007274000020300000000000003220EF00BA
:104F8000A37C2200008041001040BA000160EF00C5
:104F9000000006000D0A0000536F00006E7900004B
:104FA00020450000564900002D4800004431000013
:104FB0000D0A0000000000003220EF00837E220076
:104FC000008041001040BA000160EF0000000600C0
:104FD00020450000564900002D48000044310000E3
:104FE00020200000205000006F720000742000009C
:104FF00030200000200000003220EF0083802200DB
:10500000008041001040BA000160EF00000006007F
:105010000D0A00005661000064640000696F000022
:1050200020430000656900006C6900006E670000A5
:1050300056490000455700000D0A0000000000001E
:105040003220EF00C3822200008041001040BA00ED
:105050000160EF000000060020430000562F000012
:10506000435600004D50000020200000205000005A
:105070006F7200007420000030200000200000004B
:105080003220EF00C3842200008041001040BA00AB
:105090000160EF0000000600556E00006B6E00001E
:1050A0006F7700006E200000436100006D65000016
:1050B000726100000D0A0000000000003220EF00C5
:1050C000A3862200008041001040BA000160EF007A
:1050D00000000600205500006E6B00006E6F00009F
:1050E000776E000020200000205000006F7200004A
:1050F0007420000030200000200000003220EF006B
:10510000A3882200008041001040BA000160EF0037
:10511000000006000A0D000020410000542F00008E
:105120004D4400005F4D00006F64000065490000C1
:105130006E710000200000003220EF00838A220000
:10514000008041001040BA000160EF00000006003E
:105150000D0A00005761000069740000536F0000E1
:105160006E790000496E0000715200006573000006
:1051700070200000000000003220EF00838C22002D
:10518000008041001040BA000160EF0000000600FE
:105190000D0A0000205700006169000074530000F0
:1051A0006F6E000079410000636B0000000000009A
:1051B0003220EF00438E2200008041001040BA00F0
:1051C0000160EF00000006000D0A000020570000FB
:1051D00061690000745300006F6E000079000000E8
:1051E0003220EF00C38F2200008041001040BA003F
:1051F0000160EF00000006002A570000616900000E
:10520000745300006F6E0000790000003220EF0040
:1052100023912200008041001040BA000160EF009D
:10522000000006000D0A0000205700006169000020
:105230007452000065730000705300006F6E000030
:10524000790000003220EF00E3922200008041004C
:105250001040BA000160EF0000000600202D0000A1
:1052600020540000696D0000656F00007574000037
:105270002025000075200000286D00007329000023
:105280000D0A0000000000003220EF00039522000C
:10529000008041001040BA000160EF0000000600ED
:1052A000436100006E630000656C00002053000045
:1052B00031200000000000003220EF008396220021
:1052C000008041001040BA000160EF0000000600BD
:1052D000436100006E630000656C00002053000015
:1052E00032200000000000003220EF00039822006E
:1052F000008041001040BA000160EF00000006008D
:105300000A0D000020200000204700006574000006
:105310004252000043500000616E000054690000DA
:105320006C740000506F000073200000000000004B
:105330003220EF00439A2200008041001040BA0062
:105340000160EF000000060020200000202D00007A
:105350002D200000503A0000254C0000582C000081
:10536000543A0000254C0000582000002D2D00006C
:105370000A0D0000000000003220EF00839C220094
:10538000008041001040BA000160EF0000000600FC
:105390000A0D000020430000616D000065720000EE
:1053A00061540000797000006520000000000000DA
:1053B0003220EF00439E2200008041001040BA00DE
:1053C0000160EF00000006000A0D00002050000000
:1053D0006F77000065720000204F00006E20000013
:1053E0005265000074720000792000000000000087
:1053F0003220EF0043A02200008041001040BA009C
:105400000160EF00000006000A0D000020430000CC
:10541000616D000065720000615400007970000049
:105420006520000056310000200000003220EF000F
:1054300023A22200008041001040BA000160EF006A
:1054400000000600436100006E6F00006E20000047
:10545000425500002D340000354800000D0A0000C0
:10546000000000003220EF00E3A322000080410092
:105470001040BA000160EF0000000600204200006A
:10548000552D000034350000482000002020000089
:10549000205000006F7200007420000030200000D7
:1054A000200000003220EF00E3A522000080410030
:1054B0001040BA000160EF000000060043610000E8
:1054C0006E6F00006E200000425500002D35000078
:1054D000304800000D0A0000000000003220EF00FC
:1054E000A3A72200008041001040BA000160EF0035
:1054F0000000060020420000552D0000353000005D
:105500004820000020200000205000006F720000A2
:105510007420000030200000200000003220EF0046
:10552000A3A92200008041001040BA000160EF00F2
:1055300000000600436100006E6F00006E20000056
:10554000564300002D43000035300000490D000097
:105550000A0000003220EF0063AB2200008041000F
:105560001040BA000160EF00000006002056000065
:10557000432D00004335000030690000202000006A
:10558000205000006F7200007420000030200000E6
:10559000200000003220EF0063AD220000804100B7
:1055A0001040BA000160EF0000000600205D00001E
:1055B0000A0D0000000000003220EF0083AE220040
:1055C000008041001040BA000160EF0000000600BA
:1055D0000D0A0000205700006169000074430000BC
:1055E000616E00006F6E0000000000003220EF00CE
:1055F00023B02200008041001040BA000160EF009B
:10560000000006000D0A000020570000616900003C
:1056100074430000616E00006F6E00004E6F00006A
:105620007442000075730000790000003220EF0022
:1056300023B22200008041001040BA000160EF0058
:10564000000006000D0A00002057000061690000FC
:1056500074430000616E00006F6E00005054000043
:105660005A530000746F0000700000003220EF00F9
:1056700023B42200008041001040BA000160EF0016
:1056800000000600202D000020540000696D00007D
:10569000656F000075740000202500006C75000027
:1056A000202800006D730000290D00000A00000092
:1056B0003220EF0043B62200008041001040BA00C3
:1056C0000160EF00000006000D0A000020570000F6
:1056D0006169000074500000616E00006173000099
:1056E0006F6E000069630000000000003220EF00D0
:1056F00023B82200008041001040BA000160EF0092
:10570000000006000A0D0000553100002845000089
:1057100072720000292000005B4C00005352000010
:105720005D25000032780000000000003220EF000C
:1057300023BA2200008041001040BA000160EF004F
:10574000000006000A0D0000553200002845000048
:1057500072720000292000005B4C000053520000D0
:105760005D25000032780000000000003220EF00CC
:1057700023BC2200008041001040BA000160EF000D
:10578000000006000A0D0000436800006563000089
:105790006B5F0000584F00004E200000436C00007B
:1057A0006561000072200000655F0000586F000016
:1057B000666600005F530000656E00007400000024
:1057C0003220EF00830220008301500005003100E9
:1057D000C3BF2200008041001040BA000160EF000A
:1057E00000000600C0BF220083814100808141008B
:1057F0001380BA00000006000A0D690043686700C4
:10580000656368006B5F2800584F25004E204C00F0
:105810005365750074202900655F2000586F57009C
:10582000666669005F536E00656E640074206F00E9
:10583000436F7700756E280074282500254C75008D
:1058400075292900204800003220EF0003C3220000
:10585000008041001040BA000160EF000000060027
:105860000A0D0000584F00004E2000005365000054
:105870006E74000020490000646C00006520000088
:105880005374000061740000650000003220EF00D6
:1058900023C52200008041001040BA000160EF00E3
:1058A000000006000A0D0000436800006563000068
:1058B0006B5F0000584F0000464600002053000078
:1058C00065740000206500005F5800006F660000EE
:1058D000665F0000536500006E7400000000000069
:1058E0003220EF00C3C72200008041001040BA0000
:1058F0000160EF00000006000A0D00005072000079
:105900006F63000065730000735300006C6100005A
:105910007665000028290000206200006164000014
:10592000205300004F4D00003D250000327800005C
:10593000000000003220EF0063CA22000080410016
:105940001040BA000160EF00000006000A0D0000E0
:10595000507200006F63000065730000734D00001B
:1059600061730000746500007228000029200000A7
:105970006261000064200000534F00004D3D0000B4
:1059800025320000780000003220EF0003CD220015
:10599000008041001040BA000160EF0000000600E6
:1059A0000A0D0000436800006B4600006F630000B2
:1059B00075730000456E0000636F000064650000B1
:1059C0007228000025300000344C000078290000C7
:1059D000000000003220EF0063CF22000080410071
:1059E0001040BA000160EF00000006002020000017
:1059F000466F000063750000732000004E650000D4
:105A000061720000202500006C750000000000009D
:105A10003220EF0043D12200008041001040BA0044
:105A20000160EF000000060020200000466F00002B
:105A300063750000732000004661000072200000C2
:105A4000256C0000750000003220EF0003D3220017
:105A5000008041001040BA000160EF000000060025
:105A60000A0D0000436800006B49000072690000E5
:105A7000734500006E6300006F64000065720000F3
:105A800028250000303400004C7800002900000078
:105A90003220EF0043D52200008041001040BA00C0
:105AA0000160EF00000006000A0D000043680000DE
:105AB0006B5A00006F6F00006D4500006E630000C0
:105AC0006F6400006572000028250000303400007B
:105AD0004C780000290000003220EF0083D722001C
:105AE000008041001040BA000160EF000000060095
:105AF0000A0D0000436800006B500000616E00005A
:105B0000456E0000636F00006465000072280000AD
:105B100025300000344C000078290000000000000F
:105B20003220EF00C3D92200008041001040BA00AB
:105B30000160EF00000006000A0D0000436800004D
:105B40006B540000696C0000744500006E63000037
:105B50006F640000657200002825000030340000EA
:105B60004C780000290000003220EF0003DC220006
:105B7000008041001040BA000160EF000000060004
:105B80000A0D0000436800006B52000065640000CD
:105B9000456E0000636F000064650000722800001D
:105BA00025300000344C000078290000000000007F
:105BB0003220EF0043DE2200008041001040BA0096
:105BC0000160EF00000006000A0D000043680000BD
:105BD0006B4200006C750000654500006E630000BC
:105BE0006F6400006572000028250000303400005A
:105BF0004C780000290000003220EF0083E02200F2
:105C0000008041001040BA000160EF000000060073
:105C10000A0D0000436800006B440000657400003A
:105C2000616900006C4500006E6300006F64000055
:105C30006572000028250000303400004C78000018
:105C4000290000003220EF00E3E222000080410042
:105C50001040BA000160EF00000006000A0D0000CD
:105C6000436800006B470000616900006E4500005A
:105C70006E6300006F64000065720000282500005C
:105C8000303400004C780000290000003220EF0082
:105C900023E52200008041001040BA000160EF00BF
:105CA00000000600202000002020000047610000C6
:105CB000696E0000204E00002F41000020200000EF
:105CC000200000003220EF00E3E6220000804100C7
:105CD0001040BA000160EF00000006000A0D00004D
:105CE000203E0000000000003220EF0003E8220008
:105CF000008041001040BA000160EF000000060083
:105D00003E250000732000004E6F0000742000004C
:105D1000466F0000756E0000640A00000D3E000032
:105D2000000000003220EF00E3E922000080410083
:105D30001040BA000160EF00000006000A250000D4
:105D400073250000732000002020000020000000C8
:105D50003220EF0043EB2200008041001040BA00E7
:105D60000160EF0000000600436F00006D7000004E
:105D7000696C0000656400003A2000002573000093
:105D80002061000074200000257300000A0D00004F
:105D9000000000003220EF00E302200083015000E9
:105DA0000500310063EE2200008041001040BA007F
:105DB0000160EF000000060060EE220083814100D8
:105DC000808141001380BA00000006000D0A200007
:105DD0005379200073744400656D6500205366009C
:105DE00065746100746975006E676C00733A7400C5
:105DF0000A0D20000A0D50004465720066616500BE
:105E0000756C730074206500436174006D653A0021
:105E1000726120003A2025002564640020200A00D9
:105E200020200D00202000003220EF0003F222008D
:105E3000008041001040BA000160EF000000060041
:105E400054720000616E0000736900007469000004
:105E50006F6E000020540000696D0000653A00007C
:105E600020250000640A00000D0000003220EF0031
:105E700043032000830150000500310023F5220078
:105E8000008041001040BA000160EF0000000600F1
:105E900020F5220083814100808141001380BA00F7
:105EA000000006000A0D3A00436120006D652000E5
:105EB00072613100205020006F7220007420320087
:105EC0005365200061722000636833003A2020008F
:105ED00020312000202034003220200020332000F8
:105EE00020203500342020002035200020203600DE
:105EF00036202000203720002020370043430A00AE
:105F000055200D004D6F0000646500003220EF0049
:105F100023F92200008041001040BA000160EF0028
:105F200000000600202000002020000020200000AB
:105F30002020000020200000202000002020000061
:105F40002020000020200000202000000000000091
:105F50003220EF0043FB2200008041001040BA00D5
:105F60000160EF000000060020200000202000005B
:105F70002020000020200000202000002000000041
:105F80003220EF0043022000830150000500310061
:105F9000C3FD2200008041001040BA000160EF0004
:105FA00000000600C0FD2200838141008081410085
:105FB0001380BA00000006000A0D20005061500056
:105FC0006E53610070656E006564650020206C0092
:105FD0002020200054694C006C74690053706700E5
:105FE0006565680064207400202073005A6F0A0001
:105FF0006F6D0D00537000006565000064200000A7
:106000003220EF0003022000830150000500310020
:10601000C3012300008041001040BA000160EF007E
:1060200000000600C00123008381410080814100FF
:106030001380BA0000000600202020002025200048
:10604000642020002020200020202000202020008C
:10605000202020002020200025642500202064002E
:1060600020200A0020200D0020200A0020200D0002
:1060700025640000202000003220EF00830423006C
:10608000008041001040BA000160EF0000000600EF
:106090004A6F00007973000074690000636B0000B0
:1060A0002053000065740000757000003A0A00007B
:1060B0000D0000003220EF00230320008301500078
:1060C0000500310063072300008041001040BA0042
:1060D0000160EF000000060060072300838141009B
:1060E000808141001380BA00000006000A0D3A00CA
:1060F00020502000616E2000205031006F7220007F
:10610000742020004469320072652000637420000E
:10611000696F33006E3A20002020200031203400C7
:1061200020322000202020003320350020342000A1
:10613000202020003520360020362000202020009E
:106140003720370020530A0070650D006564000099
:106150003220EF00430B2300008041001040BA00C2
:106160000160EF0000000600202000002020000059
:10617000202000002020000020200000202000001F
:10618000202000002020000020200000202000000F
:10619000200000003220EF00630D2300008041004A
:1061A0001040BA000160EF0000000600202000004F
:1061B000202000002020000020200000000000001F
:1061C0003220EF002303200083015000050031003E
:1061D000C30F2300008041001040BA000160EF00AF
:1061E00000000600C00F2300838141008081410030
:1061F0001380BA00000006000D0A3A00546920001E
:106200006C742000205031006F7220007420200038
:10621000446932007265200063742000696F3300A6
:106220006E3A20002020200031203400203220004F
:1062300020202000332035002034200020202000A2
:10624000352036002036200020202000372037005F
:1062500020530A0070650D00656400003220EF00D5
:10626000230320008301500005003100A314230004
:10627000008041001040BA000160EF0000000600FD
:10628000A014230083814100808141001380BA0063
:10629000000006000D0A3A005A6F20006F6D2000C2
:1062A000205031006F7220007420200044693200B9
:1062B0007265200063742000696F33006E3A20001D
:1062C0002020200031203400203220002020200017
:1062D00033203500203420002020200035203600D7
:1062E00020362000202020003720370020530A00CD
:1062F00070650D00656400003220EF0083182300F4
:10630000008041001040BA000160EF00000006006C
:106310000D0A00004E6500007574000072610000F7
:106320006C2000005A6F00006E6500003A200000EB
:10633000506100006E200000546900006C74000081
:10634000205A00006F6F00006D0A00000D00000071
:106350003220EF00431B2300008041001040BA00B0
:106360000160EF0000000600202000002020000057
:10637000202000002020000020200000202000001D
:1063800020200000202500003264000020200000B2
:10639000253200006420000020200000253200008B
:1063A000640000003220EF00E31D23000080410064
:1063B0001040BA000160EF00000006000A0D000066
:1063C000507200006573000065740000733A0000AD
:1063D0000A0D00000A0D0000000000003220EF004E
:1063E000230320008301500005003100A320230077
:1063F000008041001040BA000160EF00000006007C
:10640000A020230083814100808141001380BA00D5
:1064100000000600436173006D20200050722000D0
:10642000652047004D6F6100646569006C206E0057
:106430002020200020202000202052002050650035
:10644000616E6400202020002020200020542000C5
:10645000696C420074206C00205A75006F6F6500F3
:106460006D202000204644006F6365007573740042
:1064700020492E00726900003220EF00832423009F
:10648000008041001040BA000160EF0000000600EB
:10649000205B000049720000697300002C46000078
:1064A0006F630000757300002C410000574200002C
:1064B0002C200000424C0000435D00000A0D00004B
:1064C0000A0D0000000000003220EF00E30220006F
:1064D00083015000050031000328230000804100A3
:1064E0001040BA000160EF00000006000028230001
:1064F00083814100808141001380BA0000000600C2
:1065000020252000642020002025250032644C0036
:10651000202058002531200032732000202525003E
:1065200058254C00582558005820200020252000D0
:106530004C58250020203200254C4C005820580093
:10654000202520004C58200020202000254C200031
:1065500058200000202500004C5800003220EF0099
:10656000A32B2300008041001040BA000160EF001F
:10657000000006004F6E00002020000020000000F8
:106580003220EF00C32C2300008041001040BA00ED
:106590000160EF00000006004F660000662000006A
:1065A000200000003220EF00E32D23000080410096
:1065B0001040BA000160EF00000006000A0D000064
:1065C000436100006D2000004D6F00006465000015
:1065D0006C0A00000D0000003220EF00832F230022
:1065E000008041001040BA000160EF00000006008A
:1065F0002025000064200000204E00006F200000D5
:10660000436100006D650000726100000A0D00002A
:10661000000000003220EF006331230000804100C1
:106620001040BA000160EF00000006004545000080
:10663000507200006F6D000020440000756D000076
:10664000703A00000A0D0000000000003220EF0048
:1066500023332300008041001040BA000160EF00A6
:106660000000060045450000507200006F6D0000FC
:10667000204300006F6E0000666900006720000084
:10668000447500006D7000003A0A00000D00000023
:106690003220EF0043352300008041001040BA0053
:1066A0000160EF0000000600454500005072000048
:1066B0006F6D0000205000007265000073650000DF
:1066C00074200000447500006D7000003A0A00005C
:1066D0000D0000003220EF006337230000804100EE
:1066E0001040BA000160EF000000060045450000C0
:1066F000507200006F6D00002048000069670000C4
:1067000068200000447500006D7000003A0A000027
:106710000D0000003220EF006339230000804100AB
:106720001040BA000160EF000000060020200000C9
:106730002020000020200000000000003220EF0098
:10674000A33A2300008041001040BA000160EF002E
:10675000000006000A0D00003E2000004157000026
:10676000423D00004F6E00000A0D00003E20000078
:10677000000000003220EF00633C23000080410055
:106780001040BA000160EF00000006000A0D000092
:106790003E20000041570000423D00004F660000CF
:1067A000660A00000D3E0000200000003220EF00CD
:1067B000233E2300008041001040BA000160EF003A
:1067C000000006000A0D00003E200000424C0000C0
:1067D000433D00004F6E00000A0D00003E20000007
:1067E000000000003220EF00E33F23000080410062
:1067F0001040BA000160EF00000006000A0D000022
:106800003E200000424C0000433D00004F66000067
:10681000660A00000D3E0000200000003220EF005C
:10682000A3412300008041001040BA000160EF0046
:10683000000006000A0D00000A0D000020490000BB
:106840006E760000616C0000696400002049000061
:1068500032630000204100006464000072650000A3
:10686000737300002028000025730000290A00002F
:106870000D0000003220EF0063442300008041003F
:106880001040BA000160EF00000006000A0D000091
:106890000A0D0000204900006E760000616C0000C7
:1068A00069640000204900003263000020520000AB
:1068B00065670000697300007465000072200000C5
:1068C00028250000732900000A0D000000000000C8
:1068D0003220EF0043022000830150000500310008
:1068E00043482300008041001040BA000160EF00DF
:1068F0000000060040482300838141008081410060
:106900001380BA00000006000A0D58000A0D20008E
:106910005265520061646500204973003243700083
:1069200020416F0064646E007265730073736500CC
:106930003D253D0032582500205232006567580041
:1069400069730A0074650D00723D00002532000075
:106950003220EF00030220008301500005003100C7
:10696000434C2300008041001040BA000160EF005A
:1069700000000600404C23008381410080814100DB
:106980001380BA00000006000A0D32000A0D5800FC
:1069900057722C00697444006520610041647400E2
:1069A0006472610065733D00733D2500253232003D
:1069B000582C58005265200067690A0073740D0056
:1069C000657200003D2500003220EF00034F2300D8
:1069D000008041001040BA000160EF000000060096
:1069E0000A0D000020450000727200006F72000066
:1069F0002D200000436100006D6500007261000001
:106A0000204E00006F74000020530000656C0000F1
:106A10006563000074650000640D00000A3E00001C
:106A2000200000003220EF00E351230000804100ED
:106A30001040BA000160EF00000006000A0D0000DF
:106A400045720000726F0000722D000020490000A6
:106A50007269000073200000696E00002041000090
:106A6000757400006F2000004D6F00006465000029
:106A70000A0D0000000000003220EF0083542300C4
:106A8000008041001040BA000160EF0000000600E5
:106A900020200000204900007269000073200000DF
:106AA000436F00006D6D0000616E00006420000007
:106AB000466F0000726D0000617400000A0D000056
:106AC000000000003220EF00E35623000080410068
:106AD0001040BA000160EF00000006002020000016
:106AE0002049000072690000732000004175000019
:106AF000746F000028630000722900002C20000041
:106B00004972000069730000204D0000616E0000B2
:106B1000756100006C28000063720000290A000003
:106B20000D0000003220EF00E359230000804100F7
:106B30001040BA000160EF000000060020200000B5
:106B400020490000726900007320000055700000A9
:106B50002C34000028630000722900002C20000063
:106B60004972000069730000204400006F77000044
:106B70006E2C0000303400002863000072290000F1
:106B80000A0D0000000000003220EF00035D23002A
:106B9000008041001040BA000160EF0000000600D4
:106BA0000A0D00003E2000004469000061670000FB
:106BB0003D4F00006E0A00000D3E00002000000066
:106BC0003220EF00C35E2300008041001040BA0075
:106BD0000160EF00000006000A0D00003E200000EA
:106BE00044690000616700003D4F000066660000D8
:106BF0000A0D00003E200000000000003220EF00DF
:106C0000A3602300008041001040BA000160EF0043
:106C1000000006003E200000257300002042000016
:106C200075740000746F00006E2000002573000072
:106C3000204300006C650000617200006564000084
:106C40000D0A00003E200000000000003220EF008E
:106C5000430220008301500005003100236423001B
:106C6000008041001040BA000160EF000000060003
:106C70002064230083814100808141001380BA0099
:106C8000000006003E2064002573200020456C00B3
:106C9000727265006F726E002C206700257374009D
:106CA0002042680075742000746F25006E20750006
:106CB00073742E0072690D006E670A002C203E006E
:106CC000696E2000766100006C6900003220EF00E0
:106CD000E3012000830150000500310023682300F8
:106CE000008041001040BA000160EF000000060083
:106CF0002068230083814100808141001380BA0015
:106D0000000006003E2070002573720020456F00D1
:106D1000727276006F7269002C2064004275650003
:106D2000747464006F6E0D0020730A0074723E006C
:106D3000696E2000672000006E6F00007420000064
:106D40003220EF0063022000830150000500310073
:106D5000C36B2300008041001040BA000160EF00C7
:106D600000000600C06B2300838141008081410048
:106D70001380BA00000006003E2065002573650000
:106D800020456E00727220006F7231002C202000AE
:106D90004275610074746E006F6E6400206E200096
:106DA000756D31006265340072202E0025780D006B
:106DB0002C200A006E6F3E007420200062650000E7
:106DC000747700003220EF00E301200083015000BF
:106DD00005003100E36F2300008041001040BA003D
:106DE0000160EF0000000600E06F23008381410096
:106DF000808141001380BA00000006003E20700030
:106E00002573720020456F00727276006F72690000
:106E10002C20640042756500747464006F6E2E004F
:106E2000206E0D00756D0A0062653E007220200024
:106E30006E6F0000742000003220EF008372230088
:106E4000008041001040BA000160EF000000060021
:106E50000A0D00003E200000506F00007765000022
:106E6000723D00004F6E00000A0D00003E20000041
:106E7000000000003220EF00637423000080410016
:106E80001040BA000160EF00000006000A0D00008B
:106E90003E200000506F000077650000723D00004A
:106EA0004F660000660A00000D3E00002000000052
:106EB0003220EF0043762300008041001040BA00EA
:106EC0000160EF00000006000A0D00003E200000F7
:106ED0005344000069610000673D00004F6E0000F0
:106EE0000A0D00003E200000000000003220EF00EC
:106EF00023782300008041001040BA000160EF00B9
:106F0000000006000A0D00003E200000534400006F
:106F100069610000673D00004F660000660A0000DE
:106F20000D3E0000200000003220EF002302200070
:106F30008301500005003100037B230000804100E5
:106F40001040BA000160EF0000000600007B230043
:106F500083814100808141001380BA000000060057
:106F60000A0D61003E2069004A5374004437540002
:106F7000302069002D206D004A6F6500797328006C
:106F800074692500636B7500205329006C6F0A003B
:106F900077200D0044373E00302020004F6E000067
:106FA0002C5700003220EF00230220008301500004
:106FB00005003100E37E2300008041001040BA004C
:106FC0000160EF0000000600E07E230083814100A5
:106FD000808141001380BA00000006000A0D5700AE
:106FE0003E2061004A536900443774003020540049
:106FF0002D2069004A6F6D0079736500746928005F
:10700000636B2500205375006C6F290077200A0000
:1070100044370D0030203E004F662000662C0000F3
:107020003220EF00C3812300008041001040BA00ED
:107030000160EF00000006000A0D00003E20000085
:10704000546100006C6C0000793D00004163000059
:107050007469000076650000204800006967000040
:10706000680A00000D3E0000200000003220EF0002
:1070700023842300008041001040BA000160EF002B
:10708000000006000A0D00003E20000054610000D0
:107090006C6C0000793D00004163000074690000E1
:1070A00076650000204C00006F7700000A0D00009C
:1070B0003E200000000000003220EF008386230005
:1070C000008041001040BA000160EF00000006009F
:1070D00045720000726F0000722D00002046000013
:1070E0006F63000075730000206900006E200000CF
:1070F00041750000746F0000204D00006F640000B7
:10710000650A00000D0000003220EF000389230013
:10711000008041001040BA000160EF00000006004E
:1071200020200000204600006F63000075730000FF
:10713000204300006F6D00006D6100006E64000070
:10714000204600006F7200006D610000740A0000AC
:107150000D0000003220EF00638B2300008041000F
:107160001040BA000160EF0000000600202000007F
:10717000204600006F63000075730000204100008E
:10718000757400006F28000063720000292C000055
:1071900020200000204600006F630000757300008F
:1071A000204D0000616E0000756100006C28000039
:1071B00063720000290A00000D0000003220EF0079
:1071C000A38E2300008041001040BA000160EF0050
:1071D0000000060020200000204600006F63000031
:1071E0007573000020550000702C0000342800004A
:1071F00063720000292C00002020000020460000BF
:107200006F63000075730000204400006F7700007A
:107210006E2C00003428000063720000290A000070
:107220000D0000003220EF00C30120008301500058
:1072300005003100E3922300008041001040BA00B5
:107240000160EF0000000600E0922300838141000E
:10725000808141001380BA000000060020206F00EA
:10726000204677006F636E0075732C002055300048
:10727000702C610030613000302828006372630098
:10728000292C7200204629006F630A0075730D00D7
:10729000204400003220EF0063952300008041006D
:1072A0001040BA000160EF0000000600202000003E
:1072B000204600006F630000757300002025000069
:1072C000750000003220EF00E396230000804100AB
:1072D0001040BA000160EF00000006000A0D000037
:1072E0003E200000436100006D65000072610000F7
:1072F00020250000642000004E6F00007420000074
:1073000061760000616900006C610000626C000041
:10731000650A00000D3E0000200000003220EF0052
:10732000A3992300008041001040BA000160EF00E3
:10733000000006000A0D00003E2000004A50000038
:10734000616E000053700000643A0000205000009D
:107350006F72000074200000203100002020000027
:1073600032200000203300002020000034200000E4
:1073700020350000202000003620000020370000CB
:107380000A0D0000000000003220EF000302200080
:107390008301500005003100039E2300008041005E
:1073A0001040BA000160EF0000000600009E2300BC
:1073B00083814100808141001380BA0000000600F3
:1073C00020202500202032002020640020202000E2
:1073D00020202500202032002020640020202000D2
:1073E00025322500642032002532640064200A0022
:1073F00025320D0064203E0025320000642000008C
:107400003220EF00C3A02300008041001040BA00EA
:107410000160EF00000006000D0A00003E4A000077
:10742000506100006E4400006972000020200000DE
:10743000446900007265000063740000696F000019
:107440006E3A00002031000020320000203300009E
:1074500020340000203500002036000020370000D6
:107460000A0D0000000000003220EF00E3012000C0
:10747000830150000500310003A523000080410076
:107480001040BA000160EF000000060000A52300D4
:1074900083814100808141001380BA000000060012
:1074A000202025002020630020202000202025000F
:1074B00020206300202020002020250020206300C1
:1074C00020202000202025002025630063200A00C2
:1074D00025630D0020253E00632000003220EF00D0
:1074E000A3A72300008041001040BA000160EF0014
:1074F000000006000A0D00003E2000005061000060
:107500006E53000070650000656400003D250000BA
:10751000640A00000D3E0000200000003220EF0051
:10752000C30120008301500005003100A3AA2300FD
:10753000008041001040BA000160EF00000006002A
:10754000A0AA230083814100808141001380BA00FA
:10755000000006000A0D20003E2034004A5A200098
:107560006F6F20006D533500706420003A202000BA
:10757000506F360072742000202020003120370028
:1075800020320A0020200D00332000003220EF00BE
:1075900003022000830150000500310023AE2300C8
:1075A000008041001040BA000160EF0000000600BA
:1075B00020AE230083814100808141001380BA0006
:1075C000000006002020200020202500202032007E
:1075D00020206400202020002020250020203200D0
:1075E0002020640020252000326425002025320060
:1075F0003264640020250A0032640D0020253E001C
:10760000326400003220EF00E3B02300008041002C
:107610001040BA000160EF00000006000D0A0000F3
:107620003E4A00005A6F00006F6D00004469000080
:1076300072200000204400006972000065630000B1
:10764000746900006F6E00003A20000031200000D5
:1076500032200000332000003420000035200000DC
:1076600036200000370A00000D0000003220EF0035
:1076700003022000830150000500310023B52300E0
:10768000008041001040BA000160EF0000000600D9
:1076900020B5230083814100808141001380BA001E
:1076A000000006002020630020202000202025006C
:1076B00020206300202020002020250020206300BF
:1076C00020202000202025002020630020200A0008
:1076D00025630D0020253E00632000002563000087
:1076E000202500003220EF00E3B723000080410096
:1076F0001040BA000160EF00000006000D0A000013
:107700003E4A0000546900006C74000044690000A7
:1077100072200000204400006972000065630000D0
:10772000746900006F6E00003A20000031200000F4
:1077300032200000332000003420000035200000FB
:1077400036200000370A00000D0000003220EF0054
:10775000C3012000830150000500310023BC230039
:10776000008041001040BA000160EF0000000600F8
:1077700020BC230083814100808141001380BA0036
:10778000000006000A0D20003E2034004A5420006C
:10779000696C200074533500706420003A2020008A
:1077A000506F3600727420002020200031203700F6
:1077B00020320A0020200D00332000003220EF008C
:1077C000C30120008301500005003100A3BF230046
:1077D000008041001040BA000160EF000000060088
:1077E000A0BF230083814100808141001380BA0043
:1077F000000006000A0D64003E202C0049642000B1
:107800006C655A005A6F6F006E656F003A206D000C
:1078100050613D006E3D2500256464002C200A0067
:1078200054690D006C743E003D2500003220EF00CD
:1078300023C22300008041001040BA000160EF0025
:10784000000006000A0D00003E2000005469000000
:107850006C7400005370000065650000643D00001A
:10786000256400000A0D00003E200000000000001A
:107870003220EF0043C42300008041001040BA00D2
:107880000160EF00000006000A0D00003E2000002D
:107890005A6F00006F6D00005370000065650000B6
:1078A000643D0000256400000A0D00003E20000039
:1078B000000000003220EF0063C62300008041007A
:1078C0001040BA000160EF00000006004F6E00009B
:1078D00020430000616D000065720000612000001F
:1078E000496E0000697400002C20000073650000E0
:1078F0006E640000204800006F6D000065200000ED
:10790000636F00006D6D0000616E0000640A00008E
:107910000D3E0000200000003220EF004302200056
:10792000830150000500310083CA2300008041001C
:107930001040BA000160EF000000060080CA23007A
:1079400083814100808141001380BA00000006005D
:107950004F6E6E0020436400616D200065727300FD
:1079600061206500496E7100697475002C20650006
:1079700073656E006E6463002050650072650A00D6
:1079800073650D0074203E00313420002063000038
:107990006F6D00006D6100003220EF006302200077
:1079A000830150000500310083CE23000080410098
:1079B0001040BA000160EF000000060080CE2300F6
:1079C00083814100808141001380BA0000000600DD
:1079D0000A0D34003E20200050726F006573720063
:1079E000657420004C6F3000633D29002831200071
:1079F0002D364C00206F6F0072206300312D610026
:107A000031346C0029200A00496E0D0043613E00AC
:107A10006D202000283700002D3100003220EF00BB
:107A2000A3D12300008041001040BA000160EF00A4
:107A3000000006000A0D00003E2000005072000009
:107A400065730000657400004C6F0000633D00002A
:107A5000416C00006C2000004C6F0000636100006E
:107A60006C0A00000D3E0000200000003220EF00F4
:107A700023D42300008041001040BA000160EF00D1
:107A8000000006002F6E00002F72000000000000B2
:107A90003220EF0043D52300008041001040BA009F
:107AA0000160EF00000006000A0D00003E530000D8
:107AB000657400004465000066610000756C00009C
:107AC0007420000025640000200A00000D3E000024
:107AD000200000003220EF0063D723000080410027
:107AE0001040BA000160EF00000006000A0D00001F
:107AF0003E44000065660000617500006C74000083
:107B0000436100006D20000025640000200A000091
:107B10000D3E0000200000003220EF0083D923003A
:107B2000008041001040BA000160EF000000060034
:107B30000A0D00003E20000053650000726900003D
:107B4000616C000045630000686F00003D45000067
:107B50006E610000626C0000656400000A0D0000A8
:107B60003E200000000000003220EF0003DC230074
:107B7000008041001040BA000160EF0000000600E4
:107B80000A0D00003E2000005365000072690000ED
:107B9000616C000045630000686F00003D44000018
:107BA00069730000616200006C650000640A0000F7
:107BB0000D3E0000200000003220EF0083DE230095
:107BC000008041001040BA000160EF000000060094
:107BD0000A0D00003E20000053650000726900009D
:107BE000616C0000496E0000666F00003D450000BA
:107BF0006E610000626C0000656400000A0D000008
:107C00003E200000000000003220EF0003E12300CE
:107C1000008041001040BA000160EF000000060043
:107C20000A0D00003E20000053650000726900004C
:107C3000616C0000496E0000666F00003D4400006A
:107C400069730000616200006C650000640A000056
:107C50000D3E0000200000003220EF0083E32300EF
:107C6000008041001040BA000160EF0000000600F3
:107C70000A0D00003E200000486F00006D65000006
:107C800042750000747400006F6E00003D440000F7
:107C900069730000616200006C650000640A000006
:107CA0000D3E0000200000003220EF0003E623001C
:107CB000008041001040BA000160EF0000000600A3
:107CC0000A0D00003E200000486F00006D650000B6
:107CD00042750000747400006F6E00003D450000A6
:107CE0006E610000626C0000656400000A0D000017
:107CF0003E200000000000003220EF0083E8230057
:107D0000008041001040BA000160EF000000060052
:107D1000202000002053000059530000544500006B
:107D20004D2000004D4500004E5500002020000071
:107D300020200000000000003220EF0083EA230032
:107D4000008041001040BA000160EF000000060012
:107D500020200000205300006572000069610000CF
:107D60006C200000496E0000707500007420000057
:107D700020200000000000003220EF0083EC2300F0
:107D8000008041001040BA000160EF0000000600D2
:107D9000202000002053000065720000696100008F
:107DA0006C20000045630000686F00002020000088
:107DB00020200000000000003220EF0083EE2300AE
:107DC000008041001040BA000160EF000000060092
:107DD000202000002053000065720000696100004F
:107DE0006C200000496E0000666F0000202000003B
:107DF00020200000000000003220EF0083F023006C
:107E0000008041001040BA000160EF000000060051
:107E10002020000020500000616E0000656C000012
:107E2000204C0000696700006874000073200000A7
:107E300020200000000000003220EF0083F2230029
:107E4000008041001040BA000160EF000000060011
:107E500020200000204300006C65000061720000DB
:107E6000204D0000656D00006F7200007920000059
:107E700020200000000000003220EF0083F42300E7
:107E8000008041001040BA000160EF0000000600D1
:107E900020200000204300006C650000617200009B
:107EA00020500000726500007365000074730000CC
:107EB00020200000000000003220EF0083F62300A5
:107EC000008041001040BA000160EF000000060091
:107ED00020200000506F0000776500007220000035
:107EE00055700000205000007265000073650000AE
:107EF00074200000000000003220EF0083F823000F
:107F0000008041001040BA000160EF000000060050
:107F100020200000507200006573000065740000AE
:107F2000204C00006F63000061740000696F000066
:107F30006E200000000000003220EF0083FA2300D2
:107F4000008041001040BA000160EF000000060010
:107F50002020000020440000756100006C2000001B
:107F60004C6900006E6B0000204D00006F64000043
:107F700065200000000000003220EF0083FC230099
:107F8000008041001040BA000160EF0000000600D0
:107F90002020000056690000646500006F2000008A
:107FA0005377000069740000636800006572000088
:107FB00020200000000000003220EF0083FE23009C
:107FC000008041001040BA000160EF000000060090
:107FD0002020000054720000616E000073690000F0
:107FE000746900006F6E000020540000696D00008D
:107FF00065200000000000003220EF008300240014
:10800000008041001040BA000160EF00000006004F
:108010002020000020540000616C00006C790000FA
:10802000204F00007574000070750000747300002C
:1080300020200000000000003220EF008302240016
:10804000008041001040BA000160EF00000006000F
:1080500020200000204800006F6D00006520000017
:1080600042750000747400006F6E00002020000054
:1080700020200000000000003220EF0083042400D4
:10808000008041001040BA000160EF0000000600CF
:108090002020000020500000414E0000204400003D
:1080A00049520000204D0000454E000055200000C0
:1080B00020200000000000003220EF008306240092
:1080C000008041001040BA000160EF00000006008F
:1080D0002020000020540000494C000054200000E3
:1080E00044490000522000004D4500004E5500005C
:1080F00020200000000000003220EF008308240050
:10810000008041001040BA000160EF00000006004E
:1081100020200000205A00004F4F00004D2000009A
:1081200044490000522000004D4500004E5500001B
:1081300020200000000000003220EF00830A24000D
:10814000008041001040BA000160EF00000006000E
:1081500020200000434100004D2000005345000056
:108160004152000043480000204D0000454E0000F1
:1081700055200000000000003220EF00830C240096
:10818000008041001040BA000160EF0000000600CE
:108190002020000043430000552000004D4F000008
:1081A00044450000204D0000454E000055200000D1
:1081B00020200000000000003220EF00830E240089
:1081C000008041001040BA000160EF00000006008E
:1081D000202000004E44000020460000494C0000D2
:1081E00054450000522000004D4500004E5500004F
:1081F00020200000000000003220EF008310240047
:10820000008041001040BA000160EF00000006004D
:10821000205300004855000054540000455200000F
:108220002053000050440000204D0000454E000047
:1082300055200000000000003220EF0083122400CF
:10824000008041001040BA000160EF00000006000D
:108250002020000020200000204100006C6C000065
:10826000205000006F720000747300002020000096
:1082700020200000000000003220EF0083142400C2
:10828000008041001040BA000160EF0000000600CD
:10829000202000002020000020200000506F00005F
:1082A0007274000020300000312000002020000007
:1082B00020200000000000003220EF008316240080
:1082C000008041001040BA000160EF00000006008D
:1082D000202000002020000020200000506F00001F
:1082E00072740000203000003220000020200000C6
:1082F00020200000000000003220EF00831824003E
:10830000008041001040BA000160EF00000006004C
:10831000202000002020000020200000506F0000DE
:108320007274000020300000332000002020000084
:1083300020200000000000003220EF00831A2400FB
:10834000008041001040BA000160EF00000006000C
:10835000202000002020000020200000506F00009E
:108360007274000020300000342000002020000043
:1083700020200000000000003220EF00831C2400B9
:10838000008041001040BA000160EF0000000600CC
:10839000202000002020000020200000506F00005E
:1083A0007274000020300000352000002020000002
:1083B00020200000000000003220EF00831E240077
:1083C000008041001040BA000160EF00000006008C
:1083D000202000002020000020200000506F00001E
:1083E00072740000203000003620000020200000C1
:1083F00020200000000000003220EF008320240035
:10840000008041001040BA000160EF00000006004B
:10841000202000002020000020200000506F0000DD
:10842000727400002030000037200000202000007F
:1084300020200000000000003220EF0083222400F2
:10844000008041001040BA000160EF00000006000B
:108450002020000020200000204D000041490000A5
:108460004E2000004D4500004E5500002020000029
:1084700020200000000000003220EF0083242400B0
:10848000008041001040BA000160EF0000000600CB
:10849000202000005265000073630000616E000040
:1084A00020430000616D00006572000061730000F0
:1084B00020200000000000003220EF00832624006E
:1084C000008041001040BA000160EF00000006008B
:1084D00020200000436100006D2000005365000073
:1084E0006172000063680000204D0000656E0000AE
:1084F00075200000000000003220EF0083282400D7
:10850000008041001040BA000160EF00000006004A
:108510002044000065660000617500006C74000076
:1085200020430000616D00006572000061200000C2
:108530004E6F0000000000003220EF00832A24006C
:10854000008041001040BA000160EF00000006000A
:108550002044000065660000617500006C74000036
:108560002050000072650000736500007420000058
:108570004E6F0000000000003220EF00832C24002A
:10858000008041001040BA000160EF0000000600CA
:10859000202000002043000043550000204D000033
:1085A0006F640000652000004D6500006E750000DE
:1085B00020200000000000003220EF00832E240065
:1085C000008041001040BA000160EF00000006008A
:1085D0002020000020500000616E000020440000B8
:1085E00069720000204D0000656E000075200000DB
:1085F00020200000000000003220EF008330240023
:10860000008041001040BA000160EF000000060049
:108610002020000020540000696C0000742000003D
:1086200044690000722000004D6500006E75000076
:1086300020200000000000003220EF0083322400E0
:10864000008041001040BA000160EF000000060009
:1086500020200000205A00006F6F00006D200000F5
:1086600044690000722000004D6500006E75000036
:1086700020200000000000003220EF00833424009E
:10868000008041001040BA000160EF0000000600C9
:1086900020430000616D0000657200006120000051
:1086A000536500006C650000637400002042000008
:1086B00075730000000000003220EF0083362400B4
:1086C000008041001040BA000160EF000000060089
:1086D00020500000726500007365000074200000E7
:1086E000506100006E2000005370000065650000BE
:1086F00064200000000000003220EF0083382400D6
:10870000008041001040BA000160EF000000060048
:1087100020500000726500007365000074200000A6
:10872000546900006C740000205300007065000064
:1087300065640000000000003220EF00833A24004E
:10874000008041001040BA000160EF000000060008
:108750002050000072650000736500007420000066
:108760005A6F00006F6D000020530000706500001C
:1087700065640000000000003220EF00833C24000C
:10878000008041001040BA000160EF0000000600C8
:1087900020430000616E00006F6E0000204E00005C
:1087A00044200000466900006C74000065720000FF
:1087B00020200000000000003220EF00833E240053
:1087C000008041001040BA000160EF000000060088
:1087D00020430000616E00006F6E00002053000017
:1087E000687500007474000065720000205300007A
:1087F00070640000000000003220EF00834024007D
:10880000008041001040BA000160EF000000060047
:108810002020000020200000537900007374000025
:10882000656D0000204D0000656E000075200000A1
:1088300020200000000000003220EF0083422400CE
:10884000008041001040BA000160EF000000060007
:108850002020000020200000202000005374000091
:108860006172000074200000202000002020000021
:1088700020200000000000003220EF00834424008C
:10888000008041001040BA000160EF0000000600C7
:108890002020000020200000204300006F6E000018
:1088A000747200006F6C0000204100002020000066
:1088B00020200000000000003220EF00834624004A
:1088C000008041001040BA000160EF000000060087
:1088D0002020000020200000204300006F6E0000D8
:1088E000747200006F6C0000204200002020000025
:1088F00020200000000000003220EF008348240008
:10890000008041001040BA000160EF000000060046
:108910002020000020200000202000002020000057
:108920004F4E0000202000002020000020200000EA
:1089300020200000000000003220EF00834A2400C5
:10894000008041001040BA000160EF000000060006
:10895000202000002020000020200000204F0000E8
:1089600046460000202000002020000020200000BB
:1089700020200000000000003220EF00834C240083
:10898000008041001040BA000160EF0000000600C6
:108990002020000020200000204800006F6D000013
:1089A00065200000436100006D65000072610000F9
:1089B00020200000000000003220EF00834E240041
:1089C000008041001040BA000160EF000000060086
:1089D00020200000202000002050000072650000D0
:1089E0007365000074200000313400002020000076
:1089F00020200000000000003220EF0083502400FF
:108A0000008041001040BA000160EF000000060045
:108A10002020000020200000204100006C6C00009D
:108A2000204C00006F630000616C000020200000FB
:108A300020200000000000003220EF0083522400BC
:108A4000008041001040BA000160EF000000060005
:108A50002020000036200000496E00004361000025
:108A60006D200000382000004C6F000063610000A2
:108A70006C200000000000003220EF00835424002E
:108A8000008041001040BA000160EF0000000600C5
:108A900020200000204E00006F7200006D61000079
:108AA0006C6C0000792000004F700000656E0000C3
:108AB00020200000000000003220EF008356240038
:108AC000008041001040BA000160EF000000060085
:108AD00020200000204E00006F7200006D61000039
:108AE0006C6C000079200000436C00006F73000084
:108AF00065640000000000003220EF00835824006D
:108B0000008041001040BA000160EF000000060044
:108B10002020000020200000202000002020000055
:108B20004E6F00006E650000202000002020000035
:108B300020200000000000003220EF00835A2400B3
:108B4000008041001040BA000160EF000000060004
:108B5000202000002045000064690000726F0000C2
:108B60006C200000344800002C200000335300002B
:108B700020200000000000003220EF00835C240071
:108B8000008041001040BA000160EF0000000600C4
:108B9000204900006E6F00007661000074690000DB
:108BA0006F6E000020620000792000004953000031
:108BB00049530000000000003220EF00835E2400D3
:108BC000008041001040BA000160EF000000060084
:108BD0002020000020550000736500007220000076
:108BE00044650000666900006E65000064200000B6
:108BF00020200000000000003220EF0083602400ED
:108C0000008041001040BA000160EF000000060043
:108C10002020000020200000202000004E6F0000D7
:108C2000726D0000616C0000202000002020000018
:108C300020200000000000003220EF0083622400AA
:108C4000008041001040BA000160EF000000060003
:108C5000202000002020000020200000496E00009D
:108C600076650000727400002020000020200000C3
:108C700020200000000000003220EF008364240068
:108C8000008041001040BA000160EF0000000600C3
:108C900020410000757400006F2000005365000043
:108CA0006172000063680000204D00006F640000E6
:108CB00065200000000000003220EF0083662400E1
:108CC000008041001040BA000160EF000000060083
:108CD0002020000020200000205300006F6E0000C4
:108CE000792000004F6E00006C7900002020000009
:108CF00020200000000000003220EF0083682400E4
:108D0000008041001040BA000160EF000000060042
:108D10002020000020200000436100006E6F000052
:108D20006E2000004F6E00006C79000020200000D3
:108D300020200000000000003220EF00836A2400A1
:108D4000008041001040BA000160EF000000060002
:108D500020430000616E00006F6E0000204F000095
:108D60006E6C00007920000049530000204F000085
:108D70006E200000000000003220EF00836C240011
:108D8000008041001040BA000160EF0000000600C2
:108D900020200000506100006E610000736F000031
:108DA0006E690000632000004F6E00006C790000C7
:108DB00020200000000000003220EF00836E24001D
:108DC000008041001040BA000160EF000000060082
:108DD0002020000020200000204E00006F20000016
:108DE000436100006D6500007261000020200000FA
:108DF00020200000000000003220EF0083702400DB
:108E0000008041001040BA000160EF000000060041
:108E100020200000446900007265000063740000B7
:108E200020430000616D00002043000074720000C8
:108E30006C200000000000003220EF00837224004C
:108E4000008041001040BA000160EF000000060001
:108E50002020000043430000552000004361000033
:108E60006D200000436F00006E740000726F000000
:108E70006C200000000000003220EF00837424000A
:108E8000008041001040BA000160EF0000000600C1
:108E9000202000002020000020200000204F0000A3
:108EA0006666000020200000202000002020000036
:108EB00020200000000000003220EF008376240014
:108EC000008041001040BA000160EF000000060081
:108ED0002020000020200000202000002031000081
:108EE0002F3600002020000020200000202000005D
:108EF00020200000000000003220EF0083782400D2
:108F0000008041001040BA000160EF000000060040
:108F10002020000020200000202000002031000040
:108F20002F3300003220000020200000202000000D
:108F300020200000000000003220EF00837A24008F
:108F4000008041001040BA000160EF000000060000
:108F500020200000202000002020000044690000A4
:108F600073610000626C000065200000202000009A
:108F700020200000000000003220EF00837C24004D
:108F8000008041001040BA000160EF0000000600C0
:108F9000204E00005453000043200000312F0000F9
:108FA00034200000504100004C200000312F000010
:108FB00033200000000000003220EF00837E2400F8
:108FC000008041001040BA000160EF000000060080
:108FD000202000002020000020200000312F000071
:108FE000313500002020000020200000312F00003B
:108FF00031320000000000003220EF0083802400A6
:10900000008041001040BA000160EF00000006003F
:10901000202000002020000020200000312F000030
:10902000363000002020000020200000312F0000FA
:1090300035300000000000003220EF008382240061
:10904000008041001040BA000160EF0000000600FF
:10905000202000002020000020200000312F0000F0
:1090600031300000302000002020000020200000CF
:1090700020200000000000003220EF008384240044
:10908000008041001040BA000160EF0000000600BF
:10909000202000002020000020200000312F0000B0
:1090A000313000003030000020200000202000007F
:1090B00020200000000000003220EF008386240002
:1090C000008041001040BA000160EF00000006007F
:1090D0002053000079730000746500006D200000CB
:1090E000496E000020530000746100006E640000AF
:1090F00062790000000000003220EF008388240025
:10910000008041001040BA000160EF00000006003E
:10911000556E000065780000706500006374000003
:1091200065640000205500004152000054310000E9
:1091300020450000727200006F7200000A0D0000EE
:10914000000000003220EF00E38A2400008041008C
:109150001040BA000160EF0000000600556E0000EC
:1091600065780000706500006374000065640000AD
:1091700020550000415200005432000020450000FC
:10918000727200006F7200000A0D00000000000003
:109190003220EF00438D2400008041001040BA00CF
:1091A0000160EF0000000600556E000065780000C9
:1091B00070650000637400006564000020530000C7
:1091C00054410000434B0000455200005220000073
:1091D00045720000726F0000720A00000D0000006E
:1091E0003220EF00C38F2400008041001040BA00FD
:1091F0000160EF0000000600556E00006578000079
:109200007065000063740000656400002041000088
:109210004444000052450000525200002045000026
:10922000727200006F7200000A0D00000000000062
:109230003220EF0043922400008041001040BA0029
:109240000160EF0000000600556E00006578000028
:10925000706500006374000065640000204D00002C
:1092600041540000484500005252000020450000D3
:10927000727200006F7200000A0D00000000000012
:109280003220EF00C3942400008041001040BA0057
:109290000160EF0000000600556E000065780000D8
:1092A00070650000637400006564000020640000C5
:1092B00065660000617500006C74000020450000C8
:1092C000727200006F7200000A0D000000000000C2
:1092D0003220EF0043972400008041001040BA0084
:1092E0000160EF0000000600536500007269000095
:1092F000616C0000204200006F6F000074200000CD
:109300004C6F000061640000203F0000000000007E
:109310003220EF0043992400008041001040BA0041
:109320000160EF0000000600204800006F6C0000A4
:10933000642000004D61000073740000657200003D
:10934000506F0000776500007220000000000000F0
:109350003220EF00439B2400008041001040BA00FF
:109360000160EF0000000600666F00007220000040
:10937000342000007365000063200000746F00005B
:1093800020530000746100007274000000000000AF
:109390003220EF00439D2400008041001040BA00BD
:1093A0000160EF00000006002020000020420000C5
:1093B0006F6F0000742000006C6F0000616400009B
:1093C0006572000020200000202000000000000046
:1093D0003220EF00439F2400008041001040BA007B
:1093E0000160EF00000006002020000020200000A7
:1093F0002566000020730000656300002020000047
:109400002020000020200000200000003220EF007B
:1094100023A12400008041001040BA000160EF0049
:10942000000006002020000020520000656C0000B3
:109430006561000073650000207400006F2000006B
:109440002020000020200000000000003220EF005B
:1094500023A32400008041001040BA000160EF0007
:10946000000006002020000020200000436F0000C4
:109470006E740000696E0000756500002020000019
:109480002020000020200000000000003220EF001B
:1094900023A52400008041001040BA000160EF00C5
:1094A00000000600202000002020000020200000F6
:1094B00020200000202000002020000020200000AC
:1094C0002020000020200000000000003220EF00DB
:1094D00023A72400008041001040BA000160EF0083
:1094E00000000600426F00006F7400006C6F000007
:1094F0006164000065720000205300007461000088
:109500007274000065640000000000003220EF006B
:1095100023A92400008041001040BA000160EF0040
:1095200000000600746F0000204300006F6E000012
:1095300066690000726D0000205200006571000035
:109540007565000073740000000000003220EF0019
:1095500023AB2400008041001040BA000160EF00FE
:109560000000060020200000204200006F6F000075
:1095700074200000526500007175000065730000E2
:109580007420000020200000000000003220EF00C6
:1095900023AD2400008041001040BA000160EF00BC
:1095A00000000600204300006F6E00007469000098
:1095B0006E75000065200000486F00006C640000BC
:1095C000696E000067200000000000003220EF00FC
:1095D00023AF2400008041001040BA000160EF007A
:1095E00000000600204200006F6F0000746C000055
:1095F0006F6100006420000053740000617200007D
:109600007465000064200000000000003220EF00BC
:1096100023B12400008041001040BA000160EF0037
:10962000000006002020000020200000202500006F
:10963000730000003220EF0063B22400008041007C
:109640001040BA000160EF00000006002049000051
:109650006E69000074690000616C00007A650000AA
:109660002045000045500000726F00006D20000092
:10967000000000003220EF0063B4240000804100AD
:109680001040BA000160EF00000006002045000015
:1096900045500000726F00006D200000496E000010
:1096A00069740000696100006C7A00006564000064
:1096B000200000003220EF0063B62400008041004B
:1096C0001040BA000160EF0000000600204C0000CE
:1096D0006F610000646900006E67000020440000B4
:1096E00065660000617500006C7400007320000066
:1096F000000000003220EF0063B824000080410029
:109700001040BA000160EF00000006002043000096
:1097100043550000204900006E69000074200000DD
:109720005761000069740000202000002020000024
:10973000000000003220EF0063BA240000804100E6
:109740001040BA000160EF00000006002020000079
:109750002020000020200000202000002020000009
:1097600020200000202000002020000020200000F9
:10977000200000004200F8003600F800801F78004A
:10978000200020000C000900B01F7800010020001C
:10979000010078007C480200000000008100E80021
:1097A000811F78002322AF00FEFF370020118800C0
:1097B000CF007800700120000008E600F4FF3700B9
:1097C0008C20A9008C20A900A00120000C00090019
:1097D0004F1078004F0078003600F9004200F90081
:1097E000004006004200F8003600F800801F7800B4
:1097F000200020000C000900B01F780001002000AC
:1098000001007800A2480200000000008100E8008A
:10981000811F78002322AF00FEFF3700201188004F
:10982000CF007800700120000008E600F4FF370048
:109830008C40A9008C40A900A00120000C00090068
:109840004F1078004F0078003600F9004200F90010
:10985000004006004200F8003600F800801F780043
:10986000200020000C000900B01F7800010020003B
:1098700001007800C8480200000000008100E800F4
:10988000811F78002322AF00FEFF370020118800DF
:10989000CF007800A00120000008E600F4FF3700A8
:1098A0008040A9008040A900A00120000C00090010
:1098B0004F1078004F0078003600F9004200F900A0
:1098C000004006004200F8003600F800801F7800D3
:1098D000200020000C000900B01F780001002000CB
:1098E00001007800F0480200000000008100E8005C
:1098F000811F78002322AF00FEFF3700201188006F
:10990000CF007800900120000008E600F4FF370047
:109910008060A9008060A900A00120000C0009005F
:109920004F1078004F0078003600F9004200F9002F
:10993000004006004200F8003600F800801F780062
:10994000200020000C000900B01F7800010020005A
:109950000100780018490200000000008100E800C2
:10996000811F78002322AF00FEFF370020118800FE
:10997000CF007800900120000008E600F4FF3700D7
:109980008080A9008080A900A00120000C000900AF
:109990004F1078004F0078003600F9004200F900BF
:1099A000004006004200F8003600F800801F7800F2
:1099B000200020000C000900B01F780001002000EA
:1099C0000100780040490200000000008100E8002A
:1099D000811F78002322AF00FEFF3700201188008E
:1099E000CF007800900120000008E600F4FF370067
:1099F000A00120000C0009004F1078004F007800F3
:109A00003600F9004200F900004006004200F8006C
:109A10003600F800801F7800200020000C000900AC
:109A2000B01F7800D041810000C0B300D041890050
:109A3000D04181000160EF00D04189002202AE00D8
:109A4000FEFF3700301180003A28F800F0FF9F0039
:109A50003A28F900644D80004822DE00E39A200095
:109A6000830242003A28F8004F0078004800DE00E8
:109A7000804A7800ADC9BF003A28F800E0FF9F0097
:109A80003A28F900644D80004822DE00614242001D
:109A90000440780000E0B700F40F20000024E1004B
:109AA00004003A0000003700AD69EF005C4D04008F
:109AB00000000000AD69EC00ADC9BF00AD4AE30095
:109AC00003003A0000003700D0418100ADE9B70043
:109AD000D04181004800DE006D04E10002003A0040
:109AE00000003700AE6AEC004148A80049C9BF0039
:109AF0007F4060000004E00050003A0000003700A2
:109B00008C08AE00010037004C0037004769AF00F9
:109B10000100370049003700D04181004800DE00D5
:109B2000140220000024E10001003A000C0037007C
:109B3000D04181004800DE00240220000024E10022
:109B400001003A0006003700D04181004800DE00E5
:109B5000040320000024E10010003A000000370058
:109B6000444380004822DE0013082000041CE1006A
:109B70000A003E0000003700444380004822DE0017
:109B800093082000041CE1000400390000003700A5
:109B9000D04181000160EF00D0418900D0418100B7
:109BA0004800DE007F04E1000700360000003700B7
:109BB000D04181004800DE00F40720000024E100CD
:109BC0000100360005003700D04181004800DE006A
:109BD0006804E10019003A00000037003A28F80054
:109BE0004F0078004800DE002322AF00FEFF370060
:109BF00024E2B7002562EF00D04181004800DE007A
:109C00006804E1000D003A000000370000C2B30014
:109C10002322AF00FEFF370024E2B7002562EF00E9
:109C20003A28F8004F0078004800DE002322AF00F9
:109C3000FEFF370024E2B7002562EF003A28F80063
:109C40004F0078004800DE0069E8B7009560A80082
:109C50008560A900A00120000C0009004F107800C9
:109C60004F0078003600F9004200F900004006007D
:109C70004200F8003600F800801F78002000200025
:109C80000C000900B01F7800D041810000C0B30073
:109C9000D04189003202AE00FEFF3700B0118000D3
:109CA0003A28F800E0FF9F003A28F9008C28AF001E
:109CB0000100370007003700D04181002322AF00A8
:109CC000FEFF370024E2B7002562EF00924E040049
:109CD00000000000745580004822DE0003AB200025
:109CE00083024200D0418100804298004168A80070
:109CF000745580004822DE00614242000440780032
:109D000000E0B700F40720000024E10004003E005A
:109D100000003700AF6AEF00924E04000000000020
:109D2000AF6AEC0097C0A80087C0A900A00120007E
:109D30000C0009004F1078004F0078003600F90041
:109D40004200F900004006004200F8003600F8002A
:109D5000801F7800200020000C000900B01F780050
:109D600004002000D441890004002000E44189005F
:109D700004002000F441890004002000044289000E
:109D800004002000144289000400200024428900BD
:109D900004002000344289004042810000C0B3002A
:109DA00040428900404281000160EF00404289004A
:109DB0005042810000C0B3005042890050428100EF
:109DC0000160EF00504289006042810000C0B30092
:109DD00060428900604281000160EF0060428900BA
:109DE0009500A900F4F72F0094168800D402F8001B
:109DF0003A28F900D041810000027800F0F72700EE
:109E000004006000F0418900F04181007288B600D2
:109E1000104289001418280024178800E602F80070
:109E20003C28F900E0418100000278001018280069
:109E30000400600000428900004281007488B6007E
:109E400020428900104281000000E0000100320041
:109E500004003700204281000000E000A40032002E
:109E600000003700104281000000E0005400320082
:109E700000003700104281004A28F800E0FF9F00F0
:109E80004A28F9004228F8004F0078004800DE0018
:109E90004A28F800F0FF9F004A28F900504281004C
:109EA0000160EF00544281004822DE002E08F800D5
:109EB000F4FF9F002E08F9002FE8B60072C8BF001B
:109EC0004C28F800E0FF9F004C28F90073C8BF0041
:109ED0004C28F800F0FF9F004C28F9005042810008
:109EE0004800DE00644281000960EF000440680021
:109EF0004828F800E0FF9F004828F900F041810061
:109F00004A28F800E0FF9F004A28F90050428100EB
:109F10000160EF00644281004822DE001C08F80066
:109F2000F4FF9F001C08F9001DE8B60004002000A3
:109F300034428900304281006700E1001E00310098
:109F4000000037002FC8BF00800078003042810039
:109F50000100A50001003100120037001DC8BF003C
:109F600080007800304281000100A5000100390026
:109F700007003700304281004100DD008487200067
:109F800084024000950AE900D24F0400000000005E
:109F9000304281004100DD008487200084024000BF
:109FA000950AE800304281000000E8003042890054
:109FB0009A4F0400000000003E28F8007208F900E3
:109FC000204281000000E000450032000000370020
:109FD000204281004A28F800E0FF9F004A28F9004B
:109FE0004428F8004F0078004800DE004A28F800B6
:109FF000F0FF9F004A28F900504281000160EF0005
:10A00000544281004822DE002E08F800F4FF9F0031
:10A010002E08F9002FE8B60074C8BF004C28F800DD
:10A02000E0FF9F004C28F90075C8BF004C28F800DD
:10A03000F0FF9F004C28F900504281004800DE00EC
:10A04000644281000960EF00044068004828F8007D
:10A05000E0FF9F004828F900004281004A28F800EC
:10A06000E0FF9F004A28F900504281000160EF00A4
:10A07000644281004822DE001C08F800F4FF9F00C3
:10A080001C08F9001DE8B6002F08AF0001003700DA
:10A09000070037001D08AE0001003700030037003D
:10A0A0008628ED0058500400000000008628EC00CF
:10A0B0002FE8AF0001003700070037001DE8AE00B1
:10A0C00001003700030037008828ED006C500400C1
:10A0D000000000008828EC004028F8007408F9000F
:10A0E0004108A8007628EF007A5004000000000024
:10A0F0007628EC002003A9002023A8002003AE004E
:10A10000FEFF3700001880004200DE004828F800FB
:10A11000F0FF9F004828F90064A280006D405200C3
:10A120000080FB00E4442100840240004828F8003D
:10A130004F0078004800DE00804A78004C74EC0044
:10A1400064A280006F24E1000300360000003700A5
:10A15000D0C0B3004CF4B7004CD4BF0028E3B70024
:10A160002963EF008500A9009500A8008500A900DB
:10A17000A00120000C0009004F1078004F0078006B
:10A180003600F9004200F90000400600820020007D
:10A190001E00090000000000C4E2A900C0E2A900FE
:10A1A0001F0009000000000081C0D200C4C2A90045
:10A1B0004200AF00C0C2A8004200AE00C0C2A90069
:10A1C000C0E2A800C2E2AE00FEFF37000201E900D3
:10A1D000EFFF3A001E00090000000000C4E2A900E1
:10A1E000C0E2A90000000000C0C2A8001F000900D2
:10A1F000000000001F00090000000000C0E2A800ED
:10A20000C2E2AE00FEFF37001F00090000000000A0
:10A2100000002000C2C2AF000000A000C4E2A900FC
:10A22000C0E2A900C4C2A900C0C2A9000000060083
:10A23000C0C2A8001E00090000000000C0E2A80083
:10A240001F00090000000000C2E2AE00FEFF370060
:10A25000C4C2A900C0C2A9001E000900000000007D
:10A26000C4E2A900C0E2A9009E00090000000000AD
:10A2700061C4B300C6500200000000009E00090047
:10A280000000000061428100C65002000000000092
:10A290009E000900000000004C28F800CF00780064
:10A2A000C808DE00C6500200000000009E00090041
:10A2B00000000000C0C2A90000000000C0E2A80029
:10A2C000C2E2AE00FEFF37001E00090000000000E1
:10A2D0000100090000000000C0C2A8001E00090023
:10A2E00000000000BE0009000000000000000600A1
:10A2F000204281000160EF001080B2004D0032006A
:10A300007080B200570032005080B2005500320019
:10A310007080B200530032003080B2005100320031
:10A32000F080B2004F003200D080B2004D00320009
:10A330009081B200B80032001080B200B600320046
:10A340003080B200B40032001080B200B20032009F
:10A35000F083B200B00032001080B200AE003200D4
:10A360003080B200AC0032001080B2002D0132000B
:10A370007080B2002B0132001080B200290132003F
:10A380003080B200270132001080B2002501320077
:10A39000F080B200230132001080B20021013200AF
:10A3A000D083B200AA0132007080B200A80132004E
:10A3B0001080B200A60132003080B200A401320049
:10A3C0001080B200A2013200F081B200A001320080
:10A3D0001080B2009E0132005081B200190232009A
:10A3E0001080B200170232003080B2001502320035
:10A3F0001080B20013023200F080B200110232006D
:10A400001080B2000F0232003080B2000D02320024
:10A41000C085B200880232003080B2009302320060
:10A420001080B2009E0232007080B200B40232008E
:10A43000EC023700204281004800DE000004E0000A
:10A4400004003A00DCC2A800D8C2A9002E520400C1
:10A4500000000000DCC2A900D8C2A900F257040025
:10A4600000000000204281004800DE000004E000FF
:10A4700030003A00204281000160EF006604E100F4
:10A4800004003A00241421001400A1009652040094
:10A4900000000000204281000160EF006304E10041
:10A4A00004003A00241421001410A1009652040064
:10A4B00000000000204281000160EF006404E10020
:10A4C00004003A00241421001420A1009652040034
:10A4D00000000000204281000160EF006704E100FD
:10A4E00004003A00241421001430A1009652040004
:10A4F00000000000204281000160EF006804E100DC
:10A5000004003A00241421001440A10096520400D3
:10A5100000000000204281000160EF006504E100BE
:10A5200002003A00241421001450A100F652040045
:10A5300000000000204281000160EF006604E1009D
:10A5400004003A00241421001400A000F652040074
:10A5500000000000204281000160EF006304E10080
:10A5600004003A00241421001410A000F652040044
:10A5700000000000204281000160EF006404E1005F
:10A5800004003A00241421001420A000F652040014
:10A5900000000000204281000160EF006704E1003C
:10A5A00004003A00241421001430A000F6520400E4
:10A5B00000000000204281000160EF006804E1001B
:10A5C00004003A00241421001440A000F6520400B4
:10A5D00000000000204281000160EF006504E100FE
:10A5E00002003A00241421001450A00060428100AF
:10A5F00080C0B3006042890042D1BF004C28F800FF
:10A60000F0FF9F004C28F9001851020000000000E4
:10A61000F257040000000000204281004800DE00E4
:10A620000004E0003B003A00204281000160EF009E
:10A630007C04E10004003A00441421001410A1003D
:10A640008653040000000000204281000160EF00FA
:10A650007D04E10004003A00441421001420A1000C
:10A660008653040000000000204281000160EF00DA
:10A670007E04E10004003A00441421001430A100DB
:10A680008653040000000000204281000160EF00BA
:10A690007F04E10004003A00441421001440A100AA
:10A6A0008653040000000000204281000160EF009A
:10A6B000040220000024E10004003A0044142100B8
:10A6C0001450A100865304000000000020428100C5
:10A6D0000160EF00140220000024E10004003A00B1
:10A6E000441421001460A1008653040000000000FF
:10A6F000204281000160EF00240220000024E100DC
:10A7000002003A00441421001470A100FC5304001C
:10A7100000000000204281000160EF007C04E100A5
:10A7200004003A00441421001410A000FC5304005B
:10A7300000000000204281000160EF007D04E10084
:10A7400004003A00441421001420A000FC5304002B
:10A7500000000000204281000160EF007E04E10063
:10A7600004003A00441421001430A000FC530400FB
:10A7700000000000204281000160EF007F04E10042
:10A7800004003A00441421001440A000FC530400CB
:10A7900000000000204281000160EF000402200060
:10A7A0000024E10004003A00441421001450A000E9
:10A7B000FC53040000000000204281000160EF0013
:10A7C000140220000024E10004003A004414210097
:10A7D0001460A000FC53040000000000204281002F
:10A7E0000160EF00240220000024E10002003A0092
:10A7F000441421001470A0006042810090C0B30096
:10A800006042890044D1BF004C28F800F0FF9F004F
:10A810004C28F9001851020000000000F257040013
:10A8200000000000204281004800DE000004E0003B
:10A830003F003A00204281000160EF003402200016
:10A840000024E10004003A00641421001410A10067
:10A850009454040000000000204281000160EF00D9
:10A86000440220000024E10004003A0064142100A6
:10A870001420A10094540400000000002042810034
:10A880000160EF00540220000024E10004003A00BF
:10A89000641421001430A10094540400000000004E
:10A8A000204281000160EF00640220000024E100EA
:10A8B00004003A00641421001440A10094540400E0
:10A8C00000000000204281000160EF0074022000BF
:10A8D0000024E10004003A00641421001450A10097
:10A8E0009454040000000000204281000160EF0049
:10A8F000840220000024E10004003A0064142100D6
:10A900001460A10094540400000000002042810063
:10A910000160EF00940220000024E10002003A00F0
:10A92000641421001470A1001255040000000000FE
:10A93000204281000160EF00340220000024E10089
:10A9400004003A00641421001410A0001255040001
:10A9500000000000204281000160EF00440220005E
:10A960000024E10004003A00641421001420A00037
:10A970001255040000000000204281000160EF0039
:10A98000540220000024E10004003A006414210075
:10A990001430A00012550400000000002042810085
:10A9A0000160EF00640220000024E10004003A008E
:10A9B000641421001440A00012550400000000009F
:10A9C000204281000160EF00740220000024E100B9
:10A9D00004003A00641421001450A0001255040031
:10A9E00000000000204281000160EF00840220008E
:10A9F0000024E10004003A00641421001460A00067
:10AA00001255040000000000204281000160EF00A8
:10AA1000940220000024E10002003A0064142100A6
:10AA20001470A00060428100A0C0B30060428900A1
:10AA300046D1BF004C28F800F0FF9F004C28F900D9
:10AA40001851020000000000F2570400000000004E
:10AA5000204281004800DE000004E00038003A0097
:10AA6000204281000160EF007404E10004003A001C
:10AA7000841421001410A1009C5504000000000063
:10AA8000204281000160EF007304E10004003A00FD
:10AA9000841421001420A1009C5504000000000033
:10AAA000204281000160EF007204E10004003A00DE
:10AAB000841421001430A1009C5504000000000003
:10AAC000204281000160EF007104E10004003A00BF
:10AAD000841421001440A1009C55040000000000D3
:10AAE000204281000160EF007004E10004003A00A0
:10AAF000841421001450A1009C55040000000000A3
:10AB0000204281000160EF006F04E10004003A0080
:10AB1000841421001460A1009C5504000000000072
:10AB2000204281000160EF006E04E10002003A0063
:10AB3000841421001470A1000C56040000000000D1
:10AB4000204281000160EF007404E10004003A003B
:10AB5000841421001410A0000C5604000000000012
:10AB6000204281000160EF007304E10004003A001C
:10AB7000841421001420A0000C56040000000000E2
:10AB8000204281000160EF007204E10004003A00FD
:10AB9000841421001430A0000C56040000000000B2
:10ABA000204281000160EF007104E10004003A00DE
:10ABB000841421001440A0000C5604000000000082
:10ABC000204281000160EF007004E10004003A00BF
:10ABD000841421001450A0000C5604000000000052
:10ABE000204281000160EF006F04E10004003A00A0
:10ABF000841421001460A0000C5604000000000022
:10AC0000204281000160EF006E04E10002003A0082
:10AC1000841421001470A00060428100B0C0B30011
:10AC20006042890048D1BF004C28F800F0FF9F0027
:10AC30004C28F9001851020000000000F2570400EF
:10AC400000000000204281004800DE000004E00017
:10AC500038003A00204281000160EF007B04E100EF
:10AC600004003A00A41421001410A1009656040018
:10AC700000000000204281000160EF007A04E10042
:10AC800004003A00A41421001420A10096560400E8
:10AC900000000000204281000160EF007904E10023
:10ACA00004003A00A41421001430A10096560400B8
:10ACB00000000000204281000160EF007804E10004
:10ACC00004003A00A41421001440A1009656040088
:10ACD00000000000204281000160EF007704E100E5
:10ACE00004003A00A41421001450A1009656040058
:10ACF00000000000204281000160EF007604E100C6
:10AD000004003A00A41421001460A1009656040027
:10AD100000000000204281000160EF007504E100A6
:10AD200002003A00A41421001470A1000657040088
:10AD300000000000204281000160EF007B04E10080
:10AD400004003A00A41421001410A00006570400C7
:10AD500000000000204281000160EF007A04E10061
:10AD600004003A00A41421001420A0000657040097
:10AD700000000000204281000160EF007904E10042
:10AD800004003A00A41421001430A0000657040067
:10AD900000000000204281000160EF007804E10023
:10ADA00004003A00A41421001440A0000657040037
:10ADB00000000000204281000160EF007704E10004
:10ADC00004003A00A41421001450A0000657040007
:10ADD00000000000204281000160EF007604E100E5
:10ADE00004003A00A41421001460A00006570400D7
:10ADF00000000000204281000160EF007504E100C6
:10AE000002003A00A41421001470A00060428100E6
:10AE1000C0C0B300604289004AD1BF004C28F8008E
:10AE2000F0FF9F004C28F9001851020000000000BC
:10AE3000F257040000000000F40F2000448A88004C
:10AE400060428100B0C0B3006042890048D1BF00B9
:10AE50004C28F800F0FF9F004C28F9001851020020
:10AE600000000000F257040000000000F40F200072
:10AE7000548A880060428100C0C0B30060428900EB
:10AE80004AD1BF004C28F800F0FF9F004C28F90081
:10AE90001851020000000000F257040000000000FA
:10AEA000F40F2000248A88006042810090C0B30023
:10AEB0006042890044D1BF004C28F800F0FF9F0099
:10AEC0004C28F9001851020000000000F40F200087
:10AED000348A880060428100A0C0B30060428900CB
:10AEE00046D1BF004C28F800F0FF9F004C28F90025
:10AEF0001851020000000000F2570400000000009A
:10AF0000F40F2000148A88006042810080C0B300E2
:10AF10006042890042D1BF004C28F800F0FF9F003A
:10AF20004C28F9001851020000000000F40F200026
:10AF3000248A88006042810090C0B300604289008A
:10AF400044D1BF004C28F800F0FF9F004C28F900C6
:10AF50001851020000000000F40F2000348A88001D
:10AF600060428100A0C0B3006042890046D1BF00AA
:10AF70004C28F800F0FF9F004C28F90018510200FF
:10AF800000000000F40F2000448A88006042810025
:10AF9000B0C0B3006042890048D1BF004C28F8001F
:10AFA000F0FF9F004C28F90018510200000000003B
:10AFB000F40F2000548A880060428100C0C0B300B2
:10AFC000604289004AD1BF004C28F800F0FF9F0082
:10AFD0004C28F9001851020000000000F25704004C
:10AFE0000000000000000600404281000160EF0008
:10AFF00040428900404281000160EF009082B2002F
:10B000001B0032001080B2001F003200F080B2003E
:10B01000230032001080B200270032003080B200DE
:10B020002B0032001080B2002F0032007080B2007E
:10B03000330032001080B200370032003080B2009E
:10B040003B0032001080B2003F003200F083B200BB
:10B05000430032001080B200470032003080B2005E
:10B060004B0032001080B2004F0032004E0037001B
:10B07000404281004800DE000040E8004828F80017
:10B08000F0FF9F004828F900404281004800DE00A0
:10B090000040E8004828F800F0FF9F004828F90029
:10B0A000404281004800DE000040E8004828F800E7
:10B0B000F0FF9F004828F900404281004800DE0070
:10B0C0000040E8004828F800F0FF9F004828F900F9
:10B0D000404281004800DE000040E8004828F800B7
:10B0E000F0FF9F004828F900404281004800DE0040
:10B0F0000040E8004828F800F0FF9F004828F900C9
:10B10000404281004800DE000040E8004828F80086
:10B11000F0FF9F004828F900404281004800DE000F
:10B120000040E8004828F800F0FF9F004828F90098
:10B13000404281004800DE000040E8004828F80056
:10B14000F0FF9F004828F900404281004800DE00DF
:10B150000040E8004828F800F0FF9F004828F90068
:10B16000404281004800DE000040E8004828F80026
:10B17000F0FF9F004828F900404281004800DE00AF
:10B180000040E8004828F800F0FF9F004828F90038
:10B19000404281004800DE000040E8004828F800F6
:10B1A000F0FF9F004828F900404281004800DE007F
:10B1B0000040E8004828F800F0FF9F004828F90008
:10B1C0004828F8004F0078004800DE000000060024
:10B1D000504281000160EF005042890050428100DE
:10B1E0000160EF002080B2001B0032001080B2002E
:10B1F000200032007080B200250032001080B200C2
:10B200002A0032003080B2002F0032001080B200DD
:10B2100034003200F080B200390032001080B200F9
:10B220003E0032003080B200430032001080B20095
:10B23000480032007080B2004D0032001080B20031
:10B24000520032003080B20057003200F080B2006D
:10B250005C0032005B003700504281000080FD003E
:10B26000D0C1B3000080FD0050428900F0590400B5
:10B2700000000000504281000080FD00E0C1B300EA
:10B280000080FD0050428900F059040000000000D9
:10B29000504281000080FD00F0C1B3000080FD003D
:10B2A00050428900F0590400000000005042810023
:10B2B0000080FD0000C2B3000080FD005042890004
:10B2C000F059040000000000504281000080FD00A1
:10B2D00010C2B3000080FD0050428900F059040004
:10B2E00000000000504281000080FD0020C2B30039
:10B2F0000080FD0050428900F05904000000000069
:10B30000504281000080FD0030C2B3000080FD008B
:10B3100050428900F05904000000000050428100B2
:10B320000080FD0040C2B3000080FD005042890053
:10B33000F059040000000000504281000080FD0030
:10B3400050C2B3000080FD0050428900F059040053
:10B3500000000000504281000080FD0060C2B30088
:10B360000080FD0050428900F059040000000000F8
:10B37000504281000080FD0070C2B3000080FD00DB
:10B3800050428900F0590400000000005042810042
:10B390000080FD0080C2B3000080FD0050428900A3
:10B3A000F059040000000000504281000080FD00C0
:10B3B00090C2B3000080FD0050428900F0590400A3
:10B3C00000000000504281000080FD00C0C1B300B9
:10B3D0000080FD0050428900F05904000000000088
:10B3E0004A28F8004F0078004800DE000000060000
:10B3F000851F78000400200004428900040020001A
:10B4000014428900F04181000160EF007C04E100FA
:10B4100005003100F0418100C0C1B300F041890056
:10B42000245A040000000000F04181000160EF0098
:10B43000940220000024E10003003100F04181006B
:10B4400090C2B300F0418900F04181004828F80023
:10B45000E0FF9F004828F900F457020000000000B8
:10B460004028F800E0FF9F004028F90000428100DA
:10B470000160EF0000428900004281000000E0000E
:10B480002100320004002000144289001042810093
:10B490006E00E1001C0031000042810061004000AC
:10B4A00000428900004281006E00E1000200360087
:10B4B0001400200004428900044281000960EF006A
:10B4C000E3992000030042001004E00009003A0064
:10B4D000004281004A28F800E0FF9F004A28F90056
:10B4E000E85802000000000008003700845A0400F9
:10B4F00000000000104281000000E80010428900B6
:10B50000465A0400000000000060EF00CF027800FF
:10B51000000006004200F8003600F800801F7800A6
:10B52000200020000C000900B01F7800040020005B
:10B53000D4418900E041810000C0B300E0418900AE
:10B540009A60A9006E28EC007008E2000200320048
:10B55000000037007028ED000A28EC0054408000FD
:10B560006A20E10058003900000037000A28EF0087
:10B5700004002000D4418900D04181007100E10025
:10B580005100310000003700D041810004832000C9
:10B59000040040001004E0004600320000003700C4
:10B5A000D0418100C4802000040040001004E0006D
:10B5B0003800320000003700D041810004832000B1
:10B5C000040040001042780004CEB2000F003A00A0
:10B5D00000003700D0418100C480200004004000FA
:10B5E000904278004428F800E5FF9F004428F900C5
:10B5F000204281000160EF00204289007851020062
:10B60000000000004A5B040000000000D0418100FF
:10B6100004832000040040001042780004CFB200F0
:10B6200011003A0000003700D0418100C4802000A2
:10B6300004004000904278004428F800E5FF9F0095
:10B640004428F900204281000080FD0010C0B300B2
:10B650000080FD00204289007851020000000000B7
:10B660004A5B040000000000D041810004832000F8
:10B67000040040001042780004CDB20005003A00FA
:10B6800000003700D0418100C480200084024000C7
:10B69000804AEB00D0418100C48020008402400039
:10B6A000804AEB00D04181000483200084024000E6
:10B6B000804AEB00D04181000000E800D0418900C1
:10B6C000BC5A0400000000000828EC004440800040
:10B6D000C30320000418E10072003E0000003700A0
:10B6E0000828EF0004002000D4418900D0418100E7
:10B6F0007100E1006B00310000003700D041810093
:10B70000C4802000040040001004E000600032000B
:10B7100000003700D04181006600E10024003200C3
:10B7200000003700D0418100C480200004004000A8
:10B7300090427800D0418100E48120000400400064
:10B74000104378004428F800E5FF9F004428F900E2
:10B750004428F800F6FF9F004428F90078510200C1
:10B7600000000000D0418100E4812000040040007E
:10B770001004E0000700320000003700D0418100D3
:10B78000E481200084024000804AEB00D45B040086
:10B7900000000000D0418100E481200084024000CC
:10B7A00010C0B300804A7800485C0400000000002C
:10B7B0001548E20036003A00000037001248E20067
:10B7C000330032000000370012C8BF004428F800E0
:10B7D000E0FF9F004428F900204281000080FD0026
:10B7E00010C0B3000080FD002042890078510200A3
:10B7F0000000000012C8BF003C28F800E0FF9F00D6
:10B800003C28F900E04181003E28F800E0FF9F005D
:10B810003E28F900F85902000000000012E8B700C5
:10B820001248E2001A00320000003700E0418100B7
:10B830000160EF0012C8B6000004E0000B003A00FF
:10B84000000037002448E20007003A0000003700FB
:10B8500010C0B30024E8B7009A60A80013003700B6
:10B86000365C0400000000002468EF0012C8BF002E
:10B870004428F800E0FF9F004428F900204281009E
:10B880000160EF00204289007851020000000000B2
:10B89000D04181000000E800D0418900765B0400BF
:10B8A000000000008A60A9009A60A8008A60A900D0
:10B8B000A00120000C0009004F1078004F00780014
:10B8C0003600F9004200F900004006000000E000E8
:10B8D0004220AF0004003700793E0900000000005C
:10B8E0000000E900F9FF370000000600A4F3800023
:10B8F0006124E10004003A00D842A900DC42A9001A
:10B90000885C040000000000D842A900DC42A800C6
:10B91000D802A900DC02A800DC22A900D822A900D4
:10B920001E0009000000000075DEBF00C8E2B7007D
:10B930001E00090000000000DC22A800D822A90097
:10B940001E000900000000000000060000CBB3004C
:10B950006DFEB7006E1EA80064F380006924E1004C
:10B960000300360080C0B3006CFEB7006E1EA90055
:10B970006DDEBF006C5EB4006DFEB70010C0B3009A
:10B9800074FEB7006DDEBF0075FEB700765C020086
:10B99000000000000040EB006E1EAF000000E80059
:10B9A00000000600851F78006D7EEF006E7EEF00C0
:10B9B0006F1EA80064F3800033082000041CE1001F
:10B9C0000300310030C8B3006CFEB7006F1EA90041
:10B9D0006CDEBF006DFEB7006CDEBF000160EF00E3
:10B9E0004400DE00704070006EFEB70010C0B3006F
:10B9F00074FEB7006EDEBF0075FEB700765C020015
:10BA000000000000A0002000665C020000000000B2
:10BA10006CDEBF00EF42600010C0B30074FEB700E0
:10BA20000540780075FEB700765C0200000000005B
:10BA3000A0002000665C0200000000000040EB0057
:10BA40006F1EAF000000E800CF0278000000060083
:10BA5000337CEF00347CEF0094E180006824E10047
:10BA60000400360080C0B30033FCB7003E5D040024
:10BA70000000000032DCBF0033FCB70032DCBF0046
:10BA80006CFEB700A65C0200000000006C7EEF00B8
:10BA9000D25C020000000000347CEF00A4E18000D2
:10BAA00043082000041CE10007003600747EEF000C
:10BAB000757EEF00765C020000000000347CEC0034
:10BAC0004E5D04000000000010C0B30000E0B700AD
:10BAD00000000600007CEF00007CEF0004E0800026
:10BAE0006924E1000700310000DCBF0032FCB70030
:10BAF000285D020000000000007CEC006E5D040088
:10BB00000000000000000600FE3BEF0010C0B30084
:10BB100074FEB700E0CAB30075FEB700765C0200A1
:10BB200000000000D862A900DC62A9003E01090003
:10BB300000000000D862A900DC62A800803E20005E
:10BB4000665C020000000000C602F800FE1BF9005F
:10BB500000F02F00FE3BB600FE1BF800C602F90005
:10BB60001E0009000000000010C0B30074FEB70002
:10BB700080C2B30075FEB700765C020000000000D2
:10BB800010C0B30074FEB70020CEB30075FEB7003E
:10BB9000765C02000000000010C0B30074FEB70025
:10BBA00000C1B30075FEB700765C02000000000023
:10BBB00010C0B30074FEB700757EEF00765C020023
:10BBC0000000000010C0B30074FEB70000CBB3004B
:10BBD00075FEB700765C02000000000010C0B300E4
:10BBE00074FEB70000C4B30075FEB700765C0200B7
:10BBF0000000000010C0B30074FEB70010CAB3000C
:10BC000075FEB700765C02000000000010C0B300B3
:10BC100074FEB70000CCB30075FEB700765C02007E
:10BC20000000000010C0B30074FEB700F0CAB300FB
:10BC300075FEB700765C02000000000040062000A0
:10BC4000665C02000000000010C0B30074FEB70084
:10BC500070CEB30075FEB700765C020000000000F5
:10BC60006A5D02000000000020032000665C020004
:10BC70000000000000000600851F78006F7EEF00C6
:10BC8000707EEF0074F3800003022000041CE100CA
:10BC900020003E0074F38000F3032000041CE10048
:10BCA0001C00390074F380000442B10004407800A5
:10BCB0006FFEB700707EEF0084F380006524E10022
:10BCC0001200310074F380004822DE006520B800C5
:10BCD0008002780084F380000960EF000480420055
:10BCE000C42621000400400090427800747EEF00DA
:10BCF0000540780075FEB700765C02000000000089
:10BD0000707EEC005C5E040000000000485F0400F0
:10BD10000000000074F3800003042000041CE10014
:10BD200020003E0074F38000F3052000041CE100B5
:10BD30001C00390074F380000444B1000440780012
:10BD40006FFEB700707EEF0084F380006524E10091
:10BD50001200310074F380004822DE006520B80034
:10BD60008002780084F380000960EF0004804200C4
:10BD7000C43021000400400090427800747EEF003F
:10BD80000540780075FEB700765C020000000000F8
:10BD9000707EEC00A45E040000000000485F040018
:10BDA0000000000074F3800003062000041CE10082
:10BDB00020003E0074F38000F3072000041CE10023
:10BDC0001C00390074F380000446B1000440780080
:10BDD0006FFEB700707EEF0084F380006524E10001
:10BDE0001200310074F380004822DE006520B800A4
:10BDF0008002780084F380000960EF000480420034
:10BE0000C43A21000400400090427800747EEF00A4
:10BE10000540780075FEB700765C02000000000067
:10BE2000707EEC00EC5E040000000000485F04003F
:10BE3000000000006F7EEF00707EEF0084F3800052
:10BE40006524E1001200310074F380004822DE0016
:10BE50006520B8008002780084F380000960EF005C
:10BE600004804200C4262100040040009042780073
:10BE7000747EEF000540780075FEB700765C020026
:10BE800000000000707EEC001E5F04000000000057
:10BE900010C0B30000E0B700CF0278000000060039
:10BEA000851F7800657EEF0060DEBF006CFEB70086
:10BEB000A65C02000000000061DEBF006CFEB7005F
:10BEC000D25C020000000000657EEF0065DEBF006E
:10BED00024F380000024E1001500340024F38000E6
:10BEE0004822DE0004007800621EB4009042780010
:10BEF0006E1EF800E5FF9F006E1EF9003C5E02001A
:10BF000000000000747EEF00757EEF00765C02009A
:10BF100000000000747EEF00757EEF00765C02008A
:10BF200000000000657EEC00665F04000000000079
:10BF3000CF02780000000600851F7800C5002000B1
:10BF400003000900B51F7800000278008102780024
:10BF500002037800830378000000EB008000EB0010
:10BF60000001EB008001EB000800A10007F0A60033
:10BF7000050037000800A0000402EA008582EA00FC
:10BF80000683EA008783EA008504720002003A0013
:10BF90008704730015003200394720000340A700D2
:10BFA0000B0037004200A9000482D2008582D20033
:10BFB0000683D2008783D2000080D2008180D20025
:10BFC0000281D2008381D2008904E900F3FF3A00A4
:10BFD000C44CDD004200A90009F0A1000340A1000B
:10BFE00083816C000800A70003F0A0002501200059
:10BFF00003000900CF127800CF027800000006008D
:10C00000881F78002801200004000900B81F78006C
:10C010008005EB006066B8000304780087047800B0
:10C02000FA7F20004200A9004220A90044C4DE009B
:10C03000080465000800E000700032004200A9001A
:10C040004220A900C4CCDE00890465000900E0009C
:10C050006A0032000884440009B0A70004003700D9
:10C06000F83FB1006500320064003900030037007A
:10C070001A40200085424500600031008786690033
:10C080004200A9004220A900F300B2000340A00032
:10C09000F700B2000740A000881F78000124B80014
:10C0A000002DB8000A0544008B854C000C80B000C0
:10C0B0000224B8008B0544000C864C00012CB8000B
:10C0C0008B0544000C864C000034B8000005EB00E2
:10C0D0008B0544000C864C000A80B0008005EB0004
:10C0E0000324B8000C0644000A854C000B80B00005
:10C0F000022CB8000C0644000A854C000B80B000EE
:10C100000134B8000C0644000A854C000B80B000D6
:10C11000003CB8000C0644000A854C000B80B000BF
:10C120000C0078000006EB00032CB8000A05440060
:10C130008B854C000C80B0000234B8000A05440026
:10C140008B854C000C80B0000334B8008B05440094
:10C150000C864C00013CB8000A0544008B854C005D
:10C160000C80B000023CB8008B0544000C864C00EB
:10C17000033CB8000C0644008A0078000B017800EC
:10C180008C017800540020004200A9008381D30074
:10C190000281D3008180D3000080D3000402E90033
:10C1A000F9FF3A004F0478000804E800010370002A
:10C1B0000100320002003700030371000800320062
:10C1C0000340A700060037004200A9000080D2000B
:10C1D0008180D2000281D2008381D2000804E9006C
:10C1E0004444DD0003F0A1000DF0A70003F0A0001F
:10C1F0000340A10083016C00030037006000B80019
:10C200006001B80000003700A80120000400090008
:10C210004F1478004F04780000000600881F780053
:10C220002801200004000900B81F780087866900F3
:10C230000304780087047800FA7F20004200A900F8
:10C240004220A90044C4DE00080465000800E000A4
:10C250006C0032004200A9004220A900C4CCDE00DC
:10C26000890465000900E000660032000005EB006B
:10C270000906540003003900FC3FB00061003100A2
:10C28000040037001B4020000B0656005D003900FB
:10C290005C0032000004EB008004EB000005EB00C2
:10C2A0008005EB00F301B2000340A000F701B200EB
:10C2B0000740A0008C1F78006C0320000400500091
:10C2C000858058000601590087815900020033001B
:10C2D0000600310006003A00040040008580480056
:10C2E0000601490087814900010037000800A000CD
:10C2F0000C06E9000B0032004200A9000080D200C9
:10C300008180D2000281D2008381D2004200A90044
:10C310000884D2008984D2000A85D2008B85D2009D
:10C32000E6FF37004F0678000B50A70001003700EA
:10C33000060037004200A9008B85D3000A85D30090
:10C340008984D3000884D300030037000C06E90079
:10C350004200A9002B0032004200AF000900370064
:10C360000080D2008180D2000281D2008381D2007D
:10C370000402500085825800060359008783590043
:10C38000150039000804E80013003A008904E800A9
:10C3900011003A000A05E8000F003A008B05E8009A
:10C3A0000D003A000C06E800160032000A003700C3
:10C3B0000C06E900130032000B40A700060037000E
:10C3C0004200A9000884D2008984D2000A85D200E4
:10C3D0008B85D200F8FF37004466DD004200A900DB
:10C3E0000CF0A1000DF0A7000CF0A0000B40A10084
:10C3F0008B016E000A01780089007800080078003F
:10C40000050037000000200001002000020020008D
:10C410000300200000003700A801200004000900EC
:10C420004F1478004F04780000000600851F780044
:10C43000861F780003027800030378004200A900F9
:10C4400044A2DE00F57F20000482620003003A006F
:10C450006000B8000001EB00130037000438B100A1
:10C46000F300B200370020004200A9000080D20093
:10C470008180D2000281D2008381D2008703E9004B
:10C48000F9FF3A0001007800820078000370A100F3
:10C490000480FD004200A9000482D30006F0A7003A
:10C4A00004F0A00003016A004F037800CF02780077
:10C4B00000000600811F7800A1DD80008058780010
:10C4C0008048EB00CF007800B43BEC000000060091
:10C4D000851F780082017800820278004200A9005E
:10C4E0008381D2000380FD00F30FB20003003A0005
:10C4F0006000B8006011B800160037000338B000C3
:10C50000F207B200360020000002EB004200A90052
:10C510000281D3008180D3000080D3004200AF00AD
:10C520000402E8000603E900F8FF3A000270A100E7
:10C53000C419DD0003F0A10005F0A70003F0A0007E
:10C5400083016900010178008000780081004200C9
:10C550000000EB00CF02780000000600851F780085
:10C56000C500200005000900B51F7800030478000D
:10C570008203780001037800800278008304780049
:10C580003B472000C499DE00FA7F2000830165004C
:10C5900083855500F801B2000840A0000000EB00C0
:10C5A0008000EB000001EB008001EB004200A900DD
:10C5B0000884D3008783D3000683D3008582D30009
:10C5C0008381D3000281D3008180D3000080D30017
:10C5D0008B05E900F5FF3A0009F0A60005003700D9
:10C5E0000000EA008180EA000281EA008381EA001B
:10C5F000000037006501200005000900CF12780017
:10C60000CF027800000006008C1F78008D1F780094
:10C610000004EB008004EB000005EB008005EB005C
:10C620000006EB008006EB00E80020000900200077
:10C630001000FA000C377C000884E900FDFF3B0085
:10C6400005046A0002003A0007046B002F00320064
:10C650000004EB000D0420000D0420004200A9009E
:10C660000080D2008180D2000281D2008381D2007A
:10C670000884D2008984D2000A85D2008B85D2003A
:10C680000758E10005003A0006D0E10003003A0037
:10C6900005C8E10001003A0004C0E10005003900CE
:10C6A0000404540085845C0006055D0087855D00F8
:10C6B0004200A800080F7800190798002A07980080
:10C6C0003B0798004E049000DE0490006E05900039
:10C6D000FE0590000884D2008984D2000A85D20029
:10C6E0008B85D20048079800590798006A07980080
:10C6F0007B0798001E0478009E0490002E05900091
:10C70000BE0590008D06E900D4FF3A004E0090006F
:10C71000DE0090006E019000FE0190000080FA00A3
:10C7200000003700CF0678004F06780000000600B2
:10C73000851F7800C500200007000900B51F78009C
:10C740002A00FA00880220000006EB000C377C006B
:10C750000884E900FDFF3B000900E0000E00320004
:10C76000391798004A179800470224000003EB008D
:10C770006022B80029179800470224000003EB004C
:10C780006022B8000060020000000000AE149000BB
:10C790008904E900F7FF3A00BE1490004001200030
:10C7A00020179800D71C240056D62C006022B80011
:10C7B000000F9800110F9800220F9800330F980077
:10C7C000480120000817980004002000859E2800DA
:10C7D0004630220077AC2800440F9800550F98008F
:10C7E000660F9800770F980003F0A600040037004A
:10C7F0004E1490000804E90008D0A00048179800E3
:10C8000003F0A100AE620200000000004E14900090
:10C81000BE1490000900E0004220AF000844E80088
:10C82000481798009E1490008004EB001917980098
:10C830004E0A9000DE0A90006E0B9000FE0B9000F6
:10C8400004630200000000009E1690000D00A70087
:10C8500060003700080F9800190F98002A0F980001
:10C860003B0F98009E1690000D00A2001D17980027
:10C870000000E00012003A00BE1490008904E800B5
:10C880002E159000090455000D003200CE159000C1
:10C890000B00E0000E0032007F84650008045500A4
:10C8A000010032003F0031000BF0A7003D003700CF
:10C8B0000BE0A7000600370000022000340037001C
:10C8C000CE1590000C0022008B0566004B179800D7
:10C8D000CE1590000BD0A6000E0037000BD0A100A3
:10C8E000BE1490000900E0004220AE008B05E90074
:10C8F0008005EB004B17980000057800D0C2B3000C
:10C900005A620200000000000A0078008005EB0077
:10C910004B179800BE1490002E1590000904550086
:10C920000B003A008005EB004B17980000057800DB
:10C93000E0C2B3005A62020000000000CE15900071
:10C940000C0022008B0566004B1798000A00780047
:10C9500001032000CE1590000BD0A6000C0037007C
:10C960000BD0A100BE1490000900E0004220AE00F0
:10C970008B05E9008005EB004B179800D0C2B3008F
:10C980005A620200000000000000EB0001032000DA
:10C9900000804000801F78004F0078005A6202003B
:10C9A00000000000AE1690008D06E900190032006C
:10C9B0002D1798004E089000DE0890006E09900038
:10C9C000FE099000A40020008002EB006033B80054
:10C9D0009BFF3700400F9800510F9800620F98009E
:10C9E000730F98000002780081027800020378003B
:10C9F000830378000E0890009E0890002E09900096
:10CA0000BE0990009E1690000D00A2001D17980010
:10CA10008BFF37000080FA00A50120000700090005
:10CA2000CF127800CF02780000000600F0FF2F0040
:10CA30000862AE000500370009C2AF00FEFF3700F4
:10CA40001110880009C2AF00FEFF3700000020006F
:10CA500009E2AF000000E800000006000862AE0036
:10CA6000040037000622A8000622AF00FEFF3700B0
:10CA7000030037000602A8000602AF00FEFF3700E1
:10CA80009E0009000000000091EC80001665020085
:10CA9000000000009E0009000000000093DDBF00C0
:10CAA0008000780016650200000000009E0009006A
:10CAB00000000000A1EC80001665020000000000EC
:10CAC0009E00090000000000F00120000602B600F0
:10CAD000FDFF3A000642A8000642AF00FEFF370005
:10CAE000BE0009000000000000000600F0FF2F005B
:10CAF0000862AE0011003700321080007F01610033
:10CB0000FDFF3A000662A8000100A70006A2A900E6
:10CB10000100A60006A2A800321080007F0161007B
:10CB2000FDFF3A000682A8000822AE00FEFF370093
:10CB30000010800008C2AF0008C2A9000000060073
:10CB4000851F7800947DEF000862AE000400370076
:10CB50000622A8000622AF00FEFF370003003700C0
:10CB60000602A8000602AF00FEFF3700BE00090063
:10CB70000000000091EC800016650200000000003B
:10CB8000BE0009000000000093DDBF0080007800B7
:10CB90001665020000000000BE0009000000000051
:10CBA0000862AE00040037000622A8000622AF008B
:10CBB000FEFF3700030037000602A8000602AF00A0
:10CBC000FEFF3700BE0009000000000092DDBF003C
:10CBD000E142700085407800166502000000000008
:10CBE000BE0009000000000001002000811F780045
:10CBF000CF007800766502000000000094FDB700C9
:10CC0000BE00090000000000F00120000602B6008E
:10CC1000FDFF3A000642A8000642AF00FEFF3700C3
:10CC2000DE0009000000000094DDBF0000E0B70056
:10CC3000CF02780000000600FE7BEF0040C4B30086
:10CC400092FDB70080C1B30093FDB70094FDEF00E3
:10CC50002E6502000000000040C4B30092FDB70042
:10CC600090C1B30093FDB70094FDEF002E65020064
:10CC70000000000040C4B30092FDB700A0C1B300A3
:10CC800093FDB70094FDEF002E6502000000000048
:10CC900040C4B30092FDB700B0C1B30093FDB7002C
:10CCA00094FDEF002E6502000000000040C4B300B8
:10CCB00092FDB700C0C1B30093FDB70094FDEF0033
:10CCC0002E6502000000000040C4B30092FDB700D2
:10CCD00000C2B30093FDB700947DEF002E65020003
:10CCE0000000000040C4B30092FDB70010C2B300C2
:10CCF00093FDB700947DEF002E6502000000000058
:10CD000040C4B30092FDB70020C2B30093FDB7004A
:10CD1000947DEF002E6502000000000040C4B300C7
:10CD200092FDB70030C2B30093FDB700947DEF00D1
:10CD30002E6502000000000040C4B30092FDB70061
:10CD400040C2B30093FDB700947DEF002E65020052
:10CD50000000000040C4B30092FDB700937DEF00D7
:10CD6000A065020000000000FEFBB70040C4B30055
:10CD700092FDB70010C0B30093FDB700A06502009C
:10CD800000000000FEFBB70040C4B30092FDB700F6
:10CD900020C0B30093FDB700A065020000000000B2
:10CDA000FEFBB70040C4B30092FDB70030C0B30033
:10CDB00093FDB700A065020000000000FEFBB70075
:10CDC00040C4B30092FDB70040C0B30093FDB7006C
:10CDD000A065020000000000FEFBB7004200F80062
:10CDE00042E0EF006042810080C1B30060428900F0
:10CDF000604281000160EF0060428900185102002A
:10CE0000000000004200F9004200F80042E0EF009C
:10CE10006042810090C1B30060428900604281009D
:10CE20000160EF006042890018510200000000001C
:10CE30004200F9004200F80042E0EF006042810049
:10CE4000A0C1B30060428900604281000160EF0030
:10CE50006042890018510200000000004200F90001
:10CE60004200F80042E0EF0060428100B0C1B30030
:10CE700060428900604281000160EF0060428900E9
:10CE800018510200000000004200F9004200F800C2
:10CE900042E0EF0060428100C0C1B30060428900FF
:10CEA000604281000160EF00604289001851020079
:10CEB000000000004200F9004200F80042E0EF00EC
:10CEC0006042810000C2B30060428900604281007C
:10CED00001E0EF00604289001851020000000000EC
:10CEE0004200F9004200F80042E0EF006042810099
:10CEF00010C2B300604289006042810001E0EF008F
:10CF00006042890018510200000000004200F90050
:10CF10004200F80042E0EF006042810020C2B3000E
:10CF2000604289006042810001E0EF0060428900B8
:10CF300018510200000000004200F9004200F80011
:10CF400042E0EF006042810030C2B30060428900DD
:10CF50006042810001E0EF00604289001851020048
:10CF6000000000004200F9004200F80042E0EF003B
:10CF70006042810040C2B30060428900604281008B
:10CF800001E0EF006042890018510200000000003B
:10CF90004200F900F40F2000148A88004200F800D3
:10CFA00042E0EF006042810080C0B300604289002F
:10CFB00042D1BF004C28F800F0FF9F004C28F90038
:10CFC00018510200000000004200F900F40F200098
:10CFD000248A88004200F80042E0EF0060428100AD
:10CFE00090C0B3006042890044D1BF004C28F800D3
:10CFF000F0FF9F004C28F9001851020000000000CB
:10D000004200F900F40F2000348A88004200F80042
:10D0100042E0EF0060428100A0C0B300604289009E
:10D0200046D1BF004C28F800F0FF9F004C28F900C3
:10D0300018510200000000004200F900F40F200027
:10D04000448A88004200F80042E0EF00604281001C
:10D05000B0C0B3006042890048D1BF004C28F8003E
:10D06000F0FF9F004C28F90018510200000000005A
:10D070004200F900F40F2000548A88004200F800B2
:10D0800042E0EF0060428100C0C0B300604289000E
:10D090004AD1BF004C28F800F0FF9F004C28F9004F
:10D0A00018510200000000004200F90000C4B30063
:10D0B00092FDB70040C0B30093FDB700947DEF0030
:10D0C0002E6502000000000000C4B30092FDB7000E
:10D0D00050C0B30093FDB700947DEF002E650200B1
:10D0E0000000000000C4B30092FDB70060C0B300B0
:10D0F00093FDB700947DEF002E6502000000000054
:10D1000000C4B30092FDB70070C0B30093FDB70038
:10D11000947DEF002E6502000000000000C4B30003
:10D1200092FDB70020C0B30093FDB70094FDEF005F
:10D130002E6502000000000000C4B30092FDB7009D
:10D1400030C0B30093FDB70094FDEF002E650200E0
:10D150000000000000000600851F78003A3CEF0048
:10D16000C0C0B30047E9B70040C0B30048E9B7000A
:10D170004969EF004A69EF0010C0B3004EE9B700FB
:10D1800010C0B3004FE9B70020C1B30051E9B700A8
:10D19000F0C0B30050E9B70040C0B30052E9B70097
:10D1A00040C0B30053E9B70040C0B30054E9B70032
:10D1B00090C1B30055E9B700E0C1B30071E9B70011
:10D1C000E0C1B30072E9B700E0C1B30073E9B70092
:10D1D0005669EF005769EF005869EF0080C1B3004E
:10D1E00059E9B70080C1B3005AE9B70080C1B30064
:10D1F0005BE9B70080C1B3005CE9B70080C1B30050
:10D200005DE9B70080C1B3005EE9B70080C1B3003B
:10D210005FE9B70080C1B30060E9B70040C1B30067
:10D2200061E9B70040C1B30062E9B70040C1B30093
:10D2300063E9B70040C1B30064E9B70040C1B3007F
:10D2400065E9B70040C1B30066E9B70040C1B3006B
:10D2500067E9B70040C1B30068E9B70070C0B30028
:10D2600069E9B70070C0B3006AE9B70070C0B300E5
:10D270006BE9B70070C0B3006CE9B70070C0B300D1
:10D280006DE9B70070C0B3006EE9B70070C0B300BD
:10D290006FE9B70070C0B30070E9B7007469EF00C0
:10D2A0007569EF007669EF007769EF007869EF0044
:10D2B0007969EF007A69EF007B69EF00A0C0B300E5
:10D2C00092E8B7003A3CEF00D4E180006F20E10023
:10D2D00007003100E4992000D3E1800084824100FE
:10D2E000804AEB003A3CEC00646904000000000056
:10D2F000CF02780000000600851F7800397EEF001D
:10D300000862AE00040037000622A8000622AF0023
:10D31000FEFF3700030037000602A8000602AF0038
:10D32000FEFF3700BE0009000000000001CAB30084
:10D330001665020000000000BE00090000000000A9
:10D340003BDEBF0080027800854078001665020051
:10D3500000000000D5F180008540780016650200CD
:10D3600000000000BE000900000000000862AE00DE
:10D37000040037000622A8000622AF00FEFF370097
:10D38000030037000602A8000602AF00FEFF3700C8
:10D3900011CAB3001665020000000000BE000900BB
:10D3A0000000000001002000811F7800CF007800FD
:10D3B000766502000000000039FEB700F001200091
:10D3C0000602B600FDFF3A000642A8000642AF0082
:10D3D000FEFF3700DE0009000000000039DEBF005C
:10D3E000CF02780000000600851F78001A5CE2007A
:10D3F00021003200B0E0800090427800C0E0800060
:10D400000002780014407800002CE1000E00320089
:10D41000B0E0800090427800C0E080000002780018
:10D4200014407800002CE1000300310000C0EB0044
:10D430001E6A04000000000010C0B3000F00370097
:10D440002E6A040000000000B0E080001004E0003C
:10D4500002003A000060EF0008003700B0E08000F2
:10D46000163CEC00C0E08000183CEC001A7CED009B
:10D47000F6690400000000000060EF00CF027800B1
:10D4800000000600851F7800FE3BEF00007CEF00E7
:10D49000017CEF000402220014E088000402220054
:10D4A00024E088000402220034E088000402220004
:10D4B00044E088000402220054E0880004022200B4
:10D4C00064E088000402220074E088000402220064
:10D4D00084E088000402220094E08800147CEF00BD
:10D4E000F4FC2100F4DF8800007CEF0004E0800001
:10D4F0007224E1001600310000CAB30038FEB70004
:10D50000FE1BF8003A1EF9007C69020000000000D2
:10D5100001FCB70050002000665C02000000000023
:10D5200004E080000960EF0023C021008302420074
:10D5300001DCBF00804A7800F4DF80006102420015
:10D54000F4DF8800007CEC00766A04000000000034
:10D55000147CEF0020C1B3001AFCB70024C02100E6
:10D56000B4E0880064852000C4E08800F46902000B
:10D57000000000000004E00005003A0010C0B30005
:10D5800000E0B70004003700CC6A0400000000008F
:10D5900000E0EF0000003700CF0278000000060036
:10D5A000851F7800601EF800661EF900645EE200C8
:10D5B0000C00320010F380001004E000090032007B
:10D5C00030F38000663EEC008002780010F38000AB
:10D5D000623EEC00904A7800647EED00D66A04005A
:10D5E00000000000645EE2000700320030F38000BB
:10D5F000663EEC0080027800804AEB00647EED001D
:10D60000F26A040000000000601EF8000000F9004B
:10D61000CF02780000000600C1E4210002002000D3
:10D62000120009008058EB0020C1B30064FEB7006F
:10D63000C4E4210004F388004A1EF800621EF900C9
:10D64000D06A02000000000070C0B30060FEB700A6
:10D65000617EEF0020C1B30064FEB700C4E4210086
:10D6600014F38800505F0200000000000000060074
:10D67000851F78000862AE00040037000622A8006B
:10D680000622AF00FEFF3700030037000602A800A5
:10D690000602AF00FEFF3700BE00090000000000D8
:10D6A00001CAB3001665020000000000BE000900B8
:10D6B000000000003DDEBF00800278008540780059
:10D6C0001665020000000000E5F18000854078004A
:10D6D00016650200000000009E0009000000000026
:10D6E0003BDEBF00800078001665020000000000ED
:10D6F0009E00090000000000F00120000602B600B4
:10D70000FDFF3A000642A8000642AF00FEFF3700C8
:10D71000BE00090000000000CF02780000000600F3
:10D720003C3EEF003B7EEF003C3EEF00E0F180002E
:10D73000D4F180000960EF000020E1000B0036000A
:10D74000E0F18000381EB400000278001440780038
:10D750003B7EB40050002000665C02000000000028
:10D760003C3EEC00966B040000000000D4F1800009
:10D770004822DE00F4CFB200044078003BFEB70040
:10D78000D4F180004822DE0061424200044078006B
:10D790003BFEB7003BDEBF0000000600851F78009F
:10D7A0001C3EEF001B7EEF00327EEF00331EA9000F
:10D7B0001C3EEF00E0F08000D4F080000960EF0034
:10D7C0000020E1002200360000CAB30038FEB70096
:10D7D0001C1EF8003A1EF9007C69020000000000DF
:10D7E00032FEB700E0F08000181EB400000278009E
:10D7F00014407800325EE30012003200A0002000E6
:10D80000665C020000000000E0F08000181EB4001A
:10D810009042780000CAB3003AFEB7000540780095
:10D820003BFEB7001C1EF8003C1EF900386B0200DE
:10D8300000000000A0002000665C02000000000064
:10D84000331EA8001C3EEC00DA6B04000000000050
:10D85000331EAE003E00370002002000E1E121004F
:10D86000020078007A020200000000008058780070
:10D870000201E8000004E0004220AE00F8FF37009B
:10D88000E4E1210054F288000C6B0200000000006B
:10D890004809AE000D0037000100200001007800AB
:10D8A0009A020200000000008100E800811F780059
:10D8B0002322AF00FEFF370020118800CF00780040
:10D8C000D00020000008E600F4FF37001ADEBF0099
:10D8D0003AFEB700181EF800381EF900906B0200DF
:10D8E000000000001BFEB70000CAB30038FEB700FE
:10D8F0001ADEBF003AFEB7003B7EEF007C690200F3
:10D900000000000032FEB70032DEBF001B5EE30005
:10D910000F003200A0002000665C02000000000042
:10D9200000CAB3003AFEB7001ADEBF003CFEB700E3
:10D930003D7EEF001BDEBF003BFEB700386B0200F0
:10D9400000000000A0002000665C02000000000053
:10D95000CF02780000000600851F7800861F78003F
:10D960000001EB000103780064C110004211DD00EA
:10D970000200DD00800278000C60EC000C60ED001D
:10D980000D00320005007800C42ADD004C00DE00E6
:10D99000F000B2000003B000A20320000200E1008A
:10D9A000010039000D40B4002322AF00FEFF370014
:10D9B00020118800F1FF37004F037800CF02780074
:10D9C00000000600851F78001C3EEF001E3EEF00A1
:10D9D0001B7EEF00207EEF00217EEF00227EEF0015
:10D9E000231EA90000CAB30038FEB70014002000AF
:10D9F000D4F188007C6902000000000022FEB7001C
:10DA000004F180004822DE00F4CFB20002003200B0
:10DA1000215EE20002003A00D0C0B30022FEB7004F
:10DA20001E3EEF00F4F080006220E100A50031000E
:10DA30001C3EEF00E0F08000D4F080000960EF00B1
:10DA40000020E1005C003600E0F08000181EB40009
:10DA50008002780000CAB30038FEB7001C1EF80030
:10DA60003A1EF9007C69020000000000804A78003C
:10DA7000221EAE004A00370000CAB30038FEB700CD
:10DA80001C1EF8003A1EF9007C690200000000002C
:10DA900021FEB700E0F08000181EB40010407800AE
:10DAA000215EE3003E003200231EAF000E0037006F
:10DAB000231EA800010020000100780000020200DF
:10DAC000000000008100E800811F78002322AF00E1
:10DAD000FEFF370020118800CF007800D001200021
:10DAE0000008E600F4FF3700E0F08000181EB400E4
:10DAF00090427800E0F0800041702000AC6C0200A1
:10DB0000000000002322AF00FEFF3700A403200026
:10DB1000241188002322AF00FEFF370004022000FA
:10DB200024118800054078000160EF002170220078
:10DB3000AC6C0200000000008100200001007800B1
:10DB40002C020200000000008100E800811F780024
:10DB50002322AF00FEFF370020118800CF0078009D
:10DB6000B00020000008E600F4FF370021DEBF000F
:10DB70000160EF0021702200AC6C02000000000088
:10DB80002322AF00FEFF3700A400200024118800EC
:10DB90002322AF00FEFF3700D400200024118800AC
:10DBA00050002000665C0200000000001C3EEC00FB
:10DBB0001A6D04000000000000CAB30038FEB70070
:10DBC0001ADEBF003AFEB7003B7EEF007C69020020
:10DBD0000000000020FEB7001ADEBF003AFEB700CA
:10DBE000181EF800381EF900906B020000000000BB
:10DBF0001BFEB70020DEBF001B5EE3002E003200DC
:10DC000001002000010078004A020200000000002C
:10DC10008100E800811F78002322AF00FEFF37005B
:10DC200020118800CF007800D00020000008E60016
:10DC3000F4FF370020DEBF000160EF0021702200FA
:10DC4000AC6C02000000000011012000010078000F
:10DC50004A020200000000008100E800811F7800F5
:10DC60002322AF00FEFF370020118800CF0078008C
:10DC7000D00120000008E600F4FF37001BDEBF00E3
:10DC80000160EF0021702200AC6C02000000000077
:10DC90002322AF00FEFF3700A400200024118800DB
:10DCA0002322AF00FEFF3700D4002000241188009B
:10DCB0000060EF00050037001E3EEC00126D04000E
:10DCC0000000000010C0B30000E0B700CF027800F1
:10DCD00000000600851F78004E3CEF00507CEF00EE
:10DCE000517CEF00527CEF000404200074E28800B5
:10DCF000507CEF0084E280006724E1001E003100C8
:10DD0000517CEF0084E280004822DE006E24E100B6
:10DD100016003100527CEF0094E280007724E1008D
:10DD20000F00310070E280004E3CEC008002780071
:10DD300000CAB3003AFEB7003B7EEF00E5F1880071
:10DD4000386B02000000000050002000665C0200FA
:10DD500000000000527CEC008C6E0400000000000B
:10DD6000517CEC00826E040000000000507CEC004E
:10DD70007A6E040000000000507CEF0084E2800016
:10DD80006F24E1000800310084E280000960EF00A8
:10DD9000E399200083024200804AEB00507CEC00B3
:10DDA000BE6E040000000000CF02780000000600F4
:10DDB000851F78004E3CEF00507CEF00517CEF0057
:10DDC000E490200074E28800507CEF0084E2800040
:10DDD0006E24E10015003100517CEF0084E28000E8
:10DDE0004822DE0003022000041CE1000C00360083
:10DDF00070E280004E3CEC008002780000CAB30064
:10DE00003AFEB7003B7EEF00E5F18800386B020078
:10DE100000000000517CEC00EE6E040000000000E9
:10DE2000507CEC00E66E040000000000CF02780099
:10DE300000000600851F7800023CEF00043CEF0064
:10DE4000427CEF00437CEF002453230024E288004F
:10DE5000D4D2240034E288001496270044E28800DB
:10DE6000D412230054E288000403200064E28800F6
:10DE7000C0C0B30006FCB70040C0B30007FCB70049
:10DE8000087CEF00097CEF0040C1B3000AFCB7003A
:10DE900010C0B3000BFCB70010C0B3000CFCB700FF
:10DEA00020C1B3000DFCB700F0C0B3000EFCB700FA
:10DEB00040C0B3000FFCB70040C0B30010FCB70077
:10DEC00040C0B30011FCB70090C1B30012FCB70012
:10DED000E0C1B30013FCB700E0C1B30014FCB7000D
:10DEE000E0C1B30015FCB700167CEF00177CEF0013
:10DEF000187CEF0080C1B30019FCB70080C1B300EB
:10DF00001AFCB70080C1B3001BFCB70080C1B3008E
:10DF10001CFCB70080C1B3001DFCB70080C1B3007A
:10DF20001EFCB70080C1B3001FFCB70080C1B30066
:10DF300020FCB70040C1B30021FCB70040C1B300D2
:10DF400022FCB70040C1B30023FCB70040C1B300BE
:10DF500024FCB70040C1B30025FCB70040C1B300AA
:10DF600026FCB70040C1B30027FCB70040C1B30096
:10DF700028FCB70070C0B30029FCB70070C0B30024
:10DF80002AFCB70070C0B3002BFCB70070C0B30010
:10DF90002CFCB70070C0B3002DFCB70070C0B300FC
:10DFA0002EFCB70070C0B3002FFCB70070C0B300E8
:10DFB00030FCB700317CEF00327CEF00337CEF00A7
:10DFC000347CEF00357CEF00367CEF00377CEF00CF
:10DFD000387CEF00A0C0B30039FCB7003A7CEF00FA
:10DFE0003B7CEF003C7CEF003D7CEF003E7CEF0093
:10DFF0003F7CEF00407CEF00417CEF00C0C3B300EA
:10E000001AFEB70064C02100C4F08800CE6B020085
:10E0100000000000C0C3B3001AFEB70064C02100B6
:10E02000C4F08800E26C0200000000006104E1001E
:10E030001B003200C0C3B3001AFEB70064C0210049
:10E04000C4F08800CE6B020000000000C0C3B30023
:10E050001AFEB70064C02100C4F08800E26C020020
:10E06000000000006104E1000D003200010020000A
:10E0700001007800B6020200000000008100E80004
:10E08000811F78002322AF00FEFF37002011880097
:10E09000CF007800D00120000008E600F4FF370030
:10E0A0006A6E020000000000D86E0200000000004E
:10E0B000F4FC210014E08800427CEF0014E28000B0
:10E0C0007324E1001B00310014E280000960EF00BE
:10E0D00063852000030042001040780043FCB70035
:10E0E00000CAB3003AFEB70043DCBF003BFEB700F6
:10E0F000021CF8003C1EF900386B02000000000012
:10E1000000CAB30038FEB700021CF8003A1EF9003E
:10E110007C6902000000000043FCB70014E08000AE
:10E120006102420014E08800427CEC005E70040052
:10E130000000000014FE210014E08800043CEF0001
:10E14000427CEF0014E280007324E10037003100CC
:10E1500014E280000960EF002384200003004200E5
:10E1600090427800040320000524E10004003E00F2
:10E17000940320000524E10001003900030037006A
:10E180000040EB00C87004000000000010C0B300A5
:10E190006104E10022003A0024E080006520E100F3
:10E1A0001F003E0014E280000960EF00238420007D
:10E1B000030042001040780043FCB70000CAB300DF
:10E1C0003AFEB70043DCBF003BFEB700021CF8007C
:10E1D0003C1EF900386B02000000000050002000D7
:10E1E000665C02000000000000CAB30038FEB70001
:10E1F000021CF8003A1EF9007C69020000000000D1
:10E2000043FCB70050002000665C020000000000E4
:10E21000043CEC0014E080006102420014E088003D
:10E22000427CEC00A27004000000000074FE21009B
:10E2300014E08800427CEF0014E280006924E100D1
:10E240001B00310014E280000960EF0043C421008C
:10E25000030042001040780043FCB70000CAB3003E
:10E260003AFEB70043DCBF003BFEB700021CF800DB
:10E270003C1EF900386B02000000000000CAB30029
:10E2800038FEB700021CF8003A1EF9007C69020053
:10E290000000000043FCB70014E08000610242006F
:10E2A00014E08800427CEC001C71040000000000B7
:10E2B000CF02780000000600851F7800C0C3B300BD
:10E2C0001AFEB700E4BF2100C4F08800E26C02002F
:10E2D000000000000004E0001A003A00C0C3B300D0
:10E2E0001AFEB700E4BF2100C4F08800E26C02000F
:10E2F000000000000004E00012003A004809AE00EF
:10E30000100037000100200001007800E202020046
:10E31000000000008100E800811F78002322AF0088
:10E32000FEFF370020118800CF0078003001200068
:10E330000008E600F4FF3700AC68020000000000AF
:10E3400079003700FEDBBF0047E9B700FFDBBF0005
:10E3500048E9B70000DCBF0049E9B70001DCBF00B5
:10E360004AE9B70002DCBF004BE9B70003DCBF009D
:10E370004EE9B70004DCBF004FE9B70005DCBF0081
:10E3800051E9B70006DCBF0050E9B70007DCBF0069
:10E3900052E9B70008DCBF0053E9B70009DCBF0051
:10E3A00054E9B7000ADCBF0055E9B7000BDCBF0039
:10E3B00071E9B7000CDCBF0072E9B7000DDCBF00EB
:10E3C00073E9B7000EDCBF0056E9B7000FDCBF00F1
:10E3D00057E9B70010DCBF0058E9B70011DCBF00F7
:10E3E00059E9B70012DCBF005AE9B70013DCBF00DF
:10E3F0005BE9B70014DCBF005CE9B70015DCBF00C7
:10E400005DE9B70016DCBF005EE9B70017DCBF00AE
:10E410005FE9B70018DCBF0060E9B70019DCBF0096
:10E4200061E9B7001ADCBF0062E9B7001BDCBF007E
:10E4300063E9B7001CDCBF0064E9B7001DDCBF0066
:10E4400065E9B7001EDCBF0066E9B7001FDCBF004E
:10E4500067E9B70020DCBF0068E9B70021DCBF0036
:10E4600069E9B70022DCBF006AE9B70023DCBF001E
:10E470006BE9B70024DCBF006CE9B70025DCBF0006
:10E480006DE9B70026DCBF006EE9B70027DCBF00EE
:10E490006FE9B70028DCBF0070E9B70029DCBF00D6
:10E4A00074E9B7002ADCBF0075E9B7002BDCBF00B8
:10E4B00076E9B7002CDCBF0077E9B7002DDCBF00A0
:10E4C00078E9B7002EDCBF0079E9B7002FDCBF0088
:10E4D0007AE9B70030DCBF007BE9B70031DCBF0070
:10E4E00092E8B70032DCBF007CE9B70033DCBF0044
:10E4F0007DE9B70034DCBF007EE9B70035DCBF0042
:10E500007FE9B70036DCBF0080E9B70037DCBF0029
:10E5100081E9B70038DCBF0082E9B70039DCBF0011
:10E5200083E9B7008C28EF00CF02780000000600D6
:10E530005032EF005012F8005212F900211521005C
:10E5400002002000FD0009008058EB0041C8A9002E
:10E5500000000600851F7800645580004822DE0018
:10E56000E39A200003004200C4EA800000429000C9
:10E57000C4EA8800645580004822DE0061424200FF
:10E580000440780000E0B7000160EF00F40F2000C5
:10E59000110009000480D80001407800ADEAB700FE
:10E5A000ADCABF00AD49E30001003A004148A900EF
:10E5B00058DDBF0000E0B700CF0278000000060081
:10E5C000851F78002E7CEF004148AE000500370023
:10E5D000AA720200000000002EFCB700E4720400E2
:10E5E00000000000AE6AEF00CF02780000000600D5
:10E5F000851F780080C5B30082FFB7007459800082
:10E600004822DE0003AB20000300420014FC80001F
:10E610000042900014FC8800745980004822DE00FB
:10E62000614242000440780000E0B7000160EF0062
:10E63000F4072000110009000480D8000140780090
:10E640002FEBB7002FCBBF00AF4AE30001003A0029
:10E650004168A90082DFBF0000E0B700CF02780068
:10E6600000000600851F7800767FEF004168AE004D
:10E6700008003700F87202000000000076FFB700C3
:10E68000A0002000665C0200000000003673040059
:10E6900000000000306BEF00CF02780000000600A1
:10E6A000851F7800C500200003000900B51F780011
:10E6B00000F0A6000C0037000000EA000480A00073
:10E6C00004F0A60008003700801F7800D002200068
:10E6D0002322AF00FEFF3700201188004F00780092
:10E6E0000480A1000860ED008002EB008003780048
:10E6F0008404780004F0A1000404E00006003A005D
:10E7000009F0A70002003700050020000F003700C5
:10E71000050020000D003700E64252000A003900D3
:10E720000003200009F0A600000220002322AF0011
:10E73000FEFF3700201188008502E900FBFF3B0047
:10E74000550020000100370084027800640020009A
:10E750000580A7000402E80005E0A00009F0A7007A
:10E7600005F0A00008712200110009008883D8007C
:10E77000FC7302000000000081037800883E200046
:10E78000110009008883D800FC730200000000001B
:10E790008103780048062000110009008883D80012
:10E7A000FC7302000000000081037800A800200034
:10E7B000110009008883D800FC73020000000000EB
:10E7C0000980A60005003700D00220002322AF00F8
:10E7D000FEFF3700201188000980A10000032000FF
:10E7E00000C04000500188002322AF00FEFF370028
:10E7F0002011880022003700060320000000E000FE
:10E800000E003A0005E0A600160037000402E900F9
:10E810000524E100020032004200AF0000000600C3
:10E820000000E00005003A0005E0A6000D003700FA
:10E8300005F0A600060220000A00370005E0A1004E
:10E840000980A6000700370000057800D0022000EC
:10E850002322AF00FEFF3700201188000980A100AD
:10E860000A00780000404300811F78002322AF0097
:10E87000FEFF370020118800CF007800000006005E
:10E880002501200003000900CF127800CF02780094
:10E8900000000600851F7800787FEF00797FEF0089
:10E8A00000002000761FB4001040780079FFB70008
:10E8B000795FE200320032004829AE0008003700DC
:10E8C0002322AF00FEFF3700D4002000241188006F
:10E8D0002322AF00FEFF3700A4002000241188008F
:10E8E00010C0B30078FFB70078DFBF00C4FB800022
:10E8F0004822DE000024E100210035004829AE0056
:10E900001000370078DFBF000000FB00B4FB800080
:10E9100004004000904278000B60EF000500780092
:10E9200021702200AC6C0200000000002322AF0026
:10E93000FEFF37000402200024118800A6740400A2
:10E94000000000007E3E09000000000078DFBF00EC
:10E950000000FB00B4FB80000400400090427800FF
:10E96000054078003322AF00FEFF370034E2B700E5
:10E970003562EF00787FEC00747404000000000042
:10E98000CF02780000000600851F7800C500200037
:10E9900003000900B51F7800800378008404780024
:10E9A00004F0A1000400E00006003A0009F0A7000E
:10E9B00002003700050020000F003700050020008E
:10E9C0000D003700E64252000A0039000003200023
:10E9D00009F0A600000220002322AF00FEFF37004E
:10E9E000201188008502E900FBFF3B005500200054
:10E9F00001003700840278006400200005E0A000D8
:10EA000009F0A70005F0A00008712200110009001C
:10EA10008883D8003E750200000000008103780062
:10EA2000883E2000110009008883D8003E7502004E
:10EA30000000000081037800480620001100090052
:10EA40008883D8003E750200000000008103780032
:10EA5000A8002000110009008883D8003E7502003C
:10EA6000000000000003200000C040002322AF008F
:10EA7000FEFF370020118800190037000603200030
:10EA80000000E0000E003A0005E0A6000D0037008F
:10EA90000402E9000524E100020032004200AF0058
:10EAA000000006000000E00005003A0005E0A600B6
:10EAB0000400370005F0A600060220000100370020
:10EAC00005E0A10000404300811F78002322AF0031
:10EAD000FEFF370020118800CF00780000000600FC
:10EAE0002501200003000900CF127800CF02780032
:10EAF00000000600851F7800861F7800B03EEF00FA
:10EB0000B23EEF00AD1EA9004829AE000D0037004F
:10EB1000010020000100780006290200000000002A
:10EB20008100E800811F78002322AF00FEFF37003C
:10EB300020118800CF007800E00020000008E600E7
:10EB4000F4FF37004168AF002F00370084F58000E4
:10EB5000230320000320B8008002780074F58000B1
:10EB60000520E10022003E004829AE001E003700CB
:10EB700001002000010078002229020000000000AE
:10EB80008100E800811F78002322AF00FEFF3700DC
:10EB900020118800CF007800A00020000008E600C7
:10EBA000F4FF370070F5800004002000C4740200F8
:10EBB00000000000D100200001007800222902009E
:10EBC000000000008100E800811F78002322AF00D0
:10EBD000FEFF370020118800CF00780030012000B0
:10EBE0000008E600F4FF37000060EF00D9003700AE
:10EBF00020032000665C020000000000B03EEC0034
:10EC0000A27504000000000051F580000200200001
:10EC1000ACDEBF000160EF000000E90000800900E9
:10EC20008058EB004829AE000C0037002322AF00CB
:10EC3000FEFF370004022000241188002322AF00C9
:10EC4000FEFF3700D4022000241188002322AF00E9
:10EC5000FEFF370004022000241188004168AF0045
:10EC60000700370084F58000230320000320B8004C
:10EC70000003780074F580000620E100940036005F
:10EC80004168AE005F00370090F58000AA1EB40016
:10EC900080027800F872020000000000804A7800CC
:10ECA000AD1EAF002B00370090F58000AA1EB40007
:10ECB0001042780004C9B2000500320090F58000CF
:10ECC000AA1EB4001042780084C8B2001F003A00A7
:10ECD00000002000AA1EB4008002780090F5800099
:10ECE000AA1EB400904A78001400200094F5880011
:10ECF0004829AE001400370000002000AA1EB4000E
:10ED0000904278002322AF00FEFF3700B4052000B8
:10ED1000241188002322AF00FEFF370004022000E8
:10ED200024118800054078000160EF002170200068
:10ED3000AC6C0200000000002322AF00FEFF370091
:10ED40000402200024118800AD1EA80002770400F0
:10ED5000000000004829AE000C00370090F580004C
:10ED6000AA1EB40090427800054078000160EF00D0
:10ED700021702000AC6C0200000000002322AF00D4
:10ED8000FEFF3700040220002411880090F5800067
:10ED9000AA1EB40010427800F4CFB20011003A006D
:10EDA0004829AE000C0037002322AF00FEFF3700D9
:10EDB000D4052000241188002322AF00FEFF370075
:10EDC000A4002000241188002322AF00FEFF37009A
:10EDD000D40020002411880010C0B30000E0B70068
:10EDE0005C003700B23EEC00ACDEBF000160EF001B
:10EDF00094F580000020E1000200390000E0EF00FF
:10EE0000540037004168AF002F00370084F58000C0
:10EE1000230320000320B8008002780074F58000EE
:10EE20000520E10022003E004829AE001E00370008
:10EE300001002000010078002229020000000000EB
:10EE40008100E800811F78002322AF00FEFF370019
:10EE500020118800CF007800A00020000008E60004
:10EE6000F4FF370070F5800004002000C474020035
:10EE700000000000D10020000100780022290200DB
:10EE8000000000008100E800811F78002322AF000D
:10EE9000FEFF370020118800CF00780030012000ED
:10EEA0000008E600F4FF37000060EF00290037009B
:10EEB00020032000665C020000000000B03EEC0071
:10EEC00002770400000000002E760400000000001D
:10EED0004829AE001E003700010020000100780024
:10EEE00022290200000000008100E800811F780054
:10EEF0002322AF00FEFF370020118800CF007800EA
:10EF0000A00020000008E600F4FF370070F5800044
:10EF100004002000C474020000000000D1002000A2
:10EF20000100780022290200000000008100E800B2
:10EF3000811F78002322AF00FEFF370020118800D8
:10EF4000CF007800300120000008E600F4FF370011
:10EF50000060EF004F037800CF0278000000060049
:10EF6000851F78004829AE000D0037000100200001
:10EF700001007800BC280200000000008100E800C9
:10EF8000811F78002322AF00FEFF37002011880088
:10EF9000CF007800D00020000008E600F4FF370022
:10EFA000D0C0B300ACFEB700A4E9210054F588003E
:10EFB000981EF800AE1EF9007A75020000000000ED
:10EFC0000004E000220032009BDEBF000160EF0081
:10EFD0001084B200110032003080B2000F00320005
:10EFE0002082B200120032008085B200140032008C
:10EFF0008086B200120032001080B2001000320091
:10F000003080B2000E0032003083B2000C003200BB
:10F010003080B2000A0032000B00370010C0B3008D
:10F0200000E0B7000B003700247804000000000067
:10F0300000E0EF0007003700247804000000000023
:10F040002478040000000000D077040000000000D5
:10F050000060EF00CF02780000000600851F7800F6
:10F060006410280004F488001440200014F4880080
:10F070007400200024F4880086FEEF00941028001D
:10F0800044F488001460200054F488001400200028
:10F0900064F488000430200074F4880034F02F00F9
:10F0A00084F48800937EEF00E4F38000F447B2001C
:10F0B000044078007FFEB700E4F380004822DE00C1
:10F0C000F447B2000440780087FEB700F4F38000F4
:10F0D000F447B2000440780092FEB70084498000F3
:10F0E0006E24E1000A003A00925EE200080032005D
:10F0F000844480000960EF00939620000480410062
:10F1000010407800F047B2006840700092FEB700EF
:10F110007F5EE20006003A0010C0B3007FFEB70039
:10F1200030C0B3008FFEB700AE78040000000000CE
:10F130007CDEBF000048B200040820000024E1008B
:10F1400004003A0010C0B3008FFEB700AE78040090
:10F150000000000020C0B3008FFEB70024498000EB
:10F160007224E1000A0036007FDEBF0024498000DF
:10F170000024E10006003600F4F380004822DE009F
:10F180007224E1000200360024C9BF007FFEB700F0
:10F190007FDEBF008DFEB700875EE20006003A000A
:10F1A00030C0B30090FEB70010C0B30087FEB700B8
:10F1B000F2780400000000007DDEBF000048B200CD
:10F1C000040820000024E10004003A0010C0B3004D
:10F1D00090FEB700F27804000000000020C0B300E9
:10F1E00090FEB700244980004822DE006E24E10032
:10F1F0000B00360087DEBF00244980004822DE0075
:10F200000024E1000600360034F480004822DE00CD
:10F210006E24E1000200360025C9BF0087FEB7005A
:10F2200087DEBF008EFEB700844980006A24E100BB
:10F230004E00320024C9BF007F5EE30009003A009F
:10F2400027C9BF008F5EE30006003A0025C9BF0052
:10F25000875EE30003003A0028C9BF00905EE30028
:10F26000420032007FDEBF0024E9B7008FDEBF001E
:10F2700027E9B70087DEBF0025E9B70090DEBF00B1
:10F2800028E9B70074F480004822DE006324E1001E
:10F2900003003A0084F480006324E100240032007B
:10F2A0008C88A800327302000000000084E821006E
:10F2B000B4FB88004A74020000000000844980000A
:10F2C0006124E10003003200844980006524E100EC
:10F2D00006003A00843E2000C4F48800B0770200A3
:10F2E00000000000947904000000000084498000C0
:10F2F0006324E1000C003A0048A9AE000A00370080
:10F30000A40F2000C4F48800B077020000000000C1
:10F310004BC9BF0093FEB70093DEBF000160EF0052
:10F32000665C020000000000B279040000000000EA
:10F330008C88AE000B0037008C88A9003273020065
:10F340000000000084E82100B4FB88004A74020039
:10F3500000000000843E2000C4F48800B077020062
:10F36000000000003273020000000000925EE20024
:10F3700003003A00857EEF00E479040000000000FD
:10F3800092DEBF006740600092FEB7007EDEBF00E5
:10F390000048B200040820000024E10006003A0002
:10F3A00094F480000442B3000440780085FEB70066
:10F3B000E47904000000000094F480000443B300EA
:10F3C0000440780085FEB700855EE2002D00320023
:10F3D000844980006E24E10003003A008CA8AE004E
:10F3E00001003700360037003273020000000000D1
:10F3F00004E82100B4FB88004A7402000000000009
:10F400008CA8A800844980006124E1000600320035
:10F41000844980006524E1000300320084498000B3
:10F420006A24E10006003A00843E2000C4F488000B
:10F43000B0770200000000003E7A040000000000E7
:10F44000844980006324E1000C003A0048A9AE0022
:10F450000A003700A40F2000C4F48800B07702002F
:10F46000000000004BC9BF0093FEB70093DEBF0051
:10F470000160EF00665C0200000000005C7A04009E
:10F48000000000008CA8AE000B0037008CA8A9007B
:10F49000327302000000000004E82100B4FB880081
:10F4A0004A74020000000000843E2000C4F488007A
:10F4B000B07702000000000032730200000000007C
:10F4C000CF02780000000600851F78000A3FEF0099
:10F4D000077FEF000C1FA9004168AF002F00370025
:10F4E00054F88000230320000320B8008002780035
:10F4F00044F880000520E10022003E004829AE00CB
:10F500001E003700010020000100780022290200BF
:10F51000000000008100E800811F78002322AF0076
:10F52000FEFF370020118800CF007800A0002000E7
:10F530000008E600F4FF370040F8800004002000D7
:10F54000C474020000000000D10020000100780017
:10F5500022290200000000008100E800811F7800DD
:10F560002322AF00FEFF370020118800CF00780073
:10F57000300120000008E600F4FF37000060EF00D3
:10F58000D600370020032000665C02000000000067
:10F590000A3FEC006C7A04000000000021F88000B3
:10F5A0000200200006DFBF000160EF000000E9005C
:10F5B000008009008058EB004829AE000C0037009D
:10F5C0002322AF00FEFF3700040220002411880030
:10F5D0002322AF00FEFF3700D40220002411880050
:10F5E0002322AF00FEFF3700040220002411880010
:10F5F0004168AE009800370034F880004822DE00F1
:10F6000004007800041FB40080027800F872020041
:10F6100000000000804A78000C1FAF002A0037006D
:10F6200034F880004822DE0004007800041FB40093
:10F6300010427800E4CFB20021003A000000200020
:10F64000041FB4008002780034F880004822DE00F5
:10F6500004007800041FB400904A780010C0B30082
:10F6600007FFB7004829AE00140037000000200053
:10F67000041FB400904278002322AF00FEFF370041
:10F68000B4052000241188002322AF00FEFF3700BC
:10F690000402200024118800054078000160EF007A
:10F6A00021702000AC6C0200000000002322AF009B
:10F6B000FEFF370004022000241188000C1FA80060
:10F6C000C67B0400000000004829AE000E00370091
:10F6D00034F880004822DE0004007800041FB400E3
:10F6E00090427800054078000160EF002170200012
:10F6F000AC6C0200000000002322AF00FEFF3700C8
:10F70000040220002411880034F880004822DE0022
:10F7100004007800041FB40010427800F4CEB20058
:10F7200012003A004829AE000D0037000100200009
:10F7300001007800CA2A0200000000008100E800F1
:10F74000811F78002322AF00FEFF370020118800C0
:10F75000CF007800300020000008E600F4FF3700FA
:10F7600010C0B30000E0B7005C003700077FEC007A
:10F7700006DFBF0034F880004822DE000024E100EC
:10F780000200390000E0EF00540037004168AF008C
:10F790002F00370054F88000230320000320B80016
:10F7A0008002780044F880000520E10022003E003D
:10F7B0004829AE001E00370001002000010078003B
:10F7C00022290200000000008100E800811F78006B
:10F7D0002322AF00FEFF370020118800CF00780001
:10F7E000A00020000008E600F4FF370040F8800089
:10F7F00004002000C474020000000000D1002000BA
:10F800000100780022290200000000008100E800C9
:10F81000811F78002322AF00FEFF370020118800EF
:10F82000CF007800300120000008E600F4FF370028
:10F830000060EF002900370020032000665C020012
:10F84000000000000A3FEC00C67B0400000000003E
:10F85000F87A0400000000004829AE001E003700BE
:10F8600001002000010078002229020000000000B1
:10F870008100E800811F78002322AF00FEFF3700DF
:10F8800020118800CF007800A00020000008E600CA
:10F89000F4FF370040F8800004002000C474020028
:10F8A00000000000D10020000100780022290200A1
:10F8B000000000008100E800811F78002322AF00D3
:10F8C000FEFF370020118800CF00780030012000B3
:10F8D0000008E600F4FF37000060EF00CF02780078
:10F8E00000000600851F78004829AE000D00370093
:10F8F0000100200001007800DC2A02000000000066
:10F900008100E800811F78002322AF00FEFF37004E
:10F9100020118800CF007800B00020000008E60029
:10F92000F4FF3700D0C0B30006FFB70044EF21005A
:10F9300024F88800F21EF800081FF900647A02001B
:10F94000000000000004E00022003200F7DEBF00EB
:10F950000160EF000083B200090032003080B20085
:10F960000C0032006080B2000F003200C080B20094
:10F970000D0032008080B2000F0032000A00370014
:10F9800010C0B30000E0B70013003700E67C0400AD
:10F99000000000003049E20003003A0010C0B3004C
:10F9A00000E0B7000C00370000E0EF000A0037006D
:10F9B000E67C04000000000010C0B30000E0B700C7
:10F9C00005003700E67C040000000000927C040083
:10F9D000000000000060EF00CF0278000000060089
:10F9E000537FEF0094FA80006A24E10006003100A2
:10F9F0000403200093FA800004C0410053FFB700C5
:10FA00000C7D0400000000007403200093FA8000C5
:10FA100004C0410053FFB70053DFBF0000000600E1
:10FA2000851F7800D83EEF00E4F02F00D4F6880060
:10FA300004032300E4F6880014102800F4F688007C
:10FA40004403230004F788004403230014F78800CC
:10FA50004403230024F788004403230034F788007C
:10FA6000F0CEB300E8FEB70074F68000F447B200B1
:10FA700004407800D1FEB70074F680004822DE0012
:10FA8000F447B20004407800E9FEB700D0DEBF00C2
:10FA900067406000EAFEB700D15EE20023003A0052
:10FAA000E95EE20021003A00EA5EE2001F003A004F
:10FAB000344980004822DE0004C3B20007003A0047
:10FAC0004449800004C3B20004003A004449800065
:10FAD0004822DE0004C3B200140032003273020078
:10FAE00000000000A4ED2100B4FB88004A7402006D
:10FAF00000000000843E200094F78800727C020021
:10FB00000000000000C3B30027E9B70000C3B30042
:10FB100028E9B70000C3B30029E9B7008C88A90021
:10FB200060092000665C020000000000D15EE20077
:10FB300005003A00E95EE20003003A00EA5EE200F6
:10FB400001003A005701370084F680004822DE00A9
:10FB50006124E1002500360084F680004822DE00A2
:10FB60007824E1000600390080C1B300D1FEB7005F
:10FB7000F4032000C4F68800D87D040000000000D3
:10FB8000D1DEBF00D8FEB700D97EEF00C4F68000FA
:10FB9000F30320000320B8008002780005027800FB
:10FBA00083012000110009000382D800C0F68800FC
:10FBB000D8DEBF00D1FEB700244980007E24E100DA
:10FBC0000A003600D1DEBF00244980000024E10095
:10FBD0000600360084F680004822DE007E24E10024
:10FBE0000200360024C9BF00D1FEB70044F78000F0
:10FBF0004822DE006124E1002900360044F780003D
:10FC00004822DE007424E1000600390040C1B30040
:10FC1000E9FEB700F4032000C4F688002A7E040041
:10FC200000000000E9DEBF00D8FEB700D97EEF007B
:10FC3000C4F68000F30320000320B800800278009F
:10FC40000502780043012000110009000382D8005A
:10FC5000C0F68800D8DEBF00E9FEB7002449800066
:10FC60004822DE0003032000041CE1000C003100E8
:10FC7000E9DEBF00244980004822DE000024E100C4
:10FC80000700360044F780004822DE00030320000E
:10FC9000041CE1000200310025C9BF00E9FEB700E5
:10FCA00054F780006124E1001700360054F780000B
:10FCB0006724E1000600390070C0B300EAFEB70017
:10FCC000F4032000C4F68800807E040000000000D9
:10FCD000EADEBF00D8FEB700D97EEF00C4F6800090
:10FCE000F30320000320B8008002780005027800AA
:10FCF00073002000110009000382D800C0F68800BC
:10FD0000D8DEBF00EAFEB700D15EE20004003A0090
:10FD100000C3B300EBFEB700A67E040000000000A5
:10FD2000CEDEBF000048B200040820000024E1003D
:10FD300004003A0020C3B300EBFEB700A67E040027
:10FD40000000000010C3B300EBFEB700E95EE20064
:10FD500004003A0000C3B300ECFEB700C87E040004
:10FD600000000000CFDEBF000048B2000408200001
:10FD70000024E10004003A0010C3B300ECFEB70019
:10FD8000C87E04000000000020C3B300ECFEB700F2
:10FD9000EA5EE20004003A0000C3B300EDFEB700E3
:10FDA000EA7E040000000000D0DEBF000048B20080
:10FDB000040820000024E10004003A0010C3B3004E
:10FDC000EDFEB700EA7E04000000000020C3B3008F
:10FDD000EDFEB70054F780004822DE0014C3B200E5
:10FDE00008003A00F403200083F68000C819DE0002
:10FDF00003405200D4FEB700D57EEF001A7F040006
:10FE00000000000054F780004822DE0024C3B20046
:10FE100006003A0000042000D15EB400D4FEB70012
:10FE2000D57EEF001A7F04000000000004042000CB
:10FE3000A4F6880064F7800014C3B20008003A00FA
:10FE4000F403200043F78000C819DE00034052008D
:10FE5000D2FEB700D37EEF00467F04000000000012
:10FE600064F7800024C3B20006003A0000042000BA
:10FE7000E95EB400D2FEB700D37EEF00467F0400F7
:10FE8000000000000404200094F6880064F780005D
:10FE90004822DE0024C3B20007003A00F403200029
:10FEA00053F7800003405200D6FEB700D77EEF0024
:10FEB000747F04000000000064F780004822DE0028
:10FEC00014C3B20006003A0000042000EA5EB40049
:10FED000D6FEB700D77EEF00747F0400000000005C
:10FEE00004042000B4F68800D6DEBF000160EF00F5
:10FEF0004400DE00EF426000521FF800E5FF9F0063
:10FF0000521FF900F07C020000000000E0FEB70084
:10FF1000D6DEBF00EF426000521FF800E5FF9F00F1
:10FF2000521FF900F07C020000000000E1FEB70063
:10FF3000D2DEBF000160EF004400DE00EF4260004F
:10FF4000521FF800E5FF9F00521FF900F07C0200ED
:10FF500000000000E4FEB700D2DEBF00EF42600008
:10FF6000521FF800E5FF9F00521FF900F07C0200CD
:10FF700000000000E5FEB700D4DEBF000160EF0026
:10FF80004400DE00EF426000521FF800E5FF9F00D2
:10FF9000521FF900F07C020000000000E6FEB700EE
:10FFA000D4DEBF00EF426000521FF800E5FF9F0063
:10FFB000521FF900F07C020000000000E7FEB700CD
:10FFC00024C9BF00D15EE30017003A0027C9BF0073
:10FFD000EB5EE30014003A0025C9BF00E95EE300D0
:10FFE00011003A0028C9BF00EC5EE3000E003A00A1
:10FFF00026C9BF00EA5EE3000B003A0029C9BF0032
:020000040001F9
:10000000ED5EE30008003A00549380004822DE00D1
:100010006324E10001003600220037006B72EC001F
:100020002E800400000000006B72EF00D1DEBF00E4
:1000300024E9B700EBDEBF0027E9B700E9DEBF0027
:1000400025E9B700ECDEBF0028E9B700EADEBF0013
:1000500026E9B700EDDEBF0029E9B7008C88AE00C5
:100060000500370060092000665C02000000000007
:100070003E800400000000008C88A800327302005B
:1000800000000000A4ED2100B4FB88004A740200C7
:1000900000000000047D200094F78800727C0200BC
:1000A00000000000CF02780000000600851F7800E5
:1000B00084F02F00E4F4880004032300F4F48800A3
:1000C0000400260004F588000403230014F58800CA
:1000D000F0CEB300A4FEB70074F02F0034F5880012
:1000E0000403230044F5880004202A0054F5880006
:1000F00004F32E0064F5880094F02F0074F5880056
:100100000403230084F588000400250094F588008A
:10011000B43EEF0004F02E00B4F5880094F02F00F8
:10012000C4F5880004032300D4F5880004102500DA
:10013000E4F58800BE3EEF0004F02E0004F68800CF
:1001400084F02F0014F688000403230024F68800AE
:1001500004402B0034F688001403200044F6880085
:10016000F0CEB300CAFEB700844980007024E100DD
:1001700003003200844980007124E10009003A0044
:1001800094DEBF00CEFEB70095DEBF00CFFEB70005
:1001900096DEBF00D0FEB700107D02000000000018
:1001A00010013700A4F48000F447B2000440780046
:1001B00097FEB700A4F480004822DE00F447B200A6
:1001C00004407800A5FEB700B4F48000F447B20004
:1001D00004407800CBFEB700CB5EE2000D003A0091
:1001E000444980004822DE0004C3B2000900320006
:1001F000327302000000000064EA2100B4FB8800B2
:100200004A74020000000000ACDEBF0029E9B7001C
:100210008CA8A900975EE20014003A00A55EE200F7
:1002200012003A00344980004822DE0004C3B200C4
:1002300003003A004449800004C3B2000B003200BE
:100240003273020000000000C4E92100B4FB880002
:100250004A74020000000000A2DEBF0027E9B700D8
:10026000A3DEBF0028E9B7008C88A900975EE200F2
:1002700005003A00A55EE20003003A00CB5EE20012
:1002800001003A00D7003700975EE20004003A0010
:1002900000C3B300A2FEB7006681040000000000A6
:1002A00094DEBF000048B200040820000024E100F2
:1002B00004003A0020C3B300A2FEB7006681040028
:1002C0000000000010C3B300A2FEB700A55EE2006C
:1002D00004003A0000C3B300A3FEB7008881040005
:1002E0000000000095DEBF000048B20004082000B6
:1002F0000024E10004003A0010C3B300A3FEB700DD
:10030000888104000000000020C3B300A3FEB700F2
:10031000A5DEBF000160EF00000278007E20B8007B
:1003200080027800E8824200C5F4880097DEBF00B2
:100330000160EF00140220000020B8008002780065
:10034000E8824200D5F48800D4F480006A20E100FD
:1003500002003100A4002000D4F48800D4F480000E
:10036000033220000418E1000200310004322000B2
:10037000D4F48800C4F480006A20E1000200310057
:10038000A4002000C4F48800C4F48000E326200008
:100390000418E10002003100E4262000C4F48800C3
:1003A0009BDEBF00EF426000521FF800E5FF9F0098
:1003B000521FF900F07C020000000000B4FEB700FC
:1003C0009ADEBF000160EF004400DE00EF426000F3
:1003D000521FF800E5FF9F00521FF900F07C020059
:1003E00000000000B5FEB7009ADEBF00EF426000DB
:1003F000521FF800E5FF9F00521FF900F07C020039
:1004000000000000B6FEB70099DEBF00EF426000BA
:10041000521FF800E5FF9F00521FF900F07C020018
:1004200000000000BEFEB70098DEBF000160EF00D4
:100430004400DE00EF426000521FF800E5FF9F001D
:10044000521FF900F07C020000000000BFFEB70060
:1004500098DEBF00EF426000521FF800E5FF9F00EA
:10046000521FF900F07C020000000000C0FEB7003F
:10047000975EE2000F00320014F5800004C3B20062
:100480000C0032008C88A80024C9BF00975EE300EE
:100490000800320097DEBF0024E9B7003273020083
:1004A00000000000E4EA2100B4FB88004A74020066
:1004B00000000000A55EE2001000320014F580008C
:1004C0004822DE0004C3B2000C0032008C88A80071
:1004D00025C9BF00A55EE30008003200A5DEBF000D
:1004E00025E9B700327302000000000084EB210010
:1004F000B4FB88004A7402000000000028C9BF0055
:10050000A35EE30003003A0027C9BF00A25EE30038
:100510000A003200A2DEBF0027E9B700A3DEBF0059
:1005200028E9B7003273020000000000C4E921008E
:10053000B4FB88004A74020000000000CB5EE200B9
:100540002800320096DEBF000048B20004082000F8
:100550000024E10004003A0020C3B300ACFEB70061
:10056000B88204000000000010C3B300ACFEB70066
:100570008CA8A80026C9BF00CB5EE3000E003200A5
:10058000CBDEBF0026E9B700CBDEBF0067406000CE
:10059000004278000443B30004407800C9FEB7006D
:1005A000327302000000000024EC2100B4FB88003C
:1005B0004A7402000000000029C9BF00AC5EE300DD
:1005C00008003200ACDEBF0029E9B7003273020038
:1005D0000000000064EA2100B4FB88004A740200B5
:1005E00000000000CF02780000000600851F7800A0
:1005F000C500200003000900B51F78000202B80002
:1006000003F0A600020037000383B90001003700A1
:100610000303B8004200A9008502430060844B0038
:1006200001F0A60002003700028BB900010037007C
:10063000020BB80085024B0008844B000980B00013
:10064000038BB90008044B0087834C0087017800B6
:10065000080178008500780004007800250120005A
:1006600003000900CF127800CF02780000000600D6
:10067000851F7800C500200003000900B51F780021
:10068000090020004300AF0019002000891F7800F6
:100690008384680001F0A600060037000000EA002D
:1006A0000100320002003A008100EA000100370038
:1006B0008180EA0003F0A600060037000201EA008C
:1006C0000100320002003A008301EA000100370015
:1006D0008381EA0003026900150032000002EB008A
:1006E0008002EB000003EB008003EB000802200017
:1006F0004200A9000080D2008180D2000482D20092
:100700008582D2000328E10001003A0002A0E10046
:10071000030039000202520083825A004200A800FE
:100720000683D2008783D2000804E900F0FF3A0074
:1007300009F0A600070037000600EA0001003200B9
:1007400002003A008700EA00050037008780EA00CF
:1007500003003700870078000600780000003700AB
:10076000CF0478000900E000010032000400BE0060
:100770002501200003000900CF127800CF02780085
:1007800000000600851F7800861F7800871F78000C
:1007900014002000F4FB8800803FEF00837FEF000F
:1007A000847FEF00C4FB80006020E1000E003C006D
:1007B00003003500B4FB80006020E1000A00310036
:1007C00010C0B30083FFB700B0FB8000C1FB800006
:1007D000F2FF2F00F3FF2F00F6820200000000005E
:1007E000B0FB8800C1FB88007E1FE20002003A00D7
:1007F000801FE200310032004300A900B0FB8000FE
:10080000C1FB8000D2FB800003002000388302007F
:1008100000000000F0FB880001FC880024FC800040
:100820000960EF00040078007C1FB40080027800AB
:100830004300A800B0FB8000C1FB8000D2FB800019
:100840000300200038830200000000000003BE0007
:100850000403200004004300E0834B00870078007D
:10086000804A780024FC80000960EF0004007800D2
:100870007C1FB400940320001024E1000800310024
:1008800024FC80000960EF00040078007C1FB400A5
:100890008002780015427800674242008442980046
:1008A000847FEC007E1FF800761FF900801FF8009F
:1008B000781FF900F48304000000000014FC80009D
:1008C0004822DE006124E10008003A0024FC800098
:1008D0000960EF00040078007C1FB40080027800FB
:1008E000D0C2B300804A7800847FEC00827FEF00A2
:1008F00084DFBF000160EF004100DE0014FC8000D7
:100900000024E1001F003D0014FC80000960EF009E
:10091000040078007C1FB4001040780085FFB70009
:1009200014FC80000960EF00040078007C1FB40014
:100930008002780024FC800013FC800003405200F9
:10094000614050000080FB00E4FB80000400400098
:10095000904A780024FC800013FC80000340520081
:10096000614050000080FB00E4FB800084024000F6
:1009700085DFBF00804A7800827FEC007884040025
:100980000000000024FC80000960EF0004007800F3
:100990007C1FB40080027800804AEB007C1FF800C6
:1009A0000000F900CF0378004F037800CF027800F1
:1009B00000000600851F7800761FF800781FF900F8
:1009C000C0FB80001004E00003003200783FEC0020
:1009D000E084040000000000C4FB8000B3FB800042
:1009E00003005200CF02780000000600851F780047
:1009F000583FEF0054302200D4FA88000405230049
:100A0000E4FA880004D02000F4FA88005430220070
:100A100004FB88004405230014FB880004D0200058
:100A200024FB88005430220034FB8800A4052300F6
:100A300044FB880004D0200054FB8800A4FA800006
:100A4000F447B2000440780057FFB700B4FA8000C2
:100A50004822DE006124E10014003600B4FA800070
:100A60004822DE007824E1000200360080C1B30095
:100A700057FFB70057DFBF0058FFB700597FEF009F
:100A8000C4FA8000130320000320B800800278001D
:100A90000502780083012000110009000382D800BC
:100AA000C0FA880058DFBF0057FFB700A4FA8000E3
:100AB0004822DE00F447B200044078006CFFB70023
:100AC00064FB80006124E1001300360064FB8000B9
:100AD0007424E1000200360040C1B3006CFFB7008F
:100AE0006CDFBF0058FFB700597FEF00C4FA8000E9
:100AF000130320000320B80080027800050278006C
:100B000043012000110009000382D800C0FA8800C8
:100B100058DFBF006CFFB700B4FA80007447B20022
:100B2000044078006DFFB7006DDFBF0067406000D4
:100B30006104E1000F0036006DDFBF000160EF00CF
:100B400067006000C0FA8800C4FA80001303200028
:100B50000320B800800278000502780073002000AE
:100B6000110009000382D800C0FA880058DFBF00D6
:100B70006DFFB700E1F6210002002000030009002C
:100B80008058EB00575FE20006003A0050C3B30004
:100B90005DFFB70000C3B3005EFFB70072860400BC
:100BA0000000000054DFBF000048B200040820002D
:100BB0000024E10028003A0024032000B3FA80005A
:100BC000C819DE000340520057FFB70057DFBF00CF
:100BD00076FFB700777FEF00783FEF00A40020009A
:100BE000D4FB8800E4F62100E4FB8800C283020005
:100BF00000000000800278000500E00010003200D4
:100C0000E4F62100B4FB8800DA8402000000000052
:100C10006104E100060036006EDFBF005DFFB70033
:100C20006FDFBF005EFFB7001C86040000000000FD
:100C30006EDFBF005EFFB7002886040000000000E2
:100C400050C3B3005DFFB70000C3B3005EFFB70041
:100C5000728604000000000020032000577FB400CB
:100C600057DFBF0076FFB700777FEF00783FEF00D8
:100C7000A4002000D4FB8800E4F62100E4FB8800F7
:100C8000C283020000000000800278000500E0003E
:100C900010003200E4F62100B4FB8800DA84020080
:100CA000000000006104E100060036006EDFBF00B6
:100CB0005DFFB7006FDFBF005EFFB7006686040010
:100CC000000000006EDFBF005EFFB7007286040008
:100CD0000000000050C3B3005DFFB70000C3B300C5
:100CE0005EFFB700A4F52100B4FB88004A7402003F
:100CF0000000000032730200000000006C5FE200A0
:100D000006003A0050C3B30063FFB70000C3B3004E
:100D100064FFB7002C8704000000000055DFBF000F
:100D20000048B200040820000024E10025003A0039
:100D3000200320006C7FB4006CDFBF0076FFB7009B
:100D4000777FEF00783FEF00A4002000D4FB8800FD
:100D5000E4F62100E4FB8800C283020000000000EA
:100D6000800278000500E00010003200E4F6210067
:100D7000B4FB8800DA840200000000006104E10096
:100D8000060036006EDFBF0063FFB7006FDFBF00F5
:100D900064FFB700D2860400000000006EDFBF00D1
:100DA00064FFB700DE8604000000000050C3B300FB
:100DB00063FFB70000C3B30064FFB7002C870400D3
:100DC000000000002403200063FB80000340520069
:100DD0006CFFB7006CDFBF0076FFB700777FEF00D6
:100DE000783FEF00A4002000D4FB8800E4F6210047
:100DF000E4FB8800C283020000000000800278004B
:100E00000500E00010003200E4F62100B4FB880089
:100E1000DA840200000000006104E10006003600F0
:100E20006EDFBF0063FFB7006FDFBF0064FFB70076
:100E300020870400000000006EDFBF0064FFB700E1
:100E40002C8704000000000050C3B30063FFB7000C
:100E500000C3B30064FFB70004F62100B4FB8800B0
:100E60004A7402000000000032730200000000001B
:100E70006D5FE20006003A0050C3B30069FFB7009F
:100E800000C3B3006AFFB700E88704000000000059
:100E900056DFBF000048B200040820000024E10033
:100EA00025003A00200320006D7FB4006DDFBF00F5
:100EB00076FFB700777FEF00783FEF00A4002000B7
:100EC000D4FB8800E4F62100E4FB8800C283020022
:100ED00000000000800278000500E00010003200F1
:100EE000E4F62100B4FB8800DA8402000000000070
:100EF0006104E100060036006EDFBF0069FFB70045
:100F00006FDFBF006AFFB7008C870400000000009D
:100F10006EDFBF006AFFB700988704000000000082
:100F200050C3B30069FFB70000C3B3006AFFB70046
:100F3000E8870400000000002403200063FB800019
:100F4000C819DE00034052006DFFB7006DDFBF001F
:100F500076FFB700777FEF00783FEF00A400200016
:100F6000D4FB8800E4F62100E4FB8800C283020081
:100F700000000000800278000500E0001000320050
:100F8000E4F62100B4FB8800DA84020000000000CF
:100F90006104E100060036006EDFBF0069FFB700A4
:100FA0006FDFBF006AFFB700DC87040000000000AD
:100FB0006EDFBF006AFFB700E88704000000000092
:100FC00050C3B30069FFB70000C3B3006AFFB700A6
:100FD00064F62100B4FB88004A740200000000009F
:100FE0003273020000000000CF027800000006000B
:100FF000851F78008C28A9008C08A9008C48A900BE
:101000009048E20084003200844480000960EF00D0
:101010003389200004804100104078003049E3000B
:101020007D003A0030C9BF000160EF001080B200BF
:101030001F0032007080B2001D0032004080B200FC
:101040001B0032001080B200190032006080B20034
:1010500017003200D080B200150032001080B200BC
:10106000130032006080B200110032008080B200B4
:101070000F0032003080B2000D003200A080B200BC
:101080000B0032004080B20009003200A081B200A3
:101090000E0032001080B2000C003200D081B2008D
:1010A000110032001080B200160032001C00370020
:1010B0007C7EEF007D7EEF007E7EEF002E780200CA
:1010C000000000009088040000000000CE7EEF00C9
:1010D000CF7EEF00D07EEF00107D02000000000008
:1010E0009088040000000000947EEF00957EEF00E1
:1010F000967EEF00568002000000000090880400F9
:1011000000000000547FEF00557FEF00567FEF0096
:10111000F684020000000000908804000000000037
:10112000844480000960EF00B3892000848241007C
:1011300031C9BF00804A7800844480000960EF0014
:10114000B38A20008482410046C9BF0080429800D3
:1011500090C8BF000160EF004100DD00448D200019
:1011600084024000D44980008402980084448000B6
:101170000960EF0043972000048041001040780090
:10118000704060000004E00023003A0090C8BF00F7
:101190000160EF004100DD00448C2000840240002B
:1011A000E44980008402980090C8BF000160EF000D
:1011B0004100DD00448F200084024000044A80008A
:1011C0008402980090C8BF000160EF004100DD007C
:1011D0004490200084024000144A80008402980059
:1011E00090C8BF000160EF004100DD00448E200088
:1011F00084024000F44980008402980090C8BF0037
:101200000160EF004100DD004491200084024000B5
:10121000244A800084029800A0002000665C02003E
:1012200000000000CF0278000000060082002000CD
:101230001E00090000000000E2C2A900DEC2A900F1
:101240001F0009000000000081C0D200C422A900D4
:101250004200AF00C022A8004200AE00C022A90098
:10126000DEC2A800E0C2AE00FEFF37000201E900C6
:10127000EFFF3A001E00090000000000E2C2A900D2
:10128000DEC2A90000000000C022A8001F00090063
:10129000000000001F00090000000000DEC2A800DE
:1012A000E0C2AE00FEFF37001F0009000000000092
:1012B00000002000C222AF000000A000E2C2A9008E
:1012C000DEC2A900C422A900C022A90000000600B5
:1012D000851F78004E3EEF00C022A8001E000900C6
:1012E00000000000DEC2A8001F000900000000008E
:1012F000E0C2AE00FEFF3700C422A900C022A90050
:101300001E00090000000000E2C2A900DEC2A90020
:10131000A1C9B300168902000000000051F280004C
:1013200016890200000000004E3EEF004BDEBF00B9
:101330000160EF0074F280000020E100090031003C
:1013400070F280004C1EB400904278008540780016
:1013500016890200000000004E3EEC009689040051
:1013600000000000C022A90000000000DEC2A800AA
:10137000E0C2AE00FEFF37001E00090000000000C2
:101380000100090000000000C022A8001E000900A2
:1013900000000000BE00090000000000CF0278003D
:1013A00000000600851F7800861F7800447EEF004D
:1013B000451EA900DAC2AF00010037001C02370049
:1013C0008D48AE00030037008C68AE000100370086
:1013D000170237008CE8AE0003003700451EA80056
:1013E0001E8A0400000000008C68AE000300370075
:1013F000451EA9001E8A0400000000004809AE0036
:101400000D0037000100200001007800B013020039
:10141000000000008100E800811F78002322AF0057
:10142000FEFF370020118800CF00780070002000F8
:101430000008E600F4FF3700FD01370044F18000AA
:10144000E4CEB2000700320044F18000F4CFB200D5
:101450000400320028DEBF006F4060006204E1003B
:10146000D0003A0028DEBF006F4060006204E10057
:101470006A003A008D28AE000F00370002002000FD
:10148000C1E2210002007800C61302000000000043
:10149000805878000201E8000004E0004220AE001D
:1014A000F8FF3700C4E2210054F288000C6B020000
:1014B00000000000DE0137008D88AE000400370018
:1014C0008DA8AF00010037008DA8A800D801370013
:1014D0007008E20004003A00640920008443880098
:1014E000888A0400000000002A09E20004003A0093
:1014F0002C09E20002003A002E09E200040032004A
:101500008DA8AF00010037008DA8A800C8013700E2
:101510003A4FE2000A0032003A6FED003ACFBF00C6
:10152000D47980004822DE000024E1000200360069
:101530003ACFBF003BEFB700028B04000000000071
:101540008D88AF002E0037008D88A8008DA8AF00D1
:10155000010037008DA8A8004809AE002800370018
:101560000100200001007800E613020000000000E6
:101570008100E800811F78002322AF00FEFF3700C2
:1015800020118800CF007800600120000008E600EC
:10159000F4FF370039CFBF000160EF0004002000E6
:1015A000C4740200000000009101200001007800D6
:1015B000E6130200000000008100E800811F7800AF
:1015C0002322AF00FEFF370020118800CF007800F3
:1015D000200220000008E600F4FF37003ACFBF00E9
:1015E0000160EF0004002000C4740200000000004D
:1015F0002322AF00FEFF3700940220002411880050
:101600008B0137002AC9BF0029FEB7002CC9BF00D3
:101610002AFEB7002EC9BF002BFEB7004809AE0056
:10162000410037008042EB00451EAF008502E80014
:101630002322AF00FEFF3700A40020002411880001
:101640002322AF00FEFF3700D400200024118800C1
:101650002322AF00FEFF37008402200024118800FF
:10166000054078000160EF0004002000C47402000F
:101670000000000051002000010078001A14020050
:10168000000000008100E800811F78002322AF00E5
:10169000FEFF370020118800CF00780040012000B5
:1016A0000008E600F4FF370028DEBF000160EF000D
:1016B00021702200AC6C0200000000002322AF0069
:1016C000FEFF3700040220002411880029DEBF003D
:1016D0000160EF0021702200AC6C020000000000ED
:1016E0002322AF00FEFF37000402200024118800EF
:1016F0002ADEBF000160EF0021702200AC6C020006
:10170000000000002322AF00FEFF3700040220008B
:10171000241188002BDEBF000160EF002170220041
:10172000AC6C02000000000028DEBF0040FEB700E5
:1017300029DEBF0041FEB7002ADEBF0042FEB7002F
:101740002BDEBF0043FEB7008CE8AE000900370077
:101750004A7EEF0040C0B3004BFEB70004E4210016
:1017600064F288006889020000000000CE8B04004B
:10177000000000008C68AE000800370020C0B300F5
:101780004AFEB70040C0B3004BFEB70004E421009E
:1017900064F288006889020000000000188E0400CE
:1017A0000000000094798000F30F20000418E1008D
:1017B000340031004809AE0031003700010020003C
:1017C000010078004C140200000000008100E800D5
:1017D000811F78002322AF00FEFF37002011880010
:1017E000CF007800D00120000008E600F4FF3700A9
:1017F00028DEBF000160EF0021702200AC6C020007
:10180000000000002322AF00FEFF3700040220008A
:101810002411880029DEBF000160EF002170220042
:10182000AC6C0200000000002322AF00FEFF370076
:1018300004022000241188002ADEBF000160EF00AE
:1018400021702200AC6C0200000000002322AF00D7
:10185000FEFF370004022000241188002BDEBF00A9
:101860000160EF0021702200AC6C0200000000005B
:101870002322AF00FEFF37009402200024118800CD
:10188000EB00370028DEBF006F40600044FEB70069
:101890008CC8AF00B20037008D28AE00B000370012
:1018A00024F280006124E1005B003A002A5EE2003D
:1018B00057003A0044F180004822DE006E24E10027
:1018C0000400390044F180004822DE007424E10065
:1018D0004F00360002002000C1E221000200780023
:1018E000C613020000000000805878000201E800E2
:1018F0000004E0004220AE00F8FF3700C4E22100FF
:1019000054F288000C6B0200000000004809AE0091
:101910003E0037000100200001007800881402001A
:10192000000000008100E800811F78002322AF0042
:10193000FEFF370020118800CF00780090022000C1
:101940000008E600F4FF370028DEBF000160EF006A
:1019500021702200AC6C0200000000002322AF00C6
:10196000FEFF3700040220002411880029DEBF009A
:101970000160EF0021702200AC6C0200000000004A
:101980002322AF00FEFF370004022000241188004C
:101990002ADEBF000160EF0021702200AC6C020063
:1019A000000000002322AF00FEFF370004022000E9
:1019B000241188002BDEBF000160EF00217022009F
:1019C000AC6C0200000000009103200001007800D0
:1019D00088140200000000008100E800811F7800E8
:1019E0002322AF00FEFF370020118800CF007800CF
:1019F000500420000008E600F4FF37006044800037
:101A000041702200AC6C020000000000880037002A
:101A1000B08D04000000000024F280006C24E1007E
:101A20004F00310002002000C1E2210002007800D6
:101A3000C613020000000000805878000201E80090
:101A40000004E0004220AE00F8FF3700C4E22100AD
:101A500054F288000C6B0200000000004809AE0040
:101A60003E0037000100200001007800D61402007B
:101A7000000000008100E800811F78002322AF00F1
:101A8000FEFF370020118800CF0078009002200070
:101A90000008E600F4FF370028DEBF000160EF0019
:101AA00021702200AC6C0200000000002322AF0075
:101AB000FEFF3700040220002411880029DEBF0049
:101AC0000160EF0021702200AC6C020000000000F9
:101AD0002322AF00FEFF37000402200024118800FB
:101AE0002ADEBF000160EF0021702200AC6C020012
:101AF000000000002322AF00FEFF37000402200098
:101B0000241188002BDEBF000160EF00217022004D
:101B1000AC6C02000000000091032000010078007E
:101B2000D6140200000000008100E800811F780048
:101B30002322AF00FEFF370020118800CF0078007D
:101B4000500420000008E600F4FF370060448000E5
:101B500041702200AC6C020000000000340037002D
:101B60003A4FE20010003A0044DEBF000160EF008F
:101B7000C080B200050032001080B20003003200C5
:101B8000C080B2000300320006003700D48D04008C
:101B9000000000002A5EE20002003200D48D040042
:101BA000000000002200370024F280006224E100DF
:101BB0000A00360024F280006C24E10007003100A6
:101BC0007008E20004003A006409200084438800A1
:101BD000EE8D0400000000001500370031CBBF007F
:101BE0000160EF004200DD0024B3200084024000C9
:101BF00028DEBF00B042980029DEBF00A042980056
:101C00002ADEBF00904298002BDEBF00804A780099
:101C1000322FEC00A0798000947980000020E10050
:101C200002003600320FF800340FF900316BEC007F
:101C30004F037800CF02780000000600851F78006F
:101C40008C68AE000E0037008D08AF000A00370028
:101C5000D0C8B30028FEB70036DCBF0029FEB700AD
:101C600037DCBF002AFEB70038DCBF002BFEB70010
:101C7000D2890200000000005C8E04000000000019
:101C80008CE8AE000C0037008D08AF000A0037006A
:101C9000D0CCB30028FEB70036DCBF0029FEB70069
:101CA00037DCBF002AFEB70038DCBF002BFEB700D0
:101CB000D289020000000000CF0278000000060078
:101CC000851F7800861F7800871F7800F88702003C
:101CD000000000002E1CAF0002003700CB02A9005C
:101CE00001003700CB02A8002E3CAF0002003700F5
:101CF000CB22A90001003700CB22A8002E5CAF0048
:101D000002003700CB42A90001003700CB42A800F7
:101D100050002000665C02000000000032730200E8
:101D2000000000002EDCBF000000FB003489200012
:101D300004004000844980000042900084498800EB
:101D40003229EF003429EF003629EF003829EF005F
:101D50002EDCBF0090E8B7002EDCBF000000FB00C7
:101D6000B4892000040040001040780031E9B70039
:101D70002EDCBF000000FB00B48A200004004000FD
:101D8000344A800000429000344A88002EDCBF00B4
:101D90000000FB00000278006220B800448D2000A3
:101DA00004004000901F78003A09F9008444800044
:101DB0000960EF0043972000048041001040780044
:101DC000704060000004E00028003A002EDCBF00F4
:101DD0000000FB00000278006220B800448C200064
:101DE00004004000901F78003C09F9002EDCBF0081
:101DF0000000FB00000278006220B800448F200041
:101E000004004000901F78004009F9002EDCBF005C
